:100000000C9486090C94B7090C94B7090C94B709A1
:100010000C94B7090C94B7090C94B7090C94B70960
:100020000C94B7090C94B7090C94B7090C94B70950
:100030000C94B7090C94B7090C94B7090C94093EB9
:100040000C94B7090C94B7090C94B7090C94B70930
:100050000C94B7090C94B7090C94B7090C943F6B36
:100060000C94B7090C948E5F0C94645F0C94B709E0
:100070000C94B7090C94B7090C94B7090C94B70900
:100080000C94B7090C94B7090C94B7090C94B709F0
:100090000C9454600C94C45F0C940B600C94AA24D0
:1000A0000C94B7090C94B7090C94B7090C94B709D0
:1000B0000C94B7090C94B7090C94B7090C94B709C0
:1000C0000C94B7090C94B7090C94B7090C942E5FE3
:1000D0000C94045F0C94B7090C94B7090C94B709FD
:1000E0000C94B709580B0D0B1B0B580B580B660BD8
:1000F000740B520B580B580B6D0E720E770E810E4F
:100100008B0E040F950E9D0EA50EAF0EB90EC30EED
:10011000D20EDC0E040FE60EF00EFA0E0A11FC10E1
:10012000FC100A110A110E111C111C110A110A11DE
:100130001916F415341634163416341634163416CB
:100140003416341634168312521573156C155D155A
:10015000341634163416341634163416341608167B
:100160001C1C101C101C1C1C1C1CF71B041C041C3D
:100170001C1C1C1C1F2D222D3A2D512D9A2DAD2DEE
:10018000CD2D0A3B0A3B0A3B0A3B073B073B0E3B94
:100190000E3B0E3B0E3B0E3B0E3B0E3B0E3B073B1E
:1001A000073B0E3B0E3B0E3B0E3B0E3B0C3B0A3B14
:1001B0000665F364F36406650665066511651165F9
:1001C00006650665566852685268566856685668ED
:1001D0005F68206856685668826A856A746A786AB9
:1001E0007E6ABC6A896A8D6A936A976A9B6AA16A09
:1001F000A56AA96ABC6AAF6AB36AB76A076342367E
:10020000B79BD8A71A39685618AEBAAB558C1D3CA7
:10021000B7CC5763BD6DEDFD753EF6177231BF006B
:100220000000803F08000000BE922449123EABAAA5
:10023000AA2ABECDCCCC4C3E00000080BEABAAAA00
:10024000AA3E00000000BF000000803F0000000048
:1002500000084178D3BB4387D1133D190E3CC3BD81
:100260004282AD2B3E68EC8276BED98FE1A93E4C2E
:1002700080EFFFBE01C4FF7F3F00000000000C9430
:10028000793C0C941F2D0C94E42A0C94786A0C94FD
:10029000BA230C94222D0C9478760C94A8650C94B7
:1002A000826A0C946A410C94810E0C94805C0C94CC
:1002B000F00E0C94572B0C947E6A0C948D230C94A6
:1002C000D6410C94A5650C940A2C0C94172A0C9416
:1002D000C22A0C94AF0E0C948E230C9452150C94DD
:1002E000C30E0C94B2230C94CE430C9473150C944F
:1002F000B05E0C941A2C0C94283C0C94DC0E0C94DC
:100300000C3B0C946D0E0C949B6A0C94896A0C94B3
:10031000AF4D0C94E60E0C94CC460C94DE500C942D
:1003200034160C94F9450C942A3C0C94973C0C948C
:10033000672C0C94083C0C94885D0C94563C0C94EF
:100340001C110C94580B0C94FA0E0C9404420C944F
:100350000E3B0C94EC410C94770E0C9411650C94AC
:100360008B0E0C94ED2B0C94BC6A0C94AD2D0C945C
:10037000524C0C94E24C0C94512D0C94520B0C9456
:10038000B9090C94F4150C94073B0C949D0E0C9435
:10039000AF6A0C940B450C9413470C94040F0C9407
:1003A000F4410C9420420C941B470C9467420C942B
:1003B00053450C9406650C945E2B0C94475C0C948E
:1003C000F71B0C94844C0C94CD2D0C942A450C9462
:1003D000F3640C94DC420C94E7230C94A50E0C946B
:1003E00016240C94B90E0C94D20E0C949A2D0C94E5
:1003F00018240C94041C0C94F22A0C94101C0C94D9
:100400000A110C943A2D0C94856A0C9479680C941A
:10041000443D0C94950E0C946F4C0C94A96A0C946A
:10042000976A0C94A4650C945F680C94D5410C9465
:1004300023200C9456680C9418420C94936A0C94E4
:100440005D150C941E3C0C94A25C0C942F2B0C9408
:10045000B93C0C94E45C0C9408160C942F470C9453
:1004600073440C9483120C94A56A0C9452680C94F7
:100470001B0B0C94CA1C0C94F0410C94746A0C94E1
:10048000B36A0C94B76A0C94FC100C940D420C9453
:100490000D0B0C948F230C940A3B0C94252F0C9479
:1004A000C0430C94962A0C94A16A0C941C1C0C94C6
:1004B000945C0C9415470C94DC2B0C94714D0C94AB
:1004C000A52A0C94CC450C94660B0C946C150C94DA
:1004D000740B0C948D6A0C94715C0C9421420C94F6
:1004E00020680C94A0650C947D3C0C941C240C9406
:1004F000315D0C941D2B0C940E110C948A5D0C94A0
:100500005D460C949E230C94720E0C9419160C9458
:10051000AD5D6364696E6F70737578585B003E3EC5
:100520003E004E6F204D414320636F6E66696775D4
:100530007265643A20736574206669726D776172C2
:10054000652773204D41430A00312D77697265207C
:10055000636F756E743A200020416464723A0064DF
:100560006576230020616C69766500204E6F6465B6
:100570003A00536561726368696E67004D6F64622B
:10058000757320706F6C6C696E67206572726F7224
:100590003D002D002050492056616C203A004D6FDF
:1005A0006462757320706F6C6C696E67206572721F
:1005B0006F723D002D0020464D2056616C203A00A0
:1005C0004D6F6462757320706F6C6C696E67206527
:1005D00072726F723D002056616C3A20004D423AB3
:1005E00020004E6F7420737570706F727465642094
:1005F00072656720747970650A00496C6C65676183
:100600006C20617267756D656E74730A0075707425
:10061000696D650066726565686561700024737454
:1006200061747300200020000A667265653A00203C
:100630002D746172676574207A6F6E652D00204F8E
:10064000464600204F4E00204F46460020636D6412
:100650003A00204375723A00205365743A002045F1
:100660007870697265640A003D0056432300206378
:100670006D643D003D0056435F6865617423003D35
:100680000050696E3A003D0050696E3A00204861A2
:100690006C7465640A003D00526573746F72656422
:1006A0003A20003A204E6F2073746F726564207692
:1006B000616C756573202D2064656661756C740AC4
:1006C00000466F7263652057686974650A00416C63
:1006D0007265616479204163746976650A005475B6
:1006E000726E696E6720584F4E0A00584F4646207A
:1006F000736B69707065642E205072657620636D2F
:10070000643A005475726E6564206F666620667286
:100710006F6D3A00526573746F7265642066726F14
:100720006D3A003E20003C00205061723D200020C8
:10073000436D643D00205375623D00204974656D32
:100740003D00204D454D3D00476F742049502061CC
:100750006464726573733A00276970205B69705B2B
:100760002C646E735B2C67775B2C7375626E65749B
:100770005D5D5D5D27202D20736574207374617449
:1007800069632049500A004661696C656420746F92
:1007900020636F6E6669677572652045746865725F
:1007A0006E6574207573696E6720444843502E202F
:1007B000596F752063616E20736574206970206DB8
:1007C000616E75616C6C7921005374617274696E2D
:1007D00067206C616E00246E6F6465730024666F21
:1007E000726D6174002464617461747970650030A5
:1007F0002D31303000696E746567657200687376FC
:1008000000636F6C6F72004F4E2C4F46462C484170
:100810004C542C524553542C584F4E2C584F46464E
:100820002C544F47474C4500656E756D00666C6FE4
:10083000617400322E312E300024686F6D696500BE
:10084000757074696D652C667265656865617000A8
:10085000366661363631365F323031392D30332DE0
:100860003233004C696768744875622000246E61F9
:100870006D6500726561647900207472792061672A
:1008800061696E20696E2035207365636F6E6473D5
:10089000006661696C65642C2072633D004177617C
:1008A0006974696E6720666F722072657461696E23
:1008B000656420746F7069637300636F6E6E656347
:1008C0007465642061732000202E2E2E0020757325
:1008D00065723A003A000A417474656D7074696E0D
:1008E00067204D51545420636F6E6E656374696F59
:1008F0006E20746F200024737461746500646973E2
:10090000636F6E6E6563746564005573696E67200E
:100910004D5154542070617373776F726420667206
:100920006F6D20636F6E6669670044657669636505
:10093000204E616D653A00526562696E6420737580
:1009400063636573732E204950206164647265731C
:10095000733A004572726F723A20726562696E6412
:10096000206661696C0052656E65776564207375F9
:1009700063636573732E20495020616464726573EC
:10098000733A004572726F723A2072656E657765D0
:1009900064206661696C004E6F206C696E6B00416B
:1009A0006363657074696E6720636F6D6D616E64FB
:1009B000732E2E2E0A003D00494E3A0072676200E7
:1009C000637376006865617400766F6C00706F7792
:1009D000657200736574706F696E74006D6F646525
:1009E0000074656D700073657400536574436D64C5
:1009F0003A002056616C3D002053746F72652000F0
:100A0000444543524541534500494E4352454153A5
:100A1000450066616C7365007472756500584F46D9
:100A20004600584F4E0048414C5400544F47474CE5
:100A3000450052455354004F4646004F4E000A2889
:100A40002D29524553544152545F4C414E5F4F4EF5
:100A50005F4D5154545F4552524F5253000A282D56
:100A6000294841524452455345542C207573696EB0
:100A70006720736F6674000A282D29434F554E5422
:100A80004552000A282D29444854000A282B294F92
:100A900057495245000A282B294D4F4442555300CF
:100AA0000A282B29444D58000A282B294453323454
:100AB00038322D313030000A282B294672656552B4
:100AC000616D207072696E74696E670064653A6169
:100AD000643A62653A65663A66653A6665000A4652
:100AE00069726D77617265204D4143204164647283
:100AF00065737320006C617A79686F6D652E72750D
:100B0000000A436F6E666967207365727665723A94
:100B1000000A282B295741544348444F470032309C
:100B2000313130334C0020432B2B207665727369B2
:100B30006F6E3A00366661363631365F32303139A3
:100B40002D30332D3233000A4C617A79686F6D6530
:100B50002E7275204C6967687448756220636F6EE9
:100B600074726F6C6C6572200000002000230026F8
:100B70000029002C002F00320000010000030106B4
:100B80000109013D00494E3A002F00496E3A20000C
:100B9000696E00735F6F7574006D79686F6D6500C5
:100BA00000002200250028002B002E003100340018
:100BB00002010000050108010B0100000A0B0209F7
:100BC0000C0D0E08070304010000000000000000E7
:100BD0000000000000000000000000000000000015
:100BE00000000000000012111000000000000000D2
:100BF00000000000000000000000000000000000F5
:100C000000002100240027002A002D0030003300BE
:100C100001010000040107010A010102102020085F
:100C20000810204010204080020102010804020147
:100C300001020408102040808040201008040201B6
:100C4000800402018040201008040201080402010F
:100C50000102040810204080010204081020408096
:100C600005050505070508080808020202020A0A28
:100C70000808040404040101010101010101030346
:100C8000030303030303040707070C0C0C0C0C0CF1
:100C90000C0C0202020206060606060606060B0BEE
:100CA0000B0B0B0B0B0B005EBCE2613FDD83C29CA8
:100CB0007E20A3FD1F419DC3217FFCA2401E5F013A
:100CC000E3BD3E6082DC237D9FC1421CFEA0E1BFEC
:100CD0005D0380DE3C62BEE0025CDF81633D7C221E
:100CE000C09E1D43A1FF4618FAA427799BC584DA4C
:100CF0003866E5BB5907DB856739BAE406581947FA
:100D0000A5FB7826C49A653BD987045AB8E6A7F9AB
:100D10001B45C6987A24F8A6441A99C7257B3A64DD
:100D200086D85B05E7B98CD2306EEDB3510F4E100B
:100D3000F2AC2F7193CD114FADF3702ECC92D38DB9
:100D40006F31B2EC0E50AFF1134DCE90722C6D336B
:100D5000D18F0C52B0EE326C8ED0530DEFB1F0AE9D
:100D60004C1291CF2D73CA947628ABF517490856CB
:100D7000B4EA6937D58B5709EBB536688AD495CB79
:100D80002977F4AA4816E9B7550B88D6346A2B752B
:100D900097C94A14F6A8742AC896154BA9F7B6E85D
:100DA0000A54D7896B35436F6E6E65637465642E24
:100DB00000436F6E6E2E2061626F72746564004333
:100DC000757272656E74204C414E20636F6E666959
:100DD000672869702C646E732C67772C7375626E4C
:100DE0006574293A000A5573652074686573652037
:100DF000636F6D6D616E64733A202768656C702750
:100E0000202D207468697320746578740A276D61D9
:100E1000632064653A61643A62653A65663A66657C
:100E20003A3030272073657420616E642073746FCC
:100E30007265204D41432D6164647265737320694E
:100E40006E20454550524F4D0A276970205B6970EE
:100E50005B2C646E735B2C67775B2C7375626E65BD
:100E6000745D5D5D5D27202D207365742073746152
:100E70007469632049500A277361766527202D2005
:100E80007361766520636F6E66696720696E204EB8
:100E90005652414D0A2767657427205B636F6E6663
:100EA000696720616464725D27202D206765742066
:100EB000636F6E6669672066726F6D207072652D54
:100EC000636F6E666967757265642055524C206168
:100ED0006E642073746F726520616464720A276C9B
:100EE0006F616427202D206C6F616420636F6E66D4
:100EF00069672066726F6D204E5652414D0A277009
:100F0000776427202D20646566696E65204D5154F5
:100F1000542070617373776F72640A276B696C6C0D
:100F200027202D2074657374207761746368646F63
:100F3000670A27636C65617227202D20636C6561E9
:100F40007220454550524F4D0A277265626F6F748B
:100F500027202D207265626F6F7420636F6E74722C
:100F60006F6C6C657200536F6674207265626F6F90
:100F700074696E672E2E2E00444D58696E2042759E
:100F80006666657220616C6C6F63206572720049E1
:100F90006E697420696E2063683A000944533234E4
:100FA0003832206572726F72000952657365742061
:100FB000646F6E650009436865636B696E672066E0
:100FC0006F7220312D57697265206465766963659B
:100FD000732E2E2E004453323438322D31303020CF
:100FE00070726573656E74004453323438325F3109
:100FF00030305F4932435F544F5F31575F4252494F
:1010000044474520696E69740020416464723A0067
:1010100064657623000A312D7769726520000A6DB8
:1010200071747420000A6D6F6462757320000A6920
:101030006E7075747320000A6974656D7320000A00
:10104000436F6E666967757265643A002C003D00F7
:1010500050696E3A004F6E6520776972652052655F
:101060006164790A00444D58206F7574207374616F
:10107000727465642E204368616E6E656C733A20ED
:1010800000444D5820696E20737461727465642E3B
:10109000204368616E6E656C733A000A4C6F616440
:1010A00065640A000A6C6F6164206661696C65643E
:1010B0000A000A4E6F2073746F72656420636F6E4E
:1010C0006669670A006C6F6164696E6720436F6EC2
:1010D000666967000A72657175657374204D5154B5
:1010E0005420436F6E6669670053617665642074AF
:1010F0006F20454550524F4D00536176696E672011
:10110000636F6E66696720746F20454550524F4D7E
:101110002E2E0053617665640A00454550524F4DAE
:1011200020636C65617265640A0050617373776F48
:10113000726420757064617465640A00636F756C15
:1011400064206E6F742070617273653A2000557070
:1011500064617465640A002B002D00485454502FBC
:10116000312E312025690020485454502F312E3122
:101170000D0A486F73743A2025730D0A4163636545
:1011800070743A202A2F2A0D0A436F6E6E656374BD
:10119000696F6E3A20636C6F73650D0A00257300EA
:1011A00020000D0A004745540020747279206167C1
:1011B00061696E20696E2035207365636F6E64739C
:1011C0000A006661696C656420746F20636F6E6EDF
:1011D000656374004552524F523A205365727665EA
:1011E000722072657475726E65642000446F6E655E
:1011F0002E0A004170706C79696E672E0A00436F89
:101200006E6669672070617273696E6720666169D6
:101210006C65640A00676F7420436F6E6669670AC5
:1012200000436F6E666967205552493A20687474AE
:10123000703A2F2F006C617A79686F6D652E727528
:10124000002C20002E003E3E2000496E76616C6925
:101250006420636F6D6D616E6400526574727969AC
:101260006E6720434D440A004E6F74207375707092
:101270006F727465642072656720747970650A0006
:10128000293A0028543A003D3E004D6F6462757360
:10129000206F70206661696C65640A00416374693F
:1012A00076650A0047727020636865636B3A0A00CE
:1012B0002D3E005075623A2000556E6B6E6F776E52
:1012C00020636D64200A0053746174757320646533
:1012D0006666657265640A00536B697070696E6753
:1012E0002E2E004F4F4D21005D20000A5B003A007A
:1012F000436F6E66696775726564204D41433A00BD
:101300003E003E003C00543A0000787611241FBE97
:10131000CFEFD1E2DEBFCDBF00E00CBF15E0A0E013
:10132000B2E0E8E8FFE001E00BBF02C007900D92D9
:10133000AC38B107D9F72CE0ACE8B5E001C01D929C
:10134000A230B207E1F719E0C6E8D9E000E006C034
:1013500021970109802FFE010E948D82C538D10797
:1013600080E00807A9F70E94896B0C94C2870C944F
:1013700000002F923F924F925F926F927F928F92D6
:101380009F92AF92BF92CF92DF92EF92FF920F9314
:101390001F93CF93DF93CDB7DEB76B970FB6F8945B
:1013A000DEBF0FBECDBF6C013B015B8B4A8B590189
:1013B000088BFF8AEE8ADC011296ED91FC9113975F
:1013C000E080F180FE0131961F010091F60B109133
:1013D000F70B0115110511F402E01CE062E477E05F
:1013E0008FE698E00E94CF5DA101401B510B052EB6
:1013F000000C660B770B2AE08FE698E00E94085EEF
:101400006BE377E08FE698E00E94CF5DB7018FE64F
:1014100098E00E94F65E65E377E08FE698E00E9430
:10142000CF5D4AE050E06E897F898FE698E00E94A8
:10143000995E6FE277E08FE698E00E94CF5D4AE028
:1014400050E0B3018FE698E00E94995E68E277E091
:101450008FE698E00E94CF5DD60112968D919C9107
:101460001397892B09F455C61B861A861D861C8680
:101470001F861E86A114B10479F185014E01BAE0E0
:101480008B0E911CE12CF12CEA89FB89EE16FF06EC
:101490001CF5F3E0EF16F104F9F0D801AD90BD9022
:1014A0008D01F401A192B1924F0166E277E08FE6DF
:1014B00098E00E94CF5D4AE050E0B5018FE698E0E9
:1014C0000E94995E63E277E08FE698E00E94CF5D2C
:1014D000FFEFEF1AFF0AD8CF8FE698E00E94F25E86
:1014E00060E070E0C6010E941A212C0124E062161F
:1014F000710451F037E06316710469F183E06816F6
:10150000710409F059C007C0C6010E94E367892B26
:1015100009F030C103C6D60118968C91873009F4C2
:1015200025C360E0C6010E946F21853009F0F3C534
:1015300064E177E08FE698E00E94CF5D4AE050E0FA
:1015400065E070E08FE698E00E94995E8FE698E093
:101550000E94F25EE3C5F6018085873009F406C378
:1015600060E0C6010E946F21082F10E0863091F4E0
:1015700063E077E08FE698E00E94CF5D4AE050E0BC
:10158000B8018FE698E00E94995E8FE698E00E948D
:10159000F25EF0C06BEE76E08FE698E00E94CF5DE1
:1015A0004AE050E0B8018FE698E00E94995E8FE62D
:1015B00098E00E94F25EAFC5F2E06F16710409F484
:1015C000D9C04CF46114710489F031E063167104E0
:1015D00009F019C1ACC085E06816710409F4EBC0CC
:1015E00096E06916710409F48AC00DC1D6011896F7
:1015F0008C91853021F06EE0C6010E944821F601F1
:10160000808590E08A30910508F06EC0FC01882743
:10161000EE58FF4F8F4F0C948D828C859D85892BC2
:1016200051F42A893B892330310591F48FE7D601A3
:1016300018968C9304C0EA89FB89339749F44A854C
:101640005B850C851E85B801C6010E94BE2017C0AF
:10165000C6010E94F6207B01082F1A85AB01B80154
:10166000C6010E94BE20EA86FB86802F000F990BE0
:101670009D878C87812F110F990B9F878E87F88903
:10168000FF2371F101E09E01265F3F4F43E050E0F0
:1016900060E070E0C6010E94E76623E030E03B8B2B
:1016A0002A8B22C04A855B850C851E85B80114C033
:1016B0003889332359F001E09E01265F3F4F41E016
:1016C00050E060E070E0C6010E94E7664A855B85F5
:1016D000052E000C660B770BC6010E94BE2004C0CD
:1016E00083E090E09B8B8A8B0E94336B6093EC05C8
:1016F0007093ED058093EE059093EF0584C0C601CD
:101700000E94E367892B39F46EED76E08FE698E06E
:101710000E94CF5D0CC06EEC76E08FE698E00E94F0
:10172000CF5DD60118968C91873009F0F4C4F6018C
:101730008085813009F01CC560E0C6010E946F21E0
:10174000813009F015C50E94336B0091EC051091B2
:10175000ED052091EE053091EF05DC01CB01801BFA
:10176000910BA20BB30B853F9140A105B10508F089
:10177000D9C4FEC460E0C6010E946F218530B9F073
:101780001B861A861D861C861F861E8662E0C60181
:101790000E944821F889FF2351F000E020E030E06A
:1017A00040E050E062E070E0C6010E94E766A2E01F
:1017B0006A2E712C28C0C6010E94E367181619060C
:1017C00014F51B861A861D861C861F861E8660E001
:1017D000C6010E946F21863011F462E001C065E00D
:1017E000C6010E94482100E020E030E040E050E0E7
:1017F00062E070E0C6010E94E7666DE876E08FE681
:1018000098E00E94CF5DEC84FD84C7010F2C000C92
:10181000AA0BBB0B888F998FAA8FBB8FAE85BF8514
:10182000BD8BAC8B2FEF30E00E94A482F4E68F2EAC
:10183000912CA12CB12CA50194010E943882890120
:10184000F6018085843009F47FC150F4813009F4B9
:101850004CC0F0F1823089F1833009F4DAC158C408
:10186000883009F48AC338F4863009F4A6C1873079
:1018700009F04EC47BC1893009F4EEC28F3709F0FC
:1018800047C460E0C2010E94F53E60E0C2010196DB
:101890000E94F53E60E0C20102960E94F53EAE85D0
:1018A000BF852FEF30E00E94A482A50194010E9421
:1018B0003882622FC201039644C12FEF30E0D70176
:1018C0000E94A482A50194010E943882D22E78C081
:1018D000AA85BB852FEF30E00E94A482A501940168
:1018E0000E943882622FC2012CC192012D5F3F4FAE
:1018F000390132E3E316F1040CF049C082E390E0D1
:101900008E199F09EC89FD898E9FD0018F9FB00DA4
:101910009E9FB00D11242FEF30E00E94A48228E892
:1019200033E140E050E00E943882622FC3010E9400
:10193000F53E0C851D852EEF31E0D8010E94A48272
:10194000E2E3CE2ED12CE12CF12CA70196010E94CE
:101950003882AE85BF850E949C82A50194010E94B9
:10196000388249015A019801A5E6BFEF0E949C8286
:10197000A70196010E943882DD24DA94D20E8401F8
:101980000F3F1105E9F0E4F00FEF10E019C0288DCA
:10199000398D4A8D5B8D2253310941095109ABE9DB
:1019A000B0E00E94578222E330E040E050E00E9425
:1019B000388264E6D62ED20E60E0C3010E94F53E66
:1019C000AA85BB852FEF30E00E94A4822DE631E08E
:1019D00040E050E00E943882322F122F1F71110F09
:1019E000110F812F880F15E5682F619F060E60E0AB
:1019F000611D1124922F9074207237FD24C0911123
:101A00000CC0211104C0862F8095F62E14C055E518
:101A1000F52EF60E10E06BEA36C021110FC0182F1C
:101A20003AEA139F010E10E0111D11248BEA811B6D
:101A30004AEAF42EF60E682F10E025C080E0F62E5C
:101A4000F094162F0FC0911112C021110DC0182F44
:101A50002AEA129F010E10E0111D11243BEAF32E19
:101A6000F11A1B5A60E00FC0162F10950BC0211100
:101A700004C085E5860F1BEA03C08AEA860F90E062
:101A8000161B682FF12CFFEFDF1609F42AC0DD20AA
:101A900009F423C0662329F02D2D629F060E60E015
:101AA000611DFF2039F03F2D2D2D329F030E30E0B8
:101AB000311DF32E112329F03D2D139F010E10E04F
:101AC000111D11242D2D2095229F020E20E0211D95
:101AD0001124620FF20E120F04C01FEFFF24FA94BC
:101AE0006FEF0F3F09F422C020E0002321F0009F98
:101AF000212D09F02F5F2223B1F0662321F0629F90
:101B0000060E60E0611DFF2031F03F2D329F030E75
:101B100030E0311DF32E112321F0129F010E10E051
:101B2000111D112403C010E0F12C60E0C2010E94DD
:101B3000F53E6F2DC20101960E94F53E612FC20154
:101B400002960E94F53EE4C2E480F580F7018085AC
:101B5000853009F0DDC2C7010E94FA3BA82EB12CE6
:101B6000F2E0AF16B1040CF025C4D2C2D60114962F
:101B7000ED91FC9115978085853009F0C9C2C6802A
:101B8000D780C114D10409F4C3C2F60161857285FE
:101B9000C1010E94AE61EE88FF8808899E01265F20
:101BA0003F4F4A895B89B301C1010E94B909D6013F
:101BB0001296CD90DC901397E4CFF42C61E0842D45
:101BC0000E94BD6A11E000E0B1E06B16710429F0DB
:101BD000E6E06E16710409F010E0612F8F2D0E946F
:101BE0006E3668E876E08FE698E00E94CF5D4AE0C6
:101BF00050E0B2018FE698E00E94995E66E876E0D8
:101C00008FE698E00E94CF5D4AE050E0612F702F90
:101C10001AC157FE06C051944194510801E010E0EA
:101C200002C000E010E0F42C61E0842D0E94BD6A47
:101C30008091A100887F8093A10080919100887F8E
:101C4000809391008091A10082608093A100809197
:101C50009100826080939100AA85BB85012B99F049
:101C6000CD01BB0FAA0BBB0B9C01AD012456310962
:101C700041095109AFEFB0E00E9457822CE93FEFD4
:101C80004FEF5FEF08C02FEF30E00E94A48224E600
:101C900030E040E050E00E943882890161E08F2D01
:101CA0000E94BD6A0115110509F4B1C00F3F11056D
:101CB00009F4AFC0F201FF27E654F44FE4918E2FF0
:101CC00090E0FC013197E231F10508F09DC08827D2
:101CD000E458FF4F8F4F0C948D8284B5806884BD8B
:101CE00007BD9BC084B5806284BD08BD96C080914D
:101CF00080008068809380001093890000938800A2
:101D00008CC08091800080628093800010938B0053
:101D100000938A0082C08091800088608093800058
:101D200010938D0000938C0078C08091B000806883
:101D30008093B0000093B30070C08091B0008062C7
:101D40008093B0000093B40068C0809190008068D8
:101D50008093900010939900009398005EC080914A
:101D6000900080628093900010939B0000939A00F3
:101D700054C08091900088608093900010939D00E3
:101D800000939C004AC08091A00080688093A000CE
:101D90008091A0008F7B8093A0001093A9000093F6
:101DA000A8003BC08091A00080628093A0001093A7
:101DB000AB000093AA0031C08091A000886080939E
:101DC000A0001093AD000093AC0027C080912001CB
:101DD00080688093200110932901009328011DC081
:101DE0008091200180628093200110932B01009349
:101DF0002A0113C0809120018860809320011093F4
:101E00002D0100932C0109C00038110514F460E085
:101E100001C061E08F2D0E946E3661E876E08FE6AA
:101E200098E00E94CF5D4AE050E0B2018FE698E072
:101E30000E94995E6FE776E08FE698E00E94CF5DA2
:101E40004AE050E0B8018FE698E00E94995E8FE684
:101E500098E00E94F25E5CC11A8560E070E0C60105
:101E60000E941A21082FF92E6AE676E08FE698E0A4
:101E70000E94CF5D4AE050E0602F7F2D8FE698E012
:101E80000E94995E68E676E08FE698E00E94CF5D5A
:101E9000612F012E000C770B4AE050E08FE698E0AE
:101EA0000E94995E8FE698E00E94F25E8091E70BB7
:101EB0009091E80B892B89F06AE872E18FE698E04F
:101EC0000E94CF5D662D6064C6010E944821412FAB
:101ED000110F550B660B770BB3C081E090E0909328
:101EE000E80B8093E70B26E040E855E260E070E005
:101EF00082ED97E00E94DE380093C90982ED97E0F9
:101F00009093C8098093C7091092D40A1092D60AF8
:101F10001092D50A80ED97E090934F0A80934E0A75
:101F20001092510A1092500A112339F085E090E086
:101F30009093530A8093520A04C01092530A10924D
:101F4000520A86E00E94433962E370E080E090E04C
:101F50000E94F96A82ED97E090934F0A80934E0AAF
:101F60001092510A1092500AF4E61F02A0011124A7
:101F70005093530A4093520AC4C00480F581E02D67
:101F800061857285C1010E94AE61C1010E94B120CC
:101F9000882309F4BDC08985893009F0B9C0162DA0
:101FA000EA8460E070E0C1010E941A21082FF92E36
:101FB00066E776E08FE698E00E94CF5D4AE050E069
:101FC000602F7F2D8FE698E00E94995E64E776E0AF
:101FD0008FE698E00E94CF5D6E2D0E2C000C770BE3
:101FE0004AE050E08FE698E00E94995E6EE676E067
:101FF0008FE698E00E94CF5D4AE050E0662D062C07
:10200000000C770B8FE698E00E94995E8FE698E0CF
:102010000E94F25E8091E70B9091E80B892BA1F072
:102020006AE872E18FE698E00E94CF5D662D6064F9
:10203000C6010E9448214E2DEE0C550B660B770B06
:10204000C6010E94BE2064C081E090E09093E80B3E
:102050008093E70B26E040E855E260E070E082ED17
:1020600097E00E94DE380093C90982ED97E09093D3
:10207000C8098093C7091092D40A1092D60A109208
:10208000D50A123009F4FBC1153009F4F8C16E2DE0
:10209000EE0C770B880B990B0E94DB8322E538EB63
:1020A00042E152E40E94C08220E030E040E251E48C
:1020B0000E9490842DEE3EE94CE35EE30E94318362
:1020C0006B017C0120E030E0A9010E948B8420E0BC
:1020D00030E040E05FE387FDCDC1C701B6010E945B
:1020E000C0820E94A38383ED97E090934F0A809370
:1020F0004E0A1092510A1092500A7093530A60933C
:10210000520A86E00E9443391092E80B1092E70BC6
:10211000B9C18FEF01C08DEF9FEFB4C16624639406
:10212000712C05CB61EC76E08FE698E00E94CF5DE4
:102130008FE7F60180871D861C8684E690E09F87E6
:102140008E874A855B8560E074E6C6010E94BE20EA
:10215000F889FF2309F457CB00E09E01265F3F4F2B
:1021600043E050E060E070E0C6010E94E7664BCBC0
:10217000662DC6010E944821C6010E94F620F62E57
:10218000E72E8C01D60118962C91233008F000C15F
:10219000213070F46A307105810591052CF4B2E3A9
:1021A000FB2EE12C00E010E04F2D5E2D602F0AC0C9
:1021B000611571058105910519F01A300CF412E3CF
:1021C000AB01682F712FC6010E94BE204F2D5E2DDE
:1021D000B8011416150616061706E4F5D60118966A
:1021E0008C9190E08A30910538F5FC018827E25700
:1021F000FF4F8F4F0C948D82C7019A878B87802F5A
:10220000000F990B9D878C87812F110F990B9F874A
:102210008E8753C05B874A8701E07FC05B874A8710
:10222000B889BB2309F4EFCA00E020E030E040E0C9
:1022300050E061E070E00AC0E889EE2309F4ACC028
:1022400000E020E030E040E050E0B301C6010E9431
:10225000E766A2C02AE030E08FE698E00E94515E77
:1022600063EA76E08FE698E00E94CF5DD60118968B
:102270008C918530C9F0A0F48150823008F041C0C3
:1022800084E690E09B878A871D861C869F878E87C1
:1022900044E650E060E074E6C6010E94BE200DC036
:1022A0008630C9F0883069F584E190E09B878A87A1
:1022B00044E150E060E070E02CC001E09E01265F48
:1022C0003F4F43E050E060E070E0C6010E94E766E7
:1022D00003E010E02EC084E690E09B878A8744E606
:1022E00050E060E070E0C6010E94BE20B889BB23C8
:1022F000F1F000E020E030E040E050E061E070E02C
:1023000013C084E690E09B878A8744E650E060E053
:1023100070E0C6010E94BE2000E09E01265F3F4F94
:1023200041E050E060E070E0C6010E94E76601E035
:1023300010E05E01EAE0AE0EB11CE12CF12CD501FB
:102340008D909D905D0168E976E08FE698E00E94AF
:10235000CF5D4AE050E0B7018FE698E00E94995EB9
:1023600066E976E08FE698E00E94CF5D4AE050E0B3
:10237000B4018FE698E00E94995E8FE698E00E9493
:10238000F25EBFEFEB1AFB0A0E151F05C1F604C083
:10239000243009F4FFCE1ACFF6018085813009F090
:1023A00032CA8C859D85892B09F02DCA8FE7F601ED
:1023B000808729CA60E0C7010E945F38DC01199656
:1023C0008D919C911A97998B888B61E0C7010E942F
:1023D0005F38FC0141845284638474842A843B8482
:1023E000F2E0AF16B104E9F162E0C7010E945F3884
:1023F000DC0119960D911C911A97B3E0AB16B1044C
:1024000091F163E0C7010E945F38FC0181849284EE
:10241000F4E0AF16B10451F064E0C7010E945F38E8
:10242000DC011996AD90BC901A9703C032E0A32E40
:10243000B12C8114910461F09401D1010E949C821D
:1024400024E630E040E050E00E943882790101C08B
:1024500071019501A20168897989C6010E94CA614A
:1024600057CE0FEF1FEF8FE3882E912C92E0A92E0D
:10247000B12CE2CFC701B6010E94BF8232CE60E02C
:1024800070E031CE6B960FB6F894DEBF0FBECDBFB5
:10249000DF91CF911F910F91FF90EF90DF90CF9040
:1024A000BF90AF909F908F907F906F905F904F9074
:1024B0003F902F9008954F925F926F927F928F92EC
:1024C0009F92AF92BF92CF92DF92EF92FF920F93C3
:1024D0001F93CF93DF93CDB7DEB7C15AD1400FB66C
:1024E000F894DEBF0FBECDBFE0919C05F0919D0535
:1024F0003B96E831F10508F0B7C38827E856FF4F4F
:102500008F4F0C948D820E94336B00916D0B109154
:102510006E0B20916F0B3091700B06171707280771
:10252000390708F0A1C30AE113E0CF56DE4F198343
:102530000883C159D140CD56DE4F188219821A82C4
:102540001B82C359D140CF57DE4F19830883C1582E
:10255000D140CD57DE4F188219821A821B82C35890
:10256000D140CF59DE4F19830883C156D140CD5990
:10257000DE4F188219821A821B82C356D140CF5B6C
:10258000DE4F19830883C154D140CD5BDE4F1882E2
:1025900019821A821B82C354D14069EC77E08FE61E
:1025A00098E00E94CF5DBE016F567E4F86E090E0BE
:1025B0000E946133892B09F467C167E274E08FE6FA
:1025C00098E00E94F65E1A830983CD56DE4F88811B
:1025D0009981AA81BB81C359D1408B839C83AD83F0
:1025E000BE83CE0101960E94E058BE016F577E4F18
:1025F0008AE090E00E946133892B09F42EC16DE3DB
:1026000074E08FE698E00E94F65E1A830983CD5746
:10261000DE4F88819981AA81BB81C358D1408B83C9
:102620009C83AD83BE83CE0101960E94E058BE011B
:102630006F597E4F8EE090E00E946133892B09F440
:10264000DFC063E474E08FE698E00E94F65E1A83D0
:102650000983CD59DE4F88819981AA81BB81C356F8
:10266000D1408B839C83AD83BE83CE0101960E94B3
:10267000E058BE016F5B7E4F82E190E00E946133C3
:10268000892B09F477C068E474E08FE698E00E9433
:10269000F65E1A830983CD5BDE4F88819981AA811A
:1026A000BB81C354D1408B839C83AD83BE83CE0159
:1026B00001960E94E0581A830983CD5BDE4F888122
:1026C0009981AA81BB81C354D1408B839C83AD8304
:1026D000BE83CF57DF4F19830883C158D040CD59EF
:1026E000DE4F88819981AA81BB81C356D140CD57E5
:1026F000DF4F88839983AA83BB83C358D040CF53CD
:10270000DF4F19830883C15CD040CD57DE4F8881ED
:102710009981AA81BB81C358D140CD53DF4F8883B3
:102720009983AA83BB83C35CD040CF5FDE4F1983FC
:102730000883C150D140CD56DE4F88819981AA814E
:10274000BB81C359D140CD5FDE4F88839983AA8373
:10275000BB83C350D1409E012F5F3F4FAE014F5707
:102760005F4FBE016F537F4FCE018F5F9E4F0E9420
:102770002D3785C01A830983CD59DE4F8881998111
:10278000AA81BB81C356D1408B839C83AD83BE831A
:10279000CF57DF4F19830883C158D040CD57DE4F44
:1027A00088819981AA81BB81C358D140CD57DF4F21
:1027B00088839983AA83BB83C358D040CF53DF4F0C
:1027C00019830883C15CD040CD56DE4F8881998142
:1027D000AA81BB81C359D140CD53DF4F88839983F0
:1027E000AA83BB83C35CD040AE014F5F5F4FBE0185
:1027F0006F577F4FCE018F539F4F0E9479373FC055
:102800001A830983CD57DE4F88819981AA81BB81C4
:10281000C358D1408B839C83AD83BE83CF57DF4F9A
:1028200019830883C158D040CD56DE4F88819981E5
:10283000AA81BB81C359D140CD57DF4F888399838B
:10284000AA83BB83C358D040BE016F5F7F4FCE01C8
:102850008F579F4F0E94CB3712C01A830983CD56E2
:10286000DE4F88819981AA81BB81C359D1408B8376
:102870009C83AD83BE83CE0101960E9416388FE6FD
:1028800098E00E94F25E0BC16FE474E08FE698E07E
:102890000E94F65E0FB6F894A8958091600088615A
:1028A00080936000109260000FBE80914E068111EF
:1028B00007C083E396E00E94C24281E080934E0607
:1028C00080EF95E090931909809318090E949D3636
:1028D000CE0101960E94765589819A810E94B63C6C
:1028E00046E050E06AEC77E089E090E00E94123028
:1028F0008AE193E09A8389831B821C821D821E8257
:10290000CE0103960E94A03C0E94B53C809118091C
:1029100090911909DC0192961D921D921D921C92B4
:102920009597FC0116A217A210A611A69A961D92C1
:102930001D921D921C929D9740EE5EE260E070E059
:1029400046AB57AB60AF71AF40EA5FE060E070E06C
:10295000DA964D935D936D937C93DD973E9624E1DB
:10296000DF011D922A95E9F726E0EAECF7E0DC01A9
:10297000189601900D922A95E1F7FC01EE5BFF4F4E
:1029800010820E9494318C01019709F04AC0CE0157
:1029900001960E94765589819A810E94B63C609189
:1029A000180970911909625F7F4FCE0101960E944C
:1029B000F85ECE0103960E94A03C609118097091C8
:1029C00019096A5E7F4FCE0101960E94F85ECE0122
:1029D00003960E94AE3C60911809709119096E5ED1
:1029E0007F4FCE0101960E94F85ECE0103960E94B1
:1029F000A73C0E94B53C6091180970911909625E6C
:102A00007F4FCE0101960E94F85E8B819C81AD8143
:102A1000BE818093140990931509A0931609B09371
:102A2000170999E288E10FB6F894A89580936000A1
:102A30000FBE90936000A895012B19F567E877E029
:102A40008FE698E00E94CF5D68E577E08FE698E03A
:102A50000E94CF5D86EF9FEF90939D0580939C052C
:102A60000E94336BDC01CB01805A9541AF4FBF4FC1
:102A700080936D0B90936E0BA0936F0BB093700BC4
:102A8000F3C068E477E08FE698E00E94CF5DCE0166
:102A900001960E943659CE0101960E94E05881E0CD
:102AA00090E0DEC08091560681111AC060E070E0AF
:102AB00080E090E00E94A04ED3C00E94336B009152
:102AC0006D0B10916E0B20916F0B3091700B0617F0
:102AD000170728073907C8F10E943C638111C4C059
:102AE00082E090E0BDC0A895CF55DE4F1882C15A54
:102AF000D140FE01EF56FE4F119211928EE0DF01A0
:102B00001D928A95E9F70091650B1091660B0115EE
:102B1000110529F0C8010E94FA3B811137C20E94B9
:102B20003C638111A1C0E090650BF090660BE1144D
:102B3000F10409F499C0C7010E94FA3B082F10E084
:102B4000023011050CF03FC28FC020E030E043E0BE
:102B500050E060E48E010F5F1F4FC8010E943726CE
:102B60006AE275E0C8010E94D886F8010190002051
:102B7000E9F7CF01801B910B08968138910538F554
:102B80000E943C63882319F18091AC099091AD09B2
:102B9000019611F481E090E09093AD098093AC0927
:102BA0008091AC099091AD099093310980933209DD
:102BB00047E050E06CE279E0C8010E94B362AC01EA
:102BC000455051096CE279E082EA0E94D36283E0C9
:102BD00090E090939D0580939C056FE979E08FE6E6
:102BE00098E00E94CF5D40C00E94336B00916D0B56
:102BF00010916E0B20916F0B3091700B0617170719
:102C00002807390788F510929D0510929C052CC065
:102C10000E94336B00916D0B10916E0B20916F0B26
:102C20003091700B061717072807390708F458CF9B
:102C30001BC00E94454E892B09F052CF0E94336B76
:102C4000DC01CB0188579C4EAF4FBF4F80936D0B7B
:102C500090936E0BA0936F0BB093700B86EF9FEF6A
:102C600090939D0580939C050FB6F894A89580914C
:102C70006000886180936000109260000FBE8091B8
:102C80009C0590919D05181619060CF059C10091EC
:102C90001809109119090115110509F451C10E9473
:102CA000336B4B015C017801FEE3EF0EF11CF70181
:102CB00080819181A281B381A5019401281B390BE8
:102CC0004A0B5B0BCA01B901683E33E0730781050B
:102CD000910508F446C028EE33E040E050E00E9441
:102CE0001682861A970AA80AB90AD7018D929D9270
:102CF000AD92BC921397F80186A597A5A0A9B1A99A
:102D000069017A01CC0CDD1CEE1CFF1C8C159D05A5
:102D1000AE05BF0528F416A617A610AA11AA09C069
:102D2000821B930BA40BB50BF80186A797A7A0AB4A
:102D3000B1ABF80182A993A9A4A9B5A98C159D05E9
:102D4000AE05BF0528F412AA13AA14AA15AA09C031
:102D5000821B930BA40BB50BF80182AB93ABA4AB16
:102D6000B5ABF80186A597A5A0A9B1A9892B8A2B97
:102D70008B2B69F4EE5BFF4F8081833041F484E05C
:102D80008083C8010E94943101967C0102C0E12C2D
:102D9000F12CF80182A993A9A4A9B5A9892B8A2BA2
:102DA0008B2BA1F4EE5BFF4F8081833011F08111FA
:102DB0000DC01082F8013E9684E1DF011D928A95D4
:102DC000E9F7C8010E94943103967C01B2E0EB164A
:102DD000F10429F0E4E0EE16F10409F04AC0CE0156
:102DE00001960E94765589819A810E94B63C609135
:102DF000180970911909625F7F4FCE0101960E94F8
:102E0000F85ECE0103960E94A03C60911809709173
:102E100019096A5E7F4FCE0101960E94F85ECE01CD
:102E200003960E94AE3C60911809709119096E5E7C
:102E30007F4FCE0101960E94F85ECE0103960E945C
:102E4000A73C0E94B53C6091180970911909625E17
:102E50007F4FCE0101960E94F85E8B819C81AD81EF
:102E6000BE818093140990931509A0931609B0931D
:102E70001709F3E0EF16F10409F451C064F431E0EE
:102E8000E316F10451F142E0E416F10409F058C0F0
:102E900066E679E049C054E0E516F10409F442C061
:102EA00085E0E816F10409F04BC067E979E08FE6A8
:102EB00098E00E94CF5D8FE698E00E94F25E0E944B
:102EC0003C6381110E9463590E94336BDC01CB018A
:102ED000805D9A48AF4FBF4F13C063E879E08FE63B
:102EE00098E00E94CF5D0E943C6381110E9463596B
:102EF0000E94336BDC01CB0188519C4FAF4FBF4F19
:102F000080936D0B90936E0BA0936F0BB093700B2F
:102F100086EF9FEF90939D0580939C0511C063E51C
:102F200079E0DDCF67E379E08FE698E00E94CF5D3E
:102F3000CE0101960E943659CE0101960E94E058BA
:102F400099E288E10FB6F894A895809360000FBECF
:102F50009093600080919C0590919D05CF55DE4F28
:102F60000FB6F894DEBF0FBECDBFDF91CF911F919A
:102F70000F91FF90EF90DF90CF90BF90AF909F9018
:102F80008F907F906F905F904F90089560E0C801A0
:102F90000E945F38DC0119960D911C911A971093CD
:102FA000600600935F066AE279E08FE698E00E948F
:102FB000CF5DB8018FE698E00E94F65E8FE698E05C
:102FC0000E94F25EACCD61E0C7010E945F38FC0157
:102FD000618472840230110509F44AC362E0C701BA
:102FE0000E945F38FC01818492840330110551F006
:102FF00063E0C7010E945F38DC011996ED90FC90F8
:103000001A9704C0FE01EF55FE4F7F0140E150E0EA
:10301000BE016F567E4F86E390E00E94014E892BE1
:1030200021F4053011050CF02CC38E010F561E4FF4
:103030007092C0096092BF099092C2098092C10942
:1030400088EA95E69093B8098093B7095E01FFE797
:10305000AF1AFEEFBF0A40E150E06DEF78E0C50126
:103060000E94B77A6E012FE9C21A2EEFD20A20E031
:1030700030E041E050E060E2C6010E94372640E2C5
:1030800050E066EF78E0C6010E94A77A66ED78E02E
:103090008FE698E00E94CF5DB3018FE698E00E9432
:1030A000F65E64ED78E08FE698E00E94CF5D4AE03E
:1030B00050E0B4018FE698E00E94995E6DEC78E0F4
:1030C0008FE698E00E94CF5DB7018FE698E00E94FE
:1030D000F65E68EC78E08FE698E00E94CF5D0FB670
:1030E000F894A895809160008861809360001092A8
:1030F00060000FBE80905F06909060060E943C6367
:1031000081113BC16091BF097091C00980912A096A
:1031100090912B094091C1095091C209DC01ED91B8
:10312000FC916115710521F00088F189E02D16C030
:103130000684F785E02D2AE133E03A832983409025
:10314000BB095090BC096090BD097090BE094B82CC
:103150005C826D827E82BE016F5F7F4F19958130E8
:10316000910509F003C19093AD098093AC0987E004
:10317000E4E4F2E0DE01119601900D928A95E1F708
:10318000FE013196A1E3B9E0CE01089621912D937D
:10319000E817F907D9F7E114F10429F00115110531
:1031A00021F086EF03C086E301C086EB80933809E7
:1031B000109239098FE080933A09F40101900020C0
:1031C000E9F7CF018819990940968138910508F0EF
:1031D000C1C04FE050E06CE279E0C4010E94B362EC
:1031E000F60101900020E9F73197EC19FD09E80F8D
:1031F000F91F3296E138F10508F0ACC0AC016CE281
:1032000079E0C6010E94B362F50101900020E9F760
:103210003197EA19FB09E80FF91F3296E138F105F9
:1032200008F098C0AC016CE279E0C5010E94B3627D
:10323000E114F10479F1F70101900020E9F73197E9
:10324000EE19FF099C012E5F3F4FE20FF31FE1389B
:10325000F10508F07FC0AC016CE279E0C7010E9483
:10326000B36201151105B1F0F80101900020E9F7F2
:103270003197E01BF10B9C012E5F3F4FE20FF31FD4
:10328000E138F10508F066C0AC016CE279E0C801F4
:103290000E94B362AC01455051096CE279E080E1D3
:1032A0000E94D3620E94336B6093AE097093AF09A2
:1032B0008093B0099093B1096093B2097093B309F8
:1032C0008093B4099093B50980912A0990912B09B4
:1032D000DC01ED91FC910084F185E02D1995892B9D
:1032E000C1F40E94336B0091B2091091B30920918F
:1032F000B4093091B509DC01CB01801B910BA20B05
:10330000B30B88399A43A105B105F0F28CEF9FEF1A
:103310001DC0CE018F579F4F0E9498560497D1F43D
:1033200080912F09811111C00E94336B6093B20903
:103330007093B3098093B4099093B5091092B609BC
:103340001092C6091092C50918C090E09093C60962
:103350008093C50980912A0990912B09DC01ED9198
:10336000FC910488F589E02D19959EC18EEF9FEFA1
:103370009093C6098093C50997C100915F0610918B
:1033800060066AEB78E08FE698E00E94CF5DB801B6
:103390008FE698E00E94F65E8FE698E00E94F25E6B
:1033A00099E288E10FB6F894A895809360000FBE6B
:1033B0009093600081E08093560620E030E043E087
:1033C00050E060E4CE018F5F9E4F0E9437266AE294
:1033D00075E0CE018F5F9E4F0E94D886CE018F5F31
:1033E0009E4F0E94213320E030E042E050E060E454
:1033F000CE018F5F9E4F0E9437266AE275E0CE01B4
:103400008F5F9E4F0E94D886BE016F5F7E4F8FE612
:1034100098E00E947454CE018F5F9E4F0E9421332A
:1034200020E030E041E050E060E4CE018F5F9E4F4D
:103430000E9437266AE275E0CE018F5F9E4F0E94A0
:10344000D886BE016F5F7E4F8FE698E00E9474546D
:10345000CE018F5F9E4F0E942133FE01EF53FF4F3D
:10346000119211921EE3DF01212F1D922A95E9F797
:103470001A821982FE0133968EE7DF011D928A952A
:10348000E9F720E030E041E050E060E4CE018F5306
:103490009F4F0E94372640E450E066EF78E0CE016F
:1034A0008F539F4F0E94A77A40E850E063E778E08F
:1034B000CE0101960E94B77ABE016F5F7F4FCE01A9
:1034C0008F539F4F0E94C56320E030E041E050E001
:1034D00060E4CE018F539F4F0E94372640E450E0B6
:1034E0006DE678E0CE018F539F4F0E94A77A40E8A7
:1034F00050E063E678E0CE0101960E94B77A40E89A
:1035000050E060E578E0CE0101960E94A77ABE0106
:103510006F5F7F4FCE018F539F4F0E94C56320E0A6
:1035200030E041E050E060E4CE018F539F4F0E94B5
:10353000372640E450E06DE176E0CE018F539F4F97
:103540000E94A77A40E850E060E478E0CE0101965E
:103550000E94B77ABE016F5F7F4FCE018F539F4F9E
:103560000E94C56320E030E041E050E060E4CE011D
:103570008F539F4F0E94372640E450E069E378E084
:10358000CE018F539F4F0E94A77A40E850E063E33B
:1035900078E0CE0101960E94B77ABE016F5F7F4F3F
:1035A000CE018F539F4F0E94C563A091E90BB0914C
:1035B000EA0B109709F443C080914B0290914C02A2
:1035C000AE014F5B5E4FFA01819391932EE1119210
:1035D0002A95E9F79E012F573F4FF9018193919367
:1035E00011921A95E9F716960D911C911797E09094
:1035F000E90BF090EA0BE114F10471F001151105EB
:1036000059F0D80118968C918530A9F7C8010E940D
:10361000FA3B882381F372C020E030E041E050E0C3
:1036200060E4CE018F539F4F0E94372640E450E064
:1036300066ED77E0CE018F539F4F0E94A77A84E01A
:1036400090E090939D0580939C050E94336BDC0174
:10365000CB0188579C4EAF4FBF4F80936D0B90931B
:103660006E0BA0936F0BB093700B6DE978E0B7CA47
:103670008BE5882E87E0982E9E012F553E4F7901CD
:10368000C5CC64E08091650B9091660B0E945F3819
:10369000DC0119960D911C911A976AE079E08FE68A
:1036A00098E00E94CF5DC4CC0091C5091091C60975
:1036B00061E978E08FE698E00E94CF5D4AE050E053
:1036C000B8018FE698E00E94995E69E778E08FE69E
:1036D00098E00E94CF5D0E94336BDC01CB018857DC
:1036E0009C4EAF4FBF4F80936D0B90936E0BA0938A
:1036F0006F0BB093700B8CE090E0B2CA60E0C80131
:103700000E945F38FC0181859285A385B4858A304B
:10371000910508F463C020E030E041E050E060E44F
:10372000CE018F539F4F0E943726F801608171812F
:1037300040E450E0CE018F539F4F0E94FE8663E22B
:1037400074E0CE018F539F4F0E94D88640E450E032
:1037500065EE77E0CE018F539F4F0E94A77ABE019E
:103760006F5B7E4FCE018F539F4F0E94C563CF5733
:10377000DF4F8881C158D040882361F120E030E0DC
:1037800041E050E060E4CE018F539F4F0E94372606
:10379000D8016D917C9140E450E0CE018F539F4F52
:1037A0000E94FE8663E274E0CE018F539F4F0E9419
:1037B000D88640E450E06DED77E0CE018F539F4F07
:1037C0000E94A77ABE016F577F4FCE018F539F4F44
:1037D0000E94C563F8010281138109CFFC0140E218
:1037E00050E08827E055FF4F8F4F0C948D826DE29B
:1037F00078E0CE018F5B9E4F0E94B77ACF57DF4FA4
:103800001882C158D04087CF68E278E0CE018F5B44
:103810009E4F0E94B77A40E450E067E078E017C01E
:1038200061E078E0CE018F5B9E4F0E94B77A40E462
:1038300050E06DEF77E00BC065EF77E0CE018F5B76
:103840009E4F0E94B77A40E450E06FEE77E0CE01E1
:103850008F579F4F0E94B77A5ECFBC01823091058F
:1038600008F40895613E8EE1780748F49B0195E0E5
:10387000369527959A95E1F748E0420F01C04FEF42
:1038800091E0242F30E0290F311D35952795229F97
:10389000F001239FF00DF00D11246E177F0718F42F
:1038A0004FEF420F04C02F3F39F091E0920F4917BC
:1038B00040F78FEF890F08958FEF0895CF93DF932F
:1038C000009709F447C0FC012081222309F442C07B
:1038D000EC0166EE79E00E949E7A892BF1F161EEAF
:1038E00079E0CE010E949E7A892BD1F16CED79E0CE
:1038F000CE010E949E7A892BB1F163ED79E0CE0171
:103900000E949E7A892B91F16DEC79E0CE010E94A4
:103910009E7A892B71F169EC79E0CE010E949E7A42
:10392000892B51F164EC79E0CE010E949E7A892BBB
:1039300031F160EC79E0CE010E949E7A892B11F181
:103940006CEB79E0CE010E949E7A892BF1F489E03C
:1039500090E01DC080E090E01AC081E090E017C0C8
:1039600082E090E014C083E090E011C084E090E039
:103970000EC085E090E00BC086E090E008C087E0D4
:1039800090E005C088E090E002C08FEF9FEFDF91EC
:10399000CF9108952F923F924F925F926F927F92B4
:1039A0008F929F92AF92BF92CF92DF92EF92FF924F
:1039B0000F931F93CF93DF93CDB7DEB72A970FB640
:1039C000F894DEBF0FBECDBF5C016B01042F7901FF
:1039D000672B09F487C021153105F9F0D9018C91C5
:1039E0008823D9F06FE270E0C9010E94E386009756
:1039F00039F0FC011192CF010E945E1C4C0102C003
:103A0000812C912CC7010E945E1C7C01019739F02A
:103A10008A94892809F065C002C0E12CF12C6BE37F
:103A20007AE0C6010E949E7A892B09F40BC267E3F3
:103A30007AE0C6010E949E7A892B09F41FC262E3D4
:103A40007AE0C6010E949E7A892B09F408C26BE2D3
:103A50007AE0C6010E949E7A892B09F403C266E2CD
:103A60007AE0C6010E949E7A892B09F4FEC162E2C7
:103A70007AE0C6010E949E7A892B09F4F9C16DE1B2
:103A80007AE0C6010E949E7A892B09F4F4C168E1AC
:103A90007AE0C6010E949E7A892B09F4D3C162E1C3
:103AA0007AE0C6010E949E7A892B09F4E7C169E099
:103AB0007AE0C6010E949E7A892B09F4E2C160E097
:103AC0007AE0C6010E949E7A892B09F4DDC1D601F5
:103AD0008C918D3251F090ED980F9A3030F0833206
:103AE000B9F1E0C180E090E0DDC1FE0131964F0107
:103AF000412C512C1E2F9A8632012FEF621A720A26
:103B00002301C6010E94777A1C016CE270E0C601B5
:103B10000E94E3866C01892B19F03FEFC31AD30A88
:103B2000D4012D923D924D01C114D10439F0F3E03E
:103B30006F16710409F743E0442E512CD501ED9125
:103B4000FC910190F081E02D212F3A85A20175C0F2
:103B5000CE0107969E01275F3F4F3F932F93215041
:103B600031093F932F939F938F938BE694E09F931C
:103B70008F93DF92CF920E9497870FB6F894DEBFA3
:103B80000FBECDBF039709F0ACCF1F818884998405
:103B9000812F811608F4882DC92C891508F4C82EA8
:103BA0001C198C189C189C2D90959F3F09F448C0B7
:103BB00080E090950E942D1CD82ED094882D90E006
:103BC000810F911D890D911D892BE9F5CD2CC09494
:103BD000D12C10E0212F30E0ADE6B1E00E946A82E6
:103BE000412C512C32014A94A30192010E94388247
:103BF0003A8329832D2D30E0A4E6B0E00E946A824A
:103C0000A30192010E9438823C832B832C2D30E04B
:103C1000A4E6B0E00E946A82A30192010E94388269
:103C20003E832D83D501ED91FC910190F081E02D33
:103C30009E012F5F3F4F43E050E060E070E030C1F5
:103C4000DD24DA94BBCFBFEFDB16F9F0D11002C050
:103C5000DD24D3944D2C512C612C712C6FEF7FEF10
:103C600080E090E0A30192010E943882A12FB0E091
:103C70000E945782172FA82DB0E00E945782872EEE
:103C8000A92DB0E00E945782972E682C712C610EEE
:103C9000711C690C711CEFEF6E167104FCF4611459
:103CA000710419F466246394712C930140E050E090
:103CB0006FEF7FEF80E090E00E943882A12FB0E0AC
:103CC0000E945782172FA82DB0E00E945782872E9E
:103CD000A92DB0E00E945782972E05C0FFEF6F1606
:103CE000710409F06CF42C2D362D230F08F42FEFFE
:103CF000922F2F3F29F080E00E942D1CC82E02C079
:103D0000CC24CA94892D911608F4812F881508F4C3
:103D1000882D81132FC081100DC0182F20E8121B91
:103D200008F410E020E6129F010E10E0111D11248E
:103D3000105386C0282D30E0482F50E0421B530B13
:103D40002417350744F4182D20E6129F010E10E0C9
:103D5000111D112475C016E5180D181B24E0121B47
:103D600008F410E020E6129F010E10E0111D11244E
:103D7000105E66C0881139C091101AC03BEA232F2B
:103D8000211B08F420E04FE2249F020E20E0211DB9
:103D90001124482F431B08F440E0142F30E6139FF2
:103DA000010E10E0111D1124120F1695105C48C071
:103DB000292D30E090E0821B930B192D281739072D
:103DC00044F420E6129F010E10E0111D1124105A38
:103DD00037C025E5121B08F410E020E3129F010E06
:103DE00010E0111D112410582BC011110DC0192DF8
:103DF00020E8121B08F410E020E3129F010E10E0EF
:103E0000111D112418571CC0212F30E0892D90E07E
:103E1000821B930B2817390744F420E6129F010EEA
:103E200010E0111D112410560BC025E5121B08F4DB
:103E300010E020E6129F010E10E0111D1124105415
:103E40001F5FC8CED501ED91FC910190F081E02D6E
:103E500020E030E040E050E061E070E021C063E04D
:103E600070E014C064E070E011C065E070E00EC066
:103E700066E070E00BC067E070E008C062E070E0F0
:103E800005C068E070E002C069E070E0D501ED9126
:103E9000FC910190F081E02D20E030E040E050E026
:103EA000C50119952A960FB6F894DEBF0FBECDBF97
:103EB000DF91CF911F910F91FF90EF90DF90CF9006
:103EC000BF90AF909F908F907F906F905F904F903A
:103ED0003F902F9008958F929F92AF92BF92CF9272
:103EE000DF92EF92FF920F931F93CF93DF93E091B6
:103EF000E90BF091EA0B309709F468C0812EC02FCE
:103F0000932EC22EA52ED42EB72ED62FBC01CF01B4
:103F10000E946C388C01009709F45BC0DC01189694
:103F20008C91853009F055C060E0C8010E945F386F
:103F30007C0161E0C8010E945F38FC0101851285A7
:103F4000D70119962D913C911A972130310569F0CE
:103F50002CF4232BF1F56C2FC80118C02230310549
:103F600049F027303105A9F034C06C2FC801039601
:103F70000E94F53E6D2FC8010E94F53E6D2DC801CF
:103F800001960E94F53E6C2DC80102960E94F53EF6
:103F900020C0892BF1F080858530D9F4E680F78048
:103FA000E114F104B1F00C2F182D2C2D392D4D2DCD
:103FB0005A2D6D2F7B2DF701818592850E946B1FF5
:103FC000D7011296ED90FC901397EACF80E090E035
:103FD00002C081E090E0DF91CF911F910F91FF909F
:103FE000EF90DF90CF90BF90AF909F908F9008950B
:103FF000CF92DF92EF92FF920F931F93CF93DF93B5
:10400000E091670BF091680B3097A1F090859530A7
:1040100089F469017A01EB01682FCF010E945F38B2
:10402000FC0181859285009729F09601A701BE01C8
:104030000E946B1FDF91CF911F910F91FF90EF9026
:10404000DF90CF900895AF92BF92CF92DF92EF9220
:10405000FF920F931F93CF93DF938091620B909108
:10406000630B892B09F472C0E1E0F0E0C0E0D0E01E
:10407000CC24C394D12CB6010C2E02C0660F771F3E
:104080000A94E2F740915B0650915C067F0184E060
:10409000E80EF11CCF01B12C9C01A0910602B09159
:1040A0000702A817B90720F42091060230910702F1
:1040B000A091E30BB091E40BA20FB31FAC90A091C1
:1040C000620BB091630B9C0121503109A20FB31F09
:1040D0000A2D10E02C9130E00217130729F0462B2F
:1040E000572BAC92BB24B3940196E816F906A1F6BF
:1040F00050935C0640935B06BB2011F18091620BEC
:104100009091630BE80FF91F028110E0218130E0EC
:10411000408150E03197608170E0CE010E94F81F2D
:104120000E94336BDC01CB01845D9E4FAF4FBF4FCC
:104130008093570690935806A0935906B0935A0659
:104140002196F701C430D10509F095CFDF91CF91C9
:104150001F910F91FF90EF90DF90CF90BF90AF90A5
:104160000895DC011296ED91FC911397309721F0A0
:1041700081E09085953009F080E00895CF92DF923C
:10418000EF92FF92CF93DF93DC011696ED91FC91B5
:104190001797309721F12085223009F56A017B01BC
:1041A000EC0168EF79E08FE698E00E94CF5D62EF66
:1041B00079E08FE698E00E94CF5D2AE030E0B70119
:1041C000A6018FE698E00E94515E8FE698E00E947B
:1041D000F25EEE81FF81C186D286E386F486DF91AE
:1041E000CF91FF90EF90DF90CF900895FC018681F2
:1041F0009781009789F0FC012085223041F025301D
:1042000079F460E00E945F38009779F0FC016185E5
:1042100072858385948508956FEF7FEFCB010895B4
:104220006EEF7FEF8FEF9FEF08956DEF7FEF8FEFD2
:104230009FEF08950F931F93CF93DF93FC01C481E9
:10424000D581209799F08885823029F4672B71F405
:1042500089859A8518C0853061F48B01CE010E9452
:10426000FA3B90E0081719073CF003C08FEF9FEF6F
:104270000AC08EEF9FEF07C0602FCE010E945F380B
:10428000FC0181859285DF91CF911F910F91089557
:10429000CF93C62F63E0FC01828193810E945F3837
:1042A0000097D9F04C2F50E060E070E0FC014187AE
:1042B0005287638774876AEE79E08FE698E00E9400
:1042C000CF5D4AE050E06C2F8FE698E00E94A05E40
:1042D0008FE698E0CF910C94F25ECF910895CF9342
:1042E000C62F63E0FC01828193810E945F380097B2
:1042F00031F0FC018185C11103C08F7001C08FEFC7
:10430000CF910895BF92CF92DF92EF92FF920F93D9
:104310001F93CF93DF93EC010E94B120882309F40F
:1043200041C08A819B810E94FA3B082F10E0C8019E
:10433000880F991F9C0125593D4F790132E0B32E1A
:1043400004301105D4F4F701C190D1907F010E948F
:10435000F22E009751F0FC01B086A601DD0C660B31
:10436000770B4187528763877487BC018A819B8161
:104370000E9487380F5F1F4FE3CF0A811B8160E0E7
:10438000C8010E945F38FC018185888761E0C8010F
:104390000E945F389D838C8362E0C8010E945F3871
:1043A0009F838E83DF91CF911F910F91FF90EF90AC
:1043B000DF90CF90BF900895CF93DF93EC01FB0186
:1043C0002481358140815181628173810E94515ED7
:1043D000CE01DF91CF9108958F929F92AF92BF92BD
:1043E000CF92DF92EF92FF920F931F93CF93DF93C1
:1043F000CDB7DEB7C054D1090FB6F894DEBF0FBEFB
:10440000CDBF8C015B01FC01F38068EB79E08FE6A6
:1044100098E00E94CF5D4AE050E06F2D8FE698E073
:104420000E94A05E66EB79E08FE698E00E94CF5D87
:104430004AE050E0B5018FE698E00E94995E8FE671
:1044400098E00E94F25EF801C080D18066E774E0D7
:10445000C6010E946C384C016BE774E0C6010E94F3
:104460006C387C0160E874E0C6010E946C388C01F5
:1044700065E874E0C6010E946C386C010097B9F1E0
:10448000FC016185728540E450E0CE0101960E94F6
:104490001C876FE270E0CE0101960E94E386892BB3
:1044A00051F4F6012185328543E050E060E4CE010D
:1044B00001960E943726A114B10441F0E114F104E1
:1044C00019F46AE874E00FC0F70107C0011511057F
:1044D00019F46DE874E007C0F80161857285FB018D
:1044E0008081882321F0CE0101960E94C56381144A
:1044F0009104E9F1F40161857285CE0101960E9473
:10450000AE61CE0101960E94B120882381F1AB28D3
:1045100079F0E114F10451F4E12CF12C01E020E0F8
:1045200030E040E050E061E070E00EC0F70112C002
:104530000115110571F4E12CF12C01E020E030E0CF
:1045400040E050E062E070E0CE0101960E94B909BF
:104550000EC0F80161857285FB018081882339F0E6
:1045600020E030E041E0CE0101960E94CA1CC05C10
:10457000DF4F0FB6F894DEBF0FBECDBFDF91CF91F6
:104580001F910F91FF90EF90DF90CF90BF90AF9071
:104590009F908F900895EF92FF920F931F93CF9368
:1045A000DF9380915B0690915C06C4E0D0E021E04F
:1045B00030E0AC0142235323452B29F0A90140955B
:1045C000509584239523220F331F219791F79093C1
:1045D0005C0680935B060E94336B00915706109136
:1045E00058062091590630915A06601771078207C4
:1045F000930708F459C0012B022B032B09F454C074
:1046000010925706109258061092590610925A06A8
:10461000E12CF12CE091620BF091630BEC0FFD1F8C
:10462000038110E0228130E0418150E0608170E040
:10463000C7010E94F81F8FEFE81AF80A249684E059
:10464000E816F10439F7C1E0D0E0809106029091BC
:1046500007028C179D0728F48091060290910702AB
:1046600001C0CE012091E30B3091E40BF901E80F7A
:10467000F91F4AE050E060818FE698E00E94A05E5A
:1046800061E974E08FE698E00E94F65E2196C13100
:10469000D105D9F68FE698E0DF91CF911F910F9168
:1046A000FF90EF900C94F25EDF91CF911F910F91EC
:1046B000FF90EF90089585ED8093BC008091BC0041
:1046C00084FDFCCF1092AF0B089540918706262FF2
:1046D00030E0240F311D21323105DCF42091AF0B85
:1046E0002430C9F4FC0180E090E0861758F4309142
:1046F00087062191DC01A959B94FA30FB11D2C9355
:104700000196F3CF80918706680F6093870680E05B
:10471000089581E0089582E0089508950895E09154
:10472000880B8091870BE81730F4F0E0E655F94FDD
:10473000808190E008958FEF9FEF08959091880B0E
:104740008091870B981750F4E92FF0E0E655F94F68
:10475000208130E09F5F9093880B02C02FEF3FEFE6
:10476000C90108958091870B90E02091880B821BEE
:1047700091090895CF92DF92EF92FF920F931F93CA
:10478000CF93DF937C01CB018A012091B00B2223D0
:1047900089F0EB016B01C40ED51ECC15DD0569F067
:1047A0006991D701ED91FC910190F081E02DC70155
:1047B0001995F3CF642F0E946523C801DF91CF9133
:1047C0001F910F91FF90EF90DF90CF900895CF93BE
:1047D000DF931F92CDB7DEB769832091B00B222300
:1047E000D1F02091D30B203240F021E030E0FC01E9
:1047F0003383228380E090E015C08091B10BE82FD5
:10480000F0E0EE54F44F998190838F5F8093B10B69
:104810008093D30B05C061E0CE0101960E94652311
:1048200081E090E00F90DF91CF910895A8950895D1
:1048300060E08DE00C946E3661E08DE00C946E3695
:10484000FC0181819091AF0B9111FCCF91E090938D
:10485000AF0B9093AE0B2FEF2093AD0B1092AC0BE0
:104860001092AB0B90938A0B90918A0B880F892B37
:1048700080938A0B8091890B813061F41092890BAF
:1048800080918A0B8093BB008091BC0083FDF8CFA0
:1048900085EC01C085EE8093BC008091AF0B813028
:1048A000E1F38091AC0B811103C09091AC0B01C07E
:1048B00091E0EBE8FBE0AAEAB6E080E0891721F09E
:1048C00021912D938F5FFACF1092880B8093870BE5
:1048D0008AE199E00E949E23089581E00C94185487
:1048E000FC01818191E09093B00B8093D20B1092E8
:1048F000B10B1092D30B08951F93CF93DF93EC016C
:10490000162F0E94702461EE8AE199E00E94E7234D
:10491000612F8AE199E00E94E723CE01DF91CF91D8
:104920001F910C946D24CF93DF93EC0163EC0E94F4
:104930007C24CE01DF91CF910C942024CF93DF9380
:10494000EC010E949324682F6460CE01DF91CF9127
:104950000C94B33F1F920F920FB60F9211240BB617
:104960000F922F933F934F935F936F937F938F9308
:104970009F93AF93BF93EF93FF938091B900887F8C
:10498000803609F49CC068F5883209F45BC090F465
:10499000803109F454C038F4882309F4F6C0883013
:1049A00009F44DC0F6C0883109F44CC0803209F4D6
:1049B0005DC0EFC0803409F468C048F4803309F466
:1049C00055C0883309F0E5C08093AD0BD8C0803561
:1049D00009F44FC0883509F45DC0883409F0D9C0A6
:1049E000D6C0883909F4C7C0A8F4883709F467C06D
:1049F00038F4883609F463C0803709F460C0C9C050
:104A0000883809F4B8C0803909F45FC0803809F0EB
:104A1000C0C05BC0803B09F486C038F4803A09F41A
:104A200066C0883A09F47FC0B4C0803C09F4A7C0CE
:104A3000883C09F4A4C0883B09F48AC0AAC08091CC
:104A40008A0B10C09091AC0B8091AB0B981770F54E
:104A5000E091AC0B81E08E0F8093AC0BF0E0E5575A
:104A6000F44F80818093BB0085EC86C08093AD0BB2
:104A70008EC0E091AC0B81E08E0F8093AC0B8091E7
:104A8000BB00F0E0E557F44F80839091AC0B809130
:104A9000AB0B6EC0E091AC0B81E08E0F8093AC0B42
:104AA0008091BB00F0E0E557F44F80838091AE0B1E
:104AB00081116DC081E08093890B84EA61C083E03D
:104AC0008093AF0B1092A906CFCF8091A9068032B8
:104AD00008F051C0E091A90681E08E0F8093A906ED
:104AE0008091BB00F0E0E757F94F8083BDCF85ECA4
:104AF0008093BC001092AF0B8091A906803230F4F5
:104B0000E091A906F0E0E757F94F10826091A906FD
:104B100070E0E091830BF091840B89E896E01995A1
:104B20001092A90636C084E08093AF0B10928806DD
:104B300010928706E091850BF091860B1995809174
:104B40008706811105C081E0809387061092670671
:104B5000E091880681E08E0F80938806F0E0E959A5
:104B6000F94F80818093BB009091880680918706E1
:104B7000981708F479CF85E88093BC000AC085ECCB
:104B80008093BC001092AF0B04C01092AD0B0E943A
:104B90005B23FF91EF91BF91AF919F918F917F9197
:104BA0006F915F914F913F912F910F900BBE0F909E
:104BB0000FBE0F901F9018958F929F92AF92BF9249
:104BC000CF92DF92EF92FF920F931F93CF93DF93D9
:104BD000CDB7DEB72B970FB6F894DEBF0FBECDBFB3
:104BE0008C01CE0101967C016C018AE0882E912C0B
:104BF000A12CB12CC6018E199F09411551056105E3
:104C0000710581F0CB01BA01A50194010E941682C1
:104C1000942F852F605DF60161936F01A901692FC3
:104C2000782FE8CFFC013197EE0DFF1DD8019E01D2
:104C30002150310940814D933197E217F307D1F7A5
:104C4000F801E80FF91F10822B960FB6F894DEBF1B
:104C50000FBECDBFDF91CF911F910F91FF90EF90CD
:104C6000DF90CF90BF90AF909F908F9008958F92DC
:104C70009F92AF92BF92CF92DF92EF92FF920F93EB
:104C80001F93CF93DF938C014A016901E090610685
:104C9000F0906206C62F660FDD0BE114F10449F1B6
:104CA000F7018085863029F563E974E0C7010E9429
:104CB0006C385C01F2E08F16910439F083E08816BD
:104CC000910451F46FEC74E002C068E974E0C7012C
:104CD0000E946C387C0102C0E12CF12CA114B104BB
:104CE00051F0F50161857285AE01C8010E941C87F3
:104CF00008C0E12CF12CAE0169E97BE0C8010E94FB
:104D0000B77AAE0163E274E0C8010E94FE86E11446
:104D1000F10421F0F701618572850FC0F2E08F1672
:104D20009104A1F083E08816910461F08A948928A7
:104D300099F460915F0670916006AE01C8010E940F
:104D4000FE860AC0AE0163E97BE003C0AE0160E904
:104D50007BE0C8010E94A77AAE0163E274E0C8015B
:104D60000E94FE86C114D10429F0AE01B601C8012B
:104D70000E94FE86C801DF91CF911F910F91FF9095
:104D8000EF90DF90CF90BF90AF909F908F9008955D
:104D90009FE9980F963010F4875508959FEB980F70
:104DA000963010F48753089580538A3008F080E0DD
:104DB0000895CF93DF93DA01382FEC018C2F831BFA
:104DC0008617C8F4CE01E991F0E024E0F595E79567
:104DD0002A95E1F7ED58FD4F20812C93FC0180814D
:104DE000E82FEF70F0E0ED58FD4F808111968C9325
:104DF00011971296E3CFFA01E60FF11DE60FF11DB0
:104E00001082DF91CF9108950F931F93CF93DF937B
:104E1000FC0120852530B9F48B01EC0160E00E9493
:104E20005F38FC0181859285A385B4850597A1052E
:104E3000B10549F4CE010E94FA3B282F30E081E011
:104E4000201731070CF480E0DF91CF911F910F9173
:104E500008952F923F924F925F926F927F928F921E
:104E60009F92AF92BF92CF92DF92EF92FF920F93F9
:104E70001F93CF93DF93CDB7DEB7CD55D1090FB6D2
:104E8000F894DEBF0FBECDBF00915D0610915E06A7
:104E90000115110509F4B1C20E94336BC09063067D
:104EA000D0906406E0906506F0906606C616D706B8
:104EB000E806F90608F0A1C2F801A680B780A1149F
:104EC000B10409F45DC1F5018085863009F054C153
:104ED0006396BFAEAEAE639767961FAE1EAE679782
:104EE00064961FAE649765961FAE65976DE974E092
:104EF000C5010E946C38009729F0FC0181856496F9
:104F00008FAF6497F501808191810E94777A182F85
:104F100065968FAF65976FE974E0C5010E946C38A4
:104F20000097A9F564960FAD64976BE87BE08FE678
:104F300098E00E94CF5D4AE050E0612F8FE698E054
:104F40000E94A05E69E87BE08FE698E00E94CF5D5A
:104F50004AE050E0602F8FE698E00E94A05E8FE666
:104F600098E00E94F25E40E050E06FE974E06396E2
:104F70008EAD9FAD63970E94A4386FE974E063968D
:104F80008EAD9FAD63970E946C38009729F009960B
:104F900067969FAF8EAF67976596FFAC6597FF20CA
:104FA00009F4EAC067968EAD9FAD6797892B09F427
:104FB000E3C064968FAD6497F82FF270DF2E86FF02
:104FC00006C161EA74E063968EAD9FAD63970E945F
:104FD0006C388C01D110E4C062E08F2D0E94BD6A54
:104FE00065968FAD6597863308F0865390917B0068
:104FF000282F2870977F922B90937B008770806476
:1050000080937C0080917A00806480937A00809104
:105010007A0086FDFCCFC090780080917900D12C79
:10502000D82A0115110509F4CBC1F8018085853016
:1050300009F0C6C1C8010E94FA3B6E968FAF6E9709
:10504000843008F4AFC063E0C8010E945F38FC01FF
:105050008184928462E0C8010E945F38FC0141842F
:1050600052846384748461E0C8010E945F381C012B
:1050700060E0C8010E945F38FC01218532854385CC
:1050800054856D962CAF3DAF4EAF5FAF6D97C601A7
:10509000DD0CAA0BBB0B9C01AD016D96CCACDDAC5D
:1050A000EEACFFAC6D972C193D094E095F09C401A8
:1050B000092C000CAA0BBB0BBC01CD0164197509AE
:1050C000860997090E940682F10121853285438570
:1050D00054852C193D094E095F090E943882420E01
:1050E000531E641E751E62016E96FFAD6E97F530FD
:1050F00009F058C064E0C8010E945F38FC01818556
:1051000092858C149D040CF464016E96FFAD6E972D
:10511000F23009F057C10D2C000CEE08FF0860E0DA
:10512000C8010E945F38FC0181859285A385B48502
:10513000C816D906EA06FB06C4F5C12CD12C679621
:10514000EEADFFAD6797828193818C159D0561F06F
:10515000B601CE018F5A9F4F0E94EC216796EEADAB
:10516000FFAD6797D382C2826796EEADFFAD6797BA
:10517000818185300CF496C0F501A280B3809FCE6A
:105180000E94336BDC01CB01C296A11DB11D80933F
:10519000630690936406A0936506B09366062DC1DE
:1051A00060E01BCF81E090E0ACCF61E0C8010E94DD
:1051B0005F38FC0181859285A385B4858C159D059A
:1051C000AE05BF05CCF6CC24C394D12CB8CFD110FA
:1051D00003C010E062E002C011E060E08F2D0E9489
:1051E000BD6A65962FAD659730E0F901E654F44F3E
:1051F0008491F901E65EF34F0491F901E05AF34F0F
:10520000F490FF20A1F081110E94676AEF2DF0E079
:10521000EE0FFF1FE759F44FA591B491EC910E23C7
:1052200031E020E009F430E0832F922F02C080E0CB
:1052300090E0212F30E051E02817390709F050E0C5
:10524000052F10E06796EEADFFAD67976281738121
:105250000617170719F14181442319F04150418382
:105260008BCF64964FAD649740FF0AC0281739076B
:1052700071F461E08081811160E0608370E002C0C0
:105280005083B801CE018F5A9F4F0E94EC21679640
:10529000EEADFFAD6797138302836ECF93E0C92E07
:1052A000C1826ACF828193818C159D0509F464CFF8
:1052B0006996DFAECEAE699765961FAD659765E8D6
:1052C0007BE08FE698E00E94CF5D4AE050E0612FDE
:1052D0008FE698E00E94A05E63E87BE08FE698E0AE
:1052E0000E94CF5D4AE050E0B6018FE698E00E9450
:1052F000995E8FE698E00E94F25E63960EAD1FAD58
:10530000639766E774E0C8010E946C383C0165E869
:1053100074E0C8010E946C388C01009761F1FC01B7
:105320006185728540E450E0CE0101960E941C87A1
:105330006FE270E0CE0101960E94E386892B51F462
:10534000F8012185328543E050E060E4CE0101960A
:105350000E9437264AE0BE016F5B7F4F69968EAD93
:105360009FAD69970E94F17ABE016F5B7F4FCE01BE
:1053700001960E94C56361147104D9F0F30161853F
:105380007285CE0101960E94AE61CE0101960E9407
:10539000B120882371F0E12CF12C01E09E01295A03
:1053A0003F4F41E050E060E070E0CE0101960E9486
:1053B000B9096796EEADFFAD6797D382C282DCCEA6
:1053C00081E090E06796EEADFFAD67972281338173
:1053D0007601E21AF30A9701F7FE03C03195219591
:1053E00031098217930714F41182BECE8181863071
:1053F0000CF0BACE8F5F8183B7CEC35ADF4F0FB6A2
:10540000F894DEBF0FBECDBFDF91CF911F910F91FA
:10541000FF90EF90DF90CF90BF90AF909F908F90D4
:105420007F906F905F904F903F902F900895A89538
:105430000E945B12029724F00E948E570E94292737
:105440000C94CB2267E47BE08FE698E00E94CF5D6E
:1054500064E37BE08FE698E00E94CF5D66E27BE04C
:105460008FE698E00E94CF5D6EE17BE08FE698E0EA
:105470000E94CF5D8FE698E00E94F25E61E17BE0E2
:105480008FE698E00E94CF5D61E07BE08FE698E0D8
:105490000E94CF5D65EF7AE08FE698E00E94CF5DD5
:1054A0006EED7AE08FE698E00E94CF5D6CEC7AE0DA
:1054B0008FE698E00E94CF5D67EB7AE08FE698E098
:1054C0000E94CF5D68EA7AE08FE698E00E94CF5DA7
:1054D00060EA7AE08FE698E00E94CF5D65E97AE0C5
:1054E0008FE698E00E94CF5D6BE87AE08FE698E067
:1054F0000E94CF5D63E87AE08FE698E00E94CF5D7E
:1055000067E77AE08FE698E00E94CF5D6DE57AE08C
:105510008FE698E00E94CF5D6EE37AE08FE698E038
:105520000E94CF5D8FE698E00C94F25ECF93DF93FC
:10553000EC01E881F9810284F385E02DCE01199513
:105540000196B9F7DF91CF910895FC01A285B3854B
:105550001097A9F086859785029788F0CD0101966E
:10556000938782876C93868597850197978786872F
:105570000284F385E02D108281E090E0089580E0C0
:1055800090E00895FC01868197818F3F2FEF92076D
:1055900029F02FEF3FEF378326830895A085B1854B
:1055A000109789F0248535852115310561F0CD01ED
:1055B0000196918780878C91215031093587248706
:1055C000082E000C990B0895FC01868197810196A5
:1055D00039F481E024853585232B19F480E0089582
:1055E00081E00895CF92DF92EF92FF920F931F9385
:1055F000CF93DF937C016A018B01C0E0D0E0CC1532
:10560000DD0589F0D701ED91FC910284F385E02D51
:10561000C70119958F3FBFEF9B0729F0F8018193D0
:105620008F012196ECCFCE01DF91CF911F910F9189
:10563000FF90EF90DF90CF900895CF93C62FDC01BD
:10564000ED91FC910088F189E02D1995DC01ED9137
:10565000FC910190F081E02D6C2FCF911994CF93A4
:10566000DF93EC018E819F810196D9F428853985DD
:105670008A859B85820F931F81159041A0F4E88154
:10568000F9810284F385E02DCE01199581329105CF
:105690006CF3E881F9810684F785E02D682FCE014F
:1056A000199581E001C080E0DF91CF910895062E29
:1056B000000C770BFC01778366830895CF93DF930B
:1056C000EC018E819F81019611F5E881F9810088B6
:1056D000F189E02DCE011995DC01ED91FC9100845A
:1056E000F185E02D1995892BA1F0E881F9810284DB
:1056F000F385E02DCE0119958132910534F3E881CF
:10570000F9810684F785E02D682FCE01199581E097
:1057100001C080E0DF91CF9108950F931F93CF9345
:10572000DF93EC018B0165EA74E00E94F65E0115DF
:105730001105B9F1F80161918F01662391F1603291
:1057400020F0623211F06C3541F56CE5CE010E941B
:10575000C85DF801319780818C30D1F044F48930F4
:10576000D9F08A30B9F0883029F762E616C0823263
:1057700059F024F48D30F1F662E70FC08F3231F02A
:105780008C35C1F66CE509C062E207C06FE205C066
:1057900066E603C06EE601C064E7CE010E94C85D04
:1057A000C9CF62E2CE010E94C85D80E090E0DF9147
:1057B000CF911F910F910895FC012085318582853D
:1057C0009385AC014F5F5F4F53874287820F931FD2
:1057D0000E94F88181E090E00895FC018681978124
:1057E0008F3F2FEF920729F02FEF3FEF378326836C
:1057F00008952085318582859385AC014F5F5F4F89
:1058000053874287820F931F0E94F081082E000C5D
:10581000990B0895FC01868197818F3F2FEF9207A6
:1058200029F02FEF3FEF37832683089580859185F8
:105830000C94807BCF92DF92EF92FF92CF93DF9315
:10584000EC018E819F818F3F2FEF920759F02FEF50
:105850003FEF3F832E83DF91CF91FF90EF90DF905A
:10586000CF9008950E94336B6B017C01A4EFCA0EA8
:10587000A1E0DA1EE11CF11CE881F9810088F189C0
:10588000E02DCE011995DC01ED91FC910084F185AC
:10589000E02D1995892B39F40E94336B6C157D0529
:1058A0008E059F0548F3E881F9810088F189E02D94
:1058B000CE011995DC01ED91FC910284F385E02D78
:1058C000DF91CF91FF90EF90DF90CF901994EF92FE
:1058D000FF920F931F93CF93DF93009719F48FEFED
:1058E0009FEF82C0FC01E484F584D7010D911C91E7
:1058F000D801ED91FC910688F789E02DC801199532
:10590000882369F3D801ED91FC910084F185E02DA5
:10591000C8011995D801ED91FC91892B61F302849E
:10592000F385E02DC8011995EC010196C1F2F8014B
:105930008589882339F04AE050E06C2F8FE698E0A3
:105940000E94A05ED70112968C91882309F44BC067
:10595000C532D10509F047C0D801ED91FC91008412
:10596000F185E02DC801199502975CF0D801ED9101
:10597000FC910688F789E02DC80119958111ECCFBB
:10598000AECFD1E0C0E0D801ED91FC910284F38567
:10599000E02DC80119958F3FBFEF9B0709F49FCFFA
:1059A0009C01215431092A31310530F09C012156E6
:1059B00031092A31310538F48D2F8295807F829FFD
:1059C000C00D11240AC0C0978A30910530F49D2F74
:1059D0009295907F989FC00D1124D150A0F68C2FE6
:1059E000CC0F990B01C0CE01DF91CF911F910F9188
:1059F000FF90EF9008958F929F92AF92BF92CF92B7
:105A0000DF92EF92FF920F931F93CF93DF93611575
:105A1000710509F4FFC0FB010085002E000C110B7D
:105A2000220B330B0730110508F0F4C0DB01EC0149
:105A3000F8018827E654FF4F8F4F0C948D8267EA58
:105A400074E006C019968C91882389F06CEA74E0A2
:105A5000CE01DF91CF911F910F91FF90EF90DF90DA
:105A6000CF90BF90AF909F908F900C94F35D61EBBF
:105A700074E0EECF19964D915D916D917C911C97DC
:105A80002AE030E0CE01DF91CF911F910F91FF907E
:105A9000EF90DF90CF90BF90AF909F908F900C943D
:105AA000515E1996CD90DD90ED90FC901C9720E012
:105AB00030E0A901C701B6010E942C8387FF09C00D
:105AC00067EB74E0CE010E94F65EF7FAF094F7F807
:105AD000F094C701B6010E94AA834B015C012AE041
:105AE000AB01BC01CE010E94085E69EB74E0CE01FF
:105AF0000E94F65EC501B4010E94D9839B01AC01EE
:105B0000C701B6010E94BF822DEC3CEC4CE45DE382
:105B10000E94C08220E030E040E251E40E94908484
:105B20000E94AA83AB0160E070E02AE0CE010E94EF
:105B3000085E70C019966D917C911A97CE01DF9125
:105B4000CF911F910F91FF90EF90DF90CF90BF907A
:105B5000AF909F908F900C948D2B16960D911C9169
:105B600017976BE5CE010E94C85D019619F48FEF7F
:105B70009FEF52C00115110571F0B801CE010E94CE
:105B8000FB2C0196A1F3F801028113810115110587
:105B900089F36CE2E7CF6DE52FC016960D911C914D
:105BA00017976BE7CE010E94C85D019601F30115BE
:105BB000110509F1F80160817181CE010E948D2BE0
:105BC0000196A9F26AE3CE010E94C85D019679F2BE
:105BD000B801CE010E94FB2C019649F2F801028126
:105BE00013810115110519F36CE2CE010E94C85D05
:105BF0000196E9F6BCCF6DE7CE010E94C85D21E0B9
:105C000030E0019611F020E030E088279927821BD0
:105C1000930B02C080E090E0DF91CF911F910F9134
:105C2000FF90EF90DF90CF90BF90AF909F908F90BC
:105C30000895CF93DF93EC01E881F9810284F38525
:105C4000E02DCE0119958F3F2FEF920771F0E8817B
:105C5000F9818132910594F30684F785E02D682F50
:105C6000CE01199580E090E002C08FEF9FEFDF91A9
:105C7000CF910895EF92FF920F931F93CF93DF93ED
:105C80008C017B01DC01ED91FC910284F385E02D18
:105C90001995829709F078C084E0F701808786E043
:105CA00090E00E94A777EC01892B09F46DC0EAEC23
:105CB000F6E0F983E88380E091E0DF019C011D922A
:105CC00021503040E1F79B838A831D821C82D801DA
:105CD000ED91FC910284F385E02DC80119958F3F69
:105CE000BFEF9B0709F44DC08232910509F44FC004
:105CF000803291050CF44BC08C35910511F0BE013A
:105D00003DC0D801ED91FC910284F385E02DC801DE
:105D100019958F3FBFEF9B07A1F18236910531F1B5
:105D20005CF48F329105F9F08C359105C9F08297BA
:105D300071F6BE0182E222C08E369105D1F034F4B4
:105D40008636910521F6BE018CE018C08237910598
:105D500099F08437910509F0BACFBE0189E00EC0F1
:105D6000BE018CE50BC0BE018FE208C0BE0188E019
:105D700005C0BE018AE002C0BE018DE00E949961AB
:105D8000A6CFCE010E943F788FEF9FEF24C08C8179
:105D90009D81009749F0E881F9818E0F9F1FFC01DA
:105DA00031978081882321F0BE0180E00E949961B3
:105DB0008C819D810E94A7778C01009739F06AEC55
:105DC00076E00E94F786CE010E943F78F7011287A5
:105DD000018780E090E0DF91CF911F910F91FF90BC
:105DE000EF9008958DE090E00E94A777009729F04A
:105DF0002DE0FC0111922A95E9F708950F931F9366
:105E0000CF93DF930097E1F0EC010C851D85011520
:105E1000110579F0D8018D919C91009739F0DC0142
:105E2000ED91FC910488F589E02D1995C8010E9437
:105E30003F78CE01DF91CF911F910F910C941E7B83
:105E4000DF91CF911F910F910895AF92BF92CF92A2
:105E5000DF92EF92FF920F931F93CF93DF9300D0C7
:105E60001F92CDB7DEB76115710509F496C06B01BD
:105E7000182FDB011C96AD90BC901D97F501E080BA
:105E8000F180D701ED91FC910688F789E02DC701DB
:105E90001995811104C0C6010E94FE2E7EC0F50135
:105EA0009281911114C0D701ED91FC910190F08184
:105EB000E02D612FC7011995F7018589882309F421
:105EC00069C0612F8FE698E00E94C85D63C0812F92
:105ED0008F7D81548A3138F380ED810F8A3018F339
:105EE00083ED810F8230F8F21F35E9F21E37D9F2C7
:105EF0001132B1F086EC810F823090F08AED810F83
:105F0000873070F01D3361F0812F8F7E8F3241F02A
:105F10008DED810F823020F01B3511F01D3511F40D
:105F200091FFC1CF19821A821B821C82812F012E00
:105F3000000C990B9F931F938BEB94E09F938F938F
:105F40008E010F5F1F4F1F930F930E9468876E0192
:105F5000F4E0CF0ED11C0F900F900F900F900F9088
:105F60000F90D701ED91FC910190F081E02DD801C7
:105F70006C91C7011995F7018589882331F0D80103
:105F80006C918FE698E00E94C85D0F5F1F4F0C1563
:105F90001D0539F780E090E002C08FEF9FEF0F9072
:105FA0000F900F900F90DF91CF911F910F91FF9065
:105FB000EF90DF90CF90BF90AF9008952C9A089506
:105FC0002C980895CF92DF92EF92FF920F931F9338
:105FD000CF93DF93EC017A018B016C01C40ED51EC7
:105FE000CC15DD05A9F00E94E02F8FE00E948B42C6
:105FF0008D2F0E948B428C2F0E948B42219680E035
:106000000E948B42F80181938F010E94DE2FE8CF1E
:10601000C701DF91CF911F910F91FF90EF90DF901B
:10602000CF900895CF92DF92EF92FF920F931F933C
:10603000CF93DF93EC017A018B016C01C40ED51E66
:10604000CC15DD05A1F00E94E02F80EF0E948B426D
:106050008D2F0E948B428C2F0E948B422196F8013B
:1060600081918F010E948B420E94DE2FE9CFC701F0
:10607000DF91CF911F910F91FF90EF90DF90CF9024
:1060800008951F93CF93DF93D82F192FC62F0E9407
:10609000E02F80EF0E948B42812F0E948B428D2F38
:1060A0000E948B428C2F0E948B420E94DE2F81E047
:1060B000DF91CF911F9108951F93CF93DF93182FF6
:1060C00066E270E00E941D44C82FD0E067E270E0F5
:1060D000812F0E941D44DC2FCC279E01282BC90153
:1060E000DF91CF911F9108951F93CF93DF93182FC6
:1060F00060E270E00E941D44C82FD0E061E270E0D1
:10610000812F0E941D44DC2FCC279E01282BC90122
:10611000DF91CF911F9108957F928F929F92AF92BE
:10612000BF92CF92DF92EF92FF920F931F93CF9384
:10613000DF93CDB7DEB7A6970FB6F894DEBF0FBEDC
:10614000CDBF8C01762E942E852E20E2B22ECE016C
:1061500001967C01FC012B2D11922A95E9F78AE129
:1061600093E09AA389A38FEF8BA38CA38DA38EA317
:10617000680183E4C80ED11C43E450E0BE016F5DAA
:106180007F4FC6010E94CC46019609F4B9C081E058
:1061900089838A8386E0A82EAB821C82F801648101
:1061A0007581868197810E9495826D837E838F831E
:1061B000988789869A8680E890E09C878B874CE157
:1061C00050E0B701C6010E942142F7012B2D119228
:1061D0002A95E9F7480188E0880E911CF401D7015F
:1061E00001900D92AA94E1F740E150E0B701C60199
:1061F0000E942142F7011192BA94E9F796E0A92E84
:10620000B12C40E250E0B701C6010E942142F1E00A
:10621000AF1AB108B1F783E6898392E89A8393E5D0
:106220009B838C8385E38D8381E08E837F829DE3D6
:10623000988797E099878A8786E0F401DE011B96AC
:1062400001900D928A95E1F78CE0898B8A8B61EC45
:1062500074E0CE0143960E94F786F8016385CE0173
:1062600049960E946D5AF8016485CE014B960E94B2
:106270006D5AF8016585CE014D960E946D5A4EE12A
:1062800050E0B701C6010E942142F3E07F121EC018
:1062900082E3898384E08A83F80196859B839785CE
:1062A0009C8390899D8391899E8396E39F838887B1
:1062B000828D8987838D8A87848D8B87858D8C8756
:1062C0004CE050E0B701C6010E94214287E3898378
:1062D00086E08A8391E09B8393E09C838D838FE0AB
:1062E0008E838AE38F838BE388878FEF898749E0EA
:1062F00050E0B701C6010E942142C6010E94F94543
:10630000A6960FB6F894DEBF0FBECDBFDF91CF913A
:106310001F910F91FF90EF90DF90CF90BF90AF90C3
:106320009F908F907F9008952F923F924F925F920F
:106330006F927F928F929F92AF92BF92CF92DF9295
:10634000EF92FF920F931F93CF93DF9300D000D073
:10635000CDB7DEB78C010E9413792FEC37E040E017
:1063600050E00E943882DC01CB010196A11DB11DD5
:10637000F80184839583A683B78380839183A28366
:10638000B3835801F3E4AF0EB11CC5010E94C043B2
:1063900064E470E0C5010E94CC45882309F436C14D
:1063A0000E94336B2B013C01812C912CC8018E5B28
:1063B0009F4F9E838D8348EEC42E43E0D42EE12C64
:1063C000F12C52E0252EAD81BE818C91833009F4F1
:1063D00004C1811120C0F80184819581A681B78113
:1063E0000196A11DB11D84839583A683B7830E9466
:1063F000336B6419750986099709A70196010E94F4
:106400001682A90161E0C8010E948C3081E0AD8153
:10641000BE818C93CAC08430F9F4F80184819581DF
:10642000A681B7810196A11DB11D84839583A683A2
:10643000B7830E94336B6419750986099709A70110
:1064400096010E941682A90163E0C8010E948C3067
:10645000AD81BE812C92A9C0813059F5F80142ADC1
:1064600053AD64AD75AD9E012F5F3F4FC8010E94D3
:10647000825A382EF2E08F1392C089819A81AB81C3
:10648000BC81F80184839583A683B7830E94336B14
:106490006419750986099709A70196010E94168259
:1064A000A90163E0C8010E948C30AD81BE813C929D
:1064B0007CC0823009F079C0F80142AD53AD64ADC3
:1064C00075AD9E012F5F3F4FC8010E94825A382E42
:1064D000F5E08F135DC0E3E0AD81BE81EC93F80180
:1064E00082A193A1A4A1B5A1892B8A2B8B2B41F466
:1064F00084E893E0A0E0B0E082A393A3A4A3B5A3B3
:10650000F80186A197A1A0A5B1A5892B8A2B8B2B79
:1065100061F482A193A1A4A1B5A1B695A795979581
:10652000879586A397A3A0A7B1A7F80182A593A5F5
:10653000A4A5B5A5892B8A2B8B2BA9F482A193A1A5
:10654000A4A1B5A1AC01BD0123E07695679557954F
:1065500047952A95D1F7841B950BA60BB70B82A7FD
:1065600093A7A4A7B5A7F80186A197A1A0A5B1A557
:1065700086A797A7A0ABB1AB82A593A5A4A5B5A507
:1065800082AB93ABA4ABB5AB88248394912C0DC0A4
:10659000F6E08F1304C0AD81BE811C9206C0BFEF30
:1065A0003B1203C0ED81FE811082F1E08F16910451
:1065B00009F409CF0E94336BDC01CB0184199509E2
:1065C000A609B709F80126A937A940AD51AD28178A
:1065D00039074A075B0708F0F6CEC5010E94C043A1
:1065E000F80184819581A681B7810196A11DB11D15
:1065F00084839583A683B7830E94336BF801FE964C
:106600006083718382839383C40102C080E090E041
:1066100026960FB6F894DEBF0FBECDBFDF91CF91A7
:106620001F910F91FF90EF90DF90CF90BF90AF90B0
:106630009F908F907F906F905F904F903F902F90A2
:106640000895CF93DF93FC0101900020E9F79F01AB
:10665000281B390B285F3F4F2138310570F5EC01BD
:106660000E943C63882349F18091AC099091AD0967
:10667000019611F481E090E09093AD098093AC090C
:106680008091AC099091AD099093310980933209C2
:1066900047E050E06CE279E0CE010E94B362FC0179
:1066A000EA5DF64F1682AC01445051096CE279E084
:1066B00082E8DF91CF910C94D36280E0DF91CF919B
:1066C0000895CF92DF92EF92FF920F931F93CF9393
:1066D000DF936C018B017B0182E0E80EF11CC0E0CE
:1066E000D0E0C6018C0F9D1F0E94F081F7018193BD
:1066F0007F012196C430D105A1F7F8019281992339
:1067000019F081E09F3F09F480E090E0DF91CF91A4
:106710001F910F91FF90EF90DF90CF900895EF922F
:10672000FF920F931F93CF93DF937C018B010E5F3A
:106730001F4FC0E0D0E0F80161918F01C7018C0FBD
:106740009D1F0E94F8812196C430D105A1F7DF91E9
:10675000CF911F910F91FF90EF900895FC01DC0104
:106760008D918111FDCF40E050E020E030E08AE0E3
:106770009191992301F1243031055CF59E3271F439
:106780004F3F510509F02CF5DB01A20FB31F129604
:106790004C932F5F3F4F40E050E0EACF849FD00101
:1067A000859FB00D1124492F990F550B4053510966
:1067B0004A0F5B1FDDCF4F3F510509F054F42430E1
:1067C00031053CF4FB01E20FF31F428381E090E0CE
:1067D000089580E090E008954F925F926F927F92CB
:1067E0008F929F92AF92BF92CF92DF92EF92FF92E1
:1067F0000F931F93CF93DF93CDB7DEB763970FB699
:10680000F894DEBF0FBECDBF7C015B013A01FB01F6
:1068100020E080E090E06AE03191332309F140ED1F
:10682000430F4A3080F4689FA001699F500D1124E6
:10683000CA01C097830F911D37FD9A958F3F91052F
:1068400059F350F313C03E3289F4233079F0D30169
:10685000A20FB11D12968C932F5F80E090E0DCCFE9
:10686000233021F4F301858381E021C0F7014281C7
:1068700053816481758180910E0990910F09A091D7
:106880001009B0911109481759076A077B0709F4E5
:106890009BC10E94336B8701085F1F4F6F70772782
:1068A0007C5FC8010E94CC45813019F080E090E007
:1068B000FEC18AE193E09A838983F7018281938103
:1068C000A481B5818B839C83AD83BE8345E350E077
:1068D000BE016F5F7F4FC8010E94CC46892B19F41F
:1068E000C12CD12C6CC10E94336BF7017783668376
:1068F0007627672776277A83698342E050E0BE01D6
:106900006F5F7F4FC8010E94214281E090E09E8727
:106910008D8742E050E0BE01635F7F4FC8010E9457
:10692000214280E091E09E878D8742E050E0BE01E9
:10693000635F7F4FC8010E9421421E861D8642E090
:1069400050E0BE01635F7F4FC8010E94214242E0D8
:1069500050E0BE01635F7F4FC8010E94214242E0C8
:1069600050E0BE01635F7F4FC8010E942142450194
:10697000F5018081882301F164015601F6018191BE
:106980002F01882321F08E3211F06201F6CFC81852
:10699000D9081C141D0474F4CF8641E050E0BE01F8
:1069A000615F7F4FC8010E942142A601B401C80166
:1069B0000E9421424201DCCF1F8641E050E0BE012F
:1069C000615F7F4FC8010E942142C12CDD24D39416
:1069D000DE86CD8642E050E0BE01635F7F4FC80196
:1069E0000E942142DE86CD8642E050E0BE01635F18
:1069F0007F4FC8010E942142C8010E94F945892B9E
:106A000009F46ECFE3E0AE2EB12C230122E0420E5A
:106A1000511C0E94336B3B014C01C8010E9453453D
:106A200018161906BCF00E94336BDC01CB018619E5
:106A30009709A809B909813A9F40A105B105E8F471
:106A4000A8950E94292761E070E080E090E00E9414
:106A5000F96AE3CFF7014281538164817581808DAA
:106A6000918DA28DB38D481759076A077B0749F4AA
:106A7000848D958DC59729F409C0CC24CA94DC2C4B
:106A800092C05EEFC52EDD24DA948DC0F70181A19E
:106A900092A10C970CF4A0C04CE050E0BE016F5FD7
:106AA0007F4FC8010E940B458B819C8198278927C5
:106AB00098279A8B898B29813A813227232732277D
:106AC000F701468157812417350709F080C097FFE9
:106AD0007EC08F709270892B09F0E4C06F8078843B
:106AE0007624672476246114710409F4D6C0C12C7D
:106AF000D12C8D819E81982789279827C816D90681
:106B000008F46FC0812C912C41E050E0BE016D5E15
:106B10007F4FC8010E940B458B89982F907C09F00C
:106B200092C0811186C042E050E0BE01615F7F4F9C
:106B3000C8010E940B4542E050E0BE01635F7F4FF9
:106B4000C8010E940B45C8010E942A45C8010E9445
:106B50002A45C8010E942A45C8010E942A4542E0F0
:106B600050E0BE016F5E7F4FC8010E940B458F85CC
:106B700098898115914009F06EC0CD84DE84DC24B3
:106B8000CD24DC2481E0C816D10409F064C08989D1
:106B90009A898115944009F07BC044E050E0B2012D
:106BA000C8010E940B45A8950E94292781E0A81AD8
:106BB000B10829F0FFEFCF16DF0609F42ACFC8018C
:106BC0000E94C043C60173C08EEF9FEF70C04CEFB0
:106BD000C42EDD24DA94E7CF9DEFC92EDD24DA94AC
:106BE000E2CF41E050E0BE01635F7F4FC8010E94E9
:106BF0000B458D85882351F08D859FEF980F9D87DC
:106C0000882321F0C8010E942A45F6CF8D85811185
:106C1000E8CFC8010E942A45C8010E942A45C80140
:106C20000E942A45C8010E942A45FFEFCF1ADF0AB9
:106C300060CF8B899FEF980F9B8B882341F0C80111
:106C40000E942A45F6CFC8010E942A451B8A8B89DB
:106C500081115ACF68CFC12CD12C89899A89982764
:106C600089279827C816D90638F4C8010E942A45F2
:106C7000FFEFCF1ADF0AF1CF2FEF821A920A6814C2
:106C8000790409F041CF26EFC22EDD24DA948BCFB0
:106C900077EFC72EDD24DA9486CF3AEFC32EDD24BA
:106CA000DA9481CF8BEFC82EDD24DA947CCF639603
:106CB0000FB6F894DEBF0FBECDBFDF91CF911F910D
:106CC0000F91FF90EF90DF90CF90BF90AF909F908B
:106CD0008F907F906F905F904F9008951F93CF9308
:106CE000DF93282F30E0F901E654F44F8491F90145
:106CF000E65EF34FD491F901E05AF34FC491CC23EF
:106D0000C1F0162F81110E94676AEC2FF0E0EE0FA0
:106D1000FF1FE056F44FA591B4919FB7F89411115D
:106D200004C08C91D095D82302C0EC91DE2BDC936B
:106D30009FBFDF91CF911F9108951F93CF93DF9352
:106D40001F921F92CDB7DEB76CE271E080E090E059
:106D50000E94F96A1FB7F8948091D007811127C06B
:106D6000E5E9FCE08491EFE4FCE09491E82FF0E0A9
:106D7000EE0FFF1FE050F44FA591B491EC91E92381
:106D800021F461E085E30E946E3661E085E30E94B4
:106D9000BD6A8CB580618CBD8CB580648CBD61E0B2
:106DA00084E30E94BD6A61E083E30E94BD6A809132
:106DB000D0078F5F8093D0071FBF249ACE01019622
:106DC0000E94765589819A810E94B63C67E080E0F6
:106DD00090E00E94413065E58BE190E00E944130F7
:106DE00065E58AE190E00E9441300E94B53C80E078
:106DF00090E49093740B8093730B80E090E69093F3
:106E00007C0B80937B0B80E098E49093760B8093CF
:106E1000750B80E098E690937E0B80937D0B80E06D
:106E200090E59093780B8093770B80E090E79093B8
:106E3000800B80937F0B80E098E590937A0B809392
:106E4000790B80E098E79093820B8093810B0F90F1
:106E50000F90DF91CF911F910895AF92BF92CF9283
:106E6000DF92EF92FF920F931F93CF93DF931F92C6
:106E70001F92CDB7DEB75C018B016A0179010E94D8
:106E80009D36CE0101960E94765589819A810E9495
:106E9000B63C46E050E06AEC77E089E090E00E9482
:106EA0001230C50102960E94A03CC60102960E94C3
:106EB000AE3CC70102960E94A73C0E94B53CF80177
:106EC00082819381A481B5818093140990931509DF
:106ED000A0931609B09317090F900F90DF91CF91EF
:106EE0001F910F91FF90EF90DF90CF90BF90AF90E8
:106EF0000895CF92DF92EF92FF92CF93DF93CDB7B9
:106F0000DEB768970FB6F894DEBF0FBECDBFFA01AB
:106F10002AE133E03A8329835FEF5B835C835D83FF
:106F20001E8238872F83C280D380E480F580C98693
:106F3000DA86EB86FC863E872D87FB0142815381F2
:106F4000648175814F87588B698B7A8B3C8B2B8B37
:106F5000FC0182819381A481B5818D8B9E8BAF8B47
:106F6000B88F9E012F5F3F4FAE01495F5F4FBE015B
:106F7000635F7F4FCE0143960E942D3768960FB610
:106F8000F894DEBF0FBECDBFDF91CF91FF90EF90A1
:106F9000DF90CF9008950F931F93CF93DF93CDB7DA
:106FA000DEB768970FB6F894DEBF0FBECDBFFB010A
:106FB000DC0112964D915D916D917C9115974D8BF1
:106FC0005E8B6F8B788F8AE193E09A83898321E0CF
:106FD000288F0D891E892F89388D0B831C832D8363
:106FE0003E8398878F8302811381248135810987AD
:106FF0001A872B873C879E878D874F87588B698B95
:107000007A8BAE014F5F5F4FBE01695F7F4FCE014C
:107010000D960E94793768960FB6F894DEBF0FBEC2
:10702000CDBFDF91CF911F910F910895CF93DF9343
:10703000CDB7DEB762970FB6F894DEBF0FBECDBFF7
:10704000FC0182819381A481B5818F87988BA98B64
:10705000BA8B2AE133E03A83298341E04A8B4F859A
:10706000588969897A894B835C836D837E833887ED
:107070002F8389879A87AB87BC87BE016F5F7F4F5D
:10708000CE0107960E94CB3762960FB6F894DEBF0A
:107090000FBECDBFDF91CF9108950F931F93CF9374
:1070A000DF93EC010E94CF5D8C01CE010E94F25E65
:1070B000800F911FDF91CF911F910F910895FC01D7
:1070C00086819781009739F0662329F06150FC0191
:1070D00082819381F7CF08950F931F93CF93DF930E
:1070E0008B01FC01C681D781209759F0B8018881B6
:1070F00099810E94C586892B21F00A80DB81C02DF1
:10710000F3CFCE01DF91CF911F910F910895DC0154
:107110001696ED91FC91179761157105A1F03097C6
:1071200029F417967C936E93169708958281938124
:10713000009711F0FC01FACF73836283DB0115968F
:10714000FC93EE9314970895CF92DF92EF92FF9203
:107150000F931F93CF93DF938C017B016A010E94F1
:10716000F22EEC01892B09F182E08887A601DD0C63
:10717000660B770B49875A876B877C878881998153
:10718000009711F00E943F78C7010E948C86998376
:107190008883BE01C801DF91CF911F910F91FF90AD
:1071A000EF90DF90CF900C948738DF91CF911F91B3
:1071B0000F91FF90EF90DF90CF900895CF92DF92E4
:1071C000EF92FF921F93CF93DF93EC016A017B0153
:1071D000122FE889F98982E080834115514E6105BB
:1071E0007105B1F060E079E08DE390E0A7019601D0
:1071F0000E941682DA01C9010197A109B109B69569
:10720000A795979587959C01211580E13807A8F0EF
:10721000E889F989108260E874E88EE190E0A701BE
:1072200096010E941682DA01C9010197A109B109EC
:10723000B695A795979587959C01EC85FD8530833C
:10724000EE85FF852083188EEC89FD891083EA89FD
:10725000FB89808180618083EA89FB8980818860E5
:107260008083EA89FB89808180688083EA89FB8941
:1072700080818F7D8083DF91CF911F91FF90EF9070
:10728000DF90CF9008958F929F92AF92BF92CF924E
:10729000DF92EF92FF920F931F93CF93DF93CDB7BF
:1072A000DEB7DA950FB6F894DEBF0FBECDBFC82E9D
:1072B0008091C9098983CA8221E0C216A0F074E0D6
:1072C0007C1518F487E1C8120EC08091CA0990910C
:1072D000CB099B838C838091CC099091CD099D83B0
:1072E0008E8386E001C082E08E010F5F1F4F90E128
:1072F0009C1528F0AFE0CA1630F49BEF01C09AEE5F
:107300009C0D923078F420914E0A90914F0AF8012A
:10731000E80FF11D908391E0980FF801E90FF11D3E
:107320008E5F2083BFE0CB1641F1BC1558F0E5E03D
:10733000CE16A1F0F6E0CF12B6C02091520A90917D
:10734000530A10C026E1C21609F48EC077E1C716B1
:1073500009F459C090E1C912A6C055C02091500A45
:107360009091510AF801E80FF11D908391E0980F78
:10737000F801E90FF11D8E5F95C02091500A309100
:10738000510AF801E80FF11D308342E0480F91E007
:10739000980FF801E90FF11D2083B9016770772775
:1073A000A3E036952795AA95E1F7672B19F091E0B0
:1073B000920F01C0922FB3E0B80FF801E40FF11D56
:1073C00090838C5F60E070E0A0E04FEF480F9A136D
:1073D00003C08B2F890F67C050E09B01359527951F
:1073E000400F511F220F331FF901EE5AF54FA0FD38
:1073F00002C0208101C02181FA012083AF5F6F5F4D
:107400007F4F8F5FE2CF2091500A3091510AF801EF
:10741000E80FF11D308391E0980FF801E90FF11D9D
:10742000208392E0980FF801E90FF11D8D5F922FF4
:10743000990F908390E03327E92FF0E0E217F307EC
:1074400094F5EE0FFF1FEE5AF54F50814181F80180
:10745000E80FF11D408341E0480FF801E40FF11DF2
:107460008E5F50839F5FE8CF9091520A2091530A1C
:10747000F801E80FF11D208321E0280FF801E20F49
:10748000F11D90832091540A9091550A32E0380FF3
:10749000F801E30FF11D908393E0980FF801E90FD5
:1074A000F11D8C5F20837801F8012FEF3FEFD02E84
:1074B0009E2F901B9817A0F49191292748E050E047
:1074C000B9017695679520FF06C09B0191E02927B9
:1074D00090EA392701C09B014150510989F7E8CF53
:1074E000F801E80FF11D2083B2E0BB2EB80E8F5FCC
:1074F000F801E80FF11D3083F801EB0DF11D10824A
:107500008091C7099091C809DC01ED91FC9102843A
:10751000F385E02D1995019699F7E091DD0AF09138
:10752000DE0A309709F019958091C7099091C80932
:107530002E2D2D192B1558F4F70161917F01DC01D7
:10754000ED91FC910190F081E02D1995EDCFDC01DA
:10755000ED91FC910680F781E02D1995E091DF0A0D
:10756000F091E00A309709F019950E94336B4B01B6
:107570005C01A8E0EA2EF12CD12C8091C7099091F2
:10758000C809DC01ED91FC910084F185E02D19958D
:10759000892BC1F08091C7099091C809DC01ED9158
:1075A000FC910284F385E02D19959091C909891702
:1075B00011F0FF2099F1F801EF0DF11D8083EA949D
:1075C000F39407C0E091DB0AF091DC0A309709F0F0
:1075D0001995B5E0FB1222C0EA818E2F8F7790E0DB
:1075E0008C159D0509F0A2C0E7FF04C08B8188239C
:1075F00081F181C08E2F90E0FC013197E731F105D8
:1076000068F48827EF53FF4F8F4F0C948D82F3E07F
:10761000EF2E04C0EB8002C0E5E0EE2E0E94336B3B
:10762000DC01CB0188199909AA09BB09813D974062
:10763000A105B10538F480E0EE2031F0882309F48B
:107640009CCF59C082EEF8CF811155C0F4E0FF15F0
:10765000C0F58FEF9FEF60E0EF2DF0E09F0122502B
:107660003109462F50E0D80142175307BCF4A40F4C
:10767000B51F4C91842748E050E0DC01B695A795F2
:1076800080FF06C0CD0171E0872770EA972701C00F
:10769000CD014150510989F76F5FE3CFA20FB31FAE
:1076A0002C9130E0AC0155274217530709F040C038
:1076B000892F9927EC0FFD1F208130E08217930757
:1076C000B9F58A818530B0F58330B0F5813090F01E
:1076D0005B81652F70E0759567952091DA0A40E02F
:1076E000842F90E0861797070CF452C02093DA0A93
:1076F00050FD6CC080E01092D40A1092D60A10920D
:10770000D50A1092D90AD3950FB6F894DEBF0FBEF2
:10771000CDBFDF91CF911F910F91FF90EF90DF9040
:10772000CF90BF90AF909F908F90089581EEE3CF60
:1077300083EEE1CF8731F1F66B8170E07595679547
:107740002091DA0A40E0842F90E0861797071CF01A
:107750002093DA0ACFCF4034C0F49C012E5F3F4F14
:10776000220F331F880F991FFC01E953F64FDE01EA
:10777000A20FB31F8C9190E0982F8827D801A20FF9
:10778000B31F2C91822B90878783242F4F5FDBCFF1
:107790004034C8F4880F991FFC01E953F64FA5E067
:1077A000B0E0AC0FBD1FA80FB91F2C9130E0322FF5
:1077B0002227A4E0B0E0AC0FBD1FA80FB91F8C9129
:1077C000282B30872783242F4F5F8ACF403468F4DB
:1077D000880F991FFC01E953F64FDE01A80FB91F6E
:1077E00014968C9190E09087878381E0840F80933A
:1077F000DA0A80CFDC011696ED91FC91179780E0B4
:10780000309729F08F5F0280F381E02DF9CF089542
:10781000CF93DF931F92CDB7DEB76983DC01ED9183
:10782000FC910280F381E02D41E050E0BE016F5FEA
:107830007F4F19950F90DF91CF910895DC01ED9165
:10784000FC91068CF78DE02D199591E0892708951C
:10785000862F089581E086270895CF93DF931F92A6
:10786000CDB7DEB789832091500B3981E091510B60
:10787000F091520B822F90E080959095F8940080C3
:10788000082200824BE000C05DE000005A95E9F755
:10789000008008220894379508F4022A00824A954D
:1078A00099F778940F90DF91CF9108950F931F93DC
:1078B000CF93DF931F92CDB7DEB78C01DC01ED9142
:1078C000FC910084F185E02D1995892B51F0BE01C2
:1078D0006F5F7F4FF80184850E943B44898190E06F
:1078E00002C08FEF9FEF0F90DF91CF911F910F910B
:1078F0000895FC0184850C948C44CF93DF931F92F0
:10790000CDB7DEB741E050E0BE016F5F7F4FFC01B5
:1079100084850E948C44181619061CF4898190E015
:1079200002C08FEF9FEF0F90DF91CF910895FC0180
:107930008485843011F00C94924280E090E00895A8
:1079400044E050E0BC018FE090E00C94123044E041
:1079500050E0BC0185E090E00C94123044E050E02F
:10796000BC0181E090E00C94123008958CBD9DBD67
:1079700008956F927F928F929F92AF92BF92CF9213
:10798000DF92EF92FF921F93CF93DF931F921F928C
:10799000CDB7DEB75C013B016A01FC0114851430F0
:1079A00041F481E090E0F5019383828380E090E0F0
:1079B0005BC07A014130584018F0E12C88E0F82E85
:1079C000CE0101960E94765589819A810E94B63C2B
:1079D000812F0E94515A4C0163E070E0812F0E9478
:1079E0001D44873111F08C3121F48E149F0440F333
:1079F00002C0E12CF12CCE0101960E9476558981BE
:107A00009A810E94B63C9701A30160E070E0812F4B
:107A10000E94EC5960E270E0812F0E94665562E09E
:107A200070E0812F0E941D4484FD14C063E070E06B
:107A3000812F0E941D44811104C0812F0E94514357
:107A4000B0CFCE0101960E94765589819A810E941D
:107A5000B63CE5CF40E162E070E0812F0E944743F1
:107A6000EF2809F49ECFC6010F900F90DF91CF91C0
:107A70001F91FF90EF90DF90CF90BF90AF909F90BD
:107A80008F907F906F9008958F929F92AF92BF9248
:107A9000DF92EF92FF920F931F93CF93DF931F928A
:107AA0001F92CDB7DEB7FC012485243009F083C0D6
:107AB0005A018B017C01D12C8D2D0E94AD45811185
:107AC00003C0F701D48607C08B7F8831D1F3D394EC
:107AD000F4E0DF12F1CFF7018485843009F46BC044
:107AE00020910302309104022F5F3F4F11F420E0F8
:107AF00030EC309304022093030240910302509132
:107B0000040220E061E00E947443F80182818F3F0B
:107B100051F483818F3F99F484818F3F81F4858173
:107B20008F3F69F445C081110AC0F801838181113A
:107B300006C08481811103C085818823C9F1A11405
:107B4000B104B1F1F701D484CE0101960E947655BB
:107B500089819A810E94B63CB8016E5F7F4F8D2D5E
:107B60000E945446B5018D2D0E94434664E070E0AA
:107B70008D2D0E9466550E94336B4B015C01F4E928
:107B80008F0EF1E19F1EA11CB11CC7010E947B5505
:107B9000873149F161E070E080E090E00E94F96A8D
:107BA000A8950E942927C7010E947B55811106C014
:107BB00084E0F701848780E090E01DC00E94336B71
:107BC00086169706A806B90600F7F70184850E9475
:107BD000514384E0F701848761EB7DE08FE698E014
:107BE0000E944D38E8CF66EA7DE08FE698E00E947B
:107BF0004D3881E090E00F900F90DF91CF911F9171
:107C00000F91FF90EF90DF90BF90AF909F908F907B
:107C1000089578941F920F920FB60F9211240BB60D
:107C20000F92CF92DF92EF92FF920F931F932F93B9
:107C30003F934F935F936F937F938F939F93AF93F4
:107C4000BF93CF93DF93EF93FF93809170008E7F6C
:107C5000809370000FE310E08BE1E82EF12C9BE2A3
:107C6000C92ED12CC091530BD091540B2097F9F40D
:107C70000332110508F43BC003521109E091510B86
:107C8000F091520B90812091500B822F8095982378
:107C900090839BE0D7011197F1F79150D9F780813C
:107CA000822B8083C6010197F1F780E00DC00B3075
:107CB0001105E8F00B501109E091550BF091560BAE
:107CC000EC0FFD1F319780810E942D3C2196D093AF
:107CD000540BC093530B80910102909102028C17B8
:107CE0009D0708F0BFCF1092540B1092530B809158
:107CF0007000816080937000FF91EF91DF91CF91D0
:107D0000BF91AF919F918F917F916F915F914F91B3
:107D10003F912F911F910F91FF90EF90DF90CF90A7
:107D20000F900BBE0F900FBE0F901F90189581E023
:107D300080934F0B80910002282F30E0F901E05A28
:107D4000F34FE491F0E0EE0FFF1FE056F44F459142
:107D500054915093520B4093510BF901E65EF34F4F
:107D6000E491E093500B61E00E94BD6A83E0809350
:107D7000B100E0E7F0E08081816080830895CF93D7
:107D8000DF931816190644F0809170008E7F80935F
:107D9000700010924F0B19C0EC018091550B90911F
:107DA000560B0E943F78CE01C130D24014F080E0E3
:107DB00092E090930202809301020E94A777909331
:107DC000560B8093550B892B29F4109202021092C6
:107DD000010208C080914F0B811104C0DF91CF9147
:107DE0000C94973EDF91CF910895FF920F931F93CC
:107DF000CF93DF938C01F62E80914F0B811102C03F
:107E00000E94973EE8012197C11582E0D80798F4B7
:107E100080910102909102028017910718F4C80125
:107E20000E94BF3E8091550B9091560B009719F020
:107E3000C80FD91FF882DF91CF911F910F91FF904A
:107E40000895DC0180E0615040F09D91E82FE92722
:107E5000F0E0EA55F34F8491F6CF0895AF92BF92C8
:107E6000CF92DF92EF92FF921F93CF93DF93EC01BB
:107E70000E94336B6B017C0128EEC20E23E0D21E00
:107E8000E11CF11C8BE4A82EB12C0E94336B6C1505
:107E90007D058E059F0598F460EFCE010E947C243D
:107EA000CE010E942024182F80FF11C0EF85F88991
:107EB000309709F01995C5010197F1F7E6CF81E0F8
:107EC0008A8368EC74E08FE698E00E947454812FF6
:107ED000DF91CF911F91FF90EF90DF90CF90BF90F7
:107EE000AF9008950F931F93CF93DF93EC01162F5C
:107EF000042F0E942E3F002319F0CE010E949E24E1
:107F0000CE010E94702465EA8AE199E00E94E7238D
:107F1000612F8AE199E00E94E723CE01DF91CF91A2
:107F20001F910F910C946D24EF92FF920F931F936A
:107F3000CF93DF938C017B0140E065E50E94723FA7
:107F4000E70188E0E80EF11C699140E0C8010E9459
:107F5000723FCE15DF05C1F7DF91CF911F910F91D1
:107F6000FF90EF9008951F93CF93DF93EC01162FAE
:107F70000E942E3FCE010E94702462ED8AE199E0BA
:107F80000E94E723612F70E06095709584E0660F92
:107F9000771F8A95E1F7612B8AE199E00E94E72338
:107FA000CE010E946D24CE010E942024181711F0EA
:107FB00084E08A83DF91CF911F9108951F93CF931F
:107FC000DF93EC010E942E3FCE010E94932460E0DB
:107FD000CE010E94B33FCE010E942E3FCE010E94EF
:107FE000702464EB8AE199E00E94E723CE010E94AD
:107FF0006D24CE010E942E3F182F82FF02C082E026
:108000008A838881882341F0CE010E949324682FBF
:108010006160CE010E94B33F11FB882780F9DF9198
:10802000CF911F910895CF92DF92EF92FF920F931D
:108030001F93CF93DF937C01EB018A01FC018581C3
:1080400096810E94DE3F8823C9F1BE01F701858138
:1080500096810E94943F40E06EEBF7018581968106
:108060000E94723FE8016801F9E0CF0ED11CF701D0
:1080700005811681C8010E942E3FC8010E9470240C
:1080800066E98AE199E00E94E723C8010E946D2415
:10809000C8010E942E3F61EEC8010E947C24C801E5
:1080A0000E9420248993CC16DD0609F7F70185810B
:1080B00096810E94DE3F91E0813009F090E0892FA7
:1080C000DF91CF911F910F91FF90EF90DF90CF90B4
:1080D0000895CF93DF93EA010E941340882339F07B
:1080E00068E0CE010E94213F91E02885281390E0AE
:1080F000892FDF91CF910895CF93DF93CDB7DEB76E
:1081000029970FB6F894DEBF0FBECDBFAE014F5F0B
:108110005F4F0E946940882389F08D818F3361F021
:1081200020F48F3159F489E00CC08F3519F08F3766
:1081300039F004C08BE005C08AE003C080E001C0D4
:108140008CE029960FB6F894DEBF0FBECDBFDF914D
:10815000CF9108956F927F928F929F92AF92BF922C
:10816000CF92DF92EF92FF920F931F93CF93DF9303
:10817000FC01248521119EC0872E762EEC010E94E1
:10818000DE3F811108C063ED74E08FE698E00E9445
:1081900074548FEF90C0CE010E942E3F40E060EFFC
:1081A000CE010E94723FC12CD12C66246A94EE2429
:1081B000E394F12C0C2D06950695069510E08C2D78
:1081C0008770570101C0AA0C8A95EAF78B85082EA3
:1081D000000C990BC816D90634F4FE01E00FF11F0C
:1081E00093809A2006C099249394C816D90609F062
:1081F000912CCE010E942E3FCE010E94702468E790
:108200008AE199E00E94E723911002C060E001C07A
:1082100060E88AE199E00E94E723CE010E946D2484
:10822000CE010E942E3F282F2074982F907885FF32
:1082300011C02223A9F042E050E0682F8FE698E0B9
:108240000E94A05E6FED74E08FE698E00E94745487
:108250008EEF31C0211104C0911104C06C2C08C0F4
:10826000992331F0FE01E00FF11F83818A2907C0B5
:10827000FE01E00FF11F8A2D80959381892383836E
:10828000FFEFCF1ADF0A80E4C816D10409F092CFBD
:108290006B86EFEF6E1202C081E08C87DE011396D1
:1082A000E72DF82D2B968D918193CA17DB07D9F70F
:1082B00081E001C080E0DF91CF911F910F91FF908D
:1082C000EF90DF90CF90BF90AF909F908F907F9076
:1082D0006F900895AF92BF92CF92DF92EF92FF928C
:1082E0000F931F93CF93DF93CDB7DEB7AF970FB642
:1082F000F894DEBF0FBECDBF7C015B016A010AE1CD
:1083000013E01A8309831B821C821D821E82CE0108
:1083100009960E94C2421BA70AA71CA61DA61EA65C
:108320001FA68091140990911509A0911609B0918A
:1083300017098EA39FA3A8A7B9A78B839C83AD839E
:10834000BE8318861F82AE01465D5F4FB501CE0128
:1083500001960E94EC3381309105B1F4D701ED9183
:10836000FC910684F785E02D1DA30CA38CA59DA58B
:10837000AEA5BFA58EA39FA3A8A7B9A7A601BE01BE
:108380006C5D7F4FC7011995AF960FB6F894DEBFAD
:108390000FBECDBFDF91CF911F910F91FF90EF9056
:1083A000DF90CF90BF90AF9008950895CF93DF9363
:1083B0001F92CDB7DEB76983DC01ED91FC9102809D
:1083C000F381E02D41E050E0BE016F5F7F4F1995D2
:1083D0000F90DF91CF910895FC01818D928D0895CA
:1083E000FC018489958908952AE133E0FC013183F9
:1083F0002083FB014089518962897389FC01428392
:108400005383648375830895DC01ED91FC91048CA2
:10841000F58DE02D199480E00895FC019485FB0111
:108420008485981303C081E0943009F480E00895B6
:1084300021E0FC018485843009F420E0822F089536
:1084400008958F929F92AF92BF92DF92EF92FF9228
:108450000F931F93CF93DF931F921F92CDB7DEB779
:108460007C014B018A01FC01A688B788D08CCE0123
:1084700001960E94765589819A810E94B63C8D2D85
:108480000E94515A8017910720F48D2D0E94515A55
:108490008C019801A401B5018D2D0E94EC590E9418
:1084A000B53CF70186899789800F911F978B868B42
:1084B000C8010F900F90DF91CF911F910F91FF9006
:1084C000EF90DF90BF90AF909F908F900895CF93E3
:1084D000DF93FC0124852430D1F0EC010E947B5510
:1084E000843181F0882371F0883161F08C3161F43E
:1084F000E881F9810084F185E02DCE01199521E014
:10850000892B19F420E001C021E0822F01C080E016
:10851000DF91CF9108958EBD00000DB407FEFDCF11
:108520008EB50895DF92EF92FF920F931F93CF9332
:10853000DF931F921F92CDB7DEB7D82ECE010196E2
:108540000E94765589819A810E94B63CE12CF12CDB
:108550008D2D0E945C308C01892B21F08D2D0E9485
:108560005C307C010E151F0599F70E94B53CC801CF
:108570000F900F90DF91CF911F910F91FF90EF908F
:10858000DF900895FC011382128288EE93E0A0E050
:10859000B0E084839583A683B7838CE293E09183D4
:1085A00080838AE193E097878687108A118A128AEE
:1085B000138A84E0808F0895AF92BF92CF92DF92AA
:1085C000EF92FF920F931F93CF93DF93CDB7DEB758
:1085D000AF970FB6F894DEBF0FBECDBF7C015B0135
:1085E0006A010AE113E01A8309831B821C821D823F
:1085F0001E82CE0109960E94C2421BA70AA71CA692
:108600001DA61EA61FA68091140990911509A09180
:108610001609B09117098EA39FA3A8A7B9A78B83AA
:108620009C83AD83BE8318861F82AE01465D5F4F7B
:10863000B501CE0101960E94EC3381309105B1F471
:10864000D701ED91FC910488F589E02D1DA30CA3C1
:108650008CA59DA5AEA5BFA58EA39FA3A8A7B9A7CE
:10866000A601BE016C5D7F4FC7011995AF960FB68D
:10867000F894DEBF0FBECDBFDF91CF911F910F9158
:10868000FF90EF90DF90CF90BF90AF9008959B0147
:1086900090E00496982F8827642F820F931F0C94E4
:1086A00041301F93CF93DF931F921F92CDB7DEB758
:1086B000182FCE0101960E94765589819A810E94D9
:1086C000B63C60E170E0812F0E9466554FEF62E09A
:1086D00070E0812F0E9447430E94B53C0F900F909D
:1086E000DF91CF911F910895DF92EF92FF920F9348
:1086F0001F93CF93DF931F921F92CDB7DEB7182F32
:10870000D62E7A01022F0E945143CE0101960E947B
:10871000765589819A810E94B63C4D2D402B60E0B0
:1087200070E0812F0E944743E114F10459F4E09076
:108730005F0BF090600B8FEFE81AF80AF092600B75
:10874000E0925F0B4F2D64E070E0812F0E94474361
:108750004E2D65E070E0812F0E94474361E070E09C
:10876000812F0E9466550E94B53C81E00F900F90CA
:10877000DF91CF911F910F91FF90EF90DF900895BF
:10878000CF93DF93FC01808D843029F0EF010E94AC
:10879000514384E0888FDF91CF910895CF92DF928B
:1087A000EF92FF920F931F93CF93DF931F921F922D
:1087B000CDB7DEB7FC01F484F4E0FF1699F18C012B
:1087C000CE0101960E94765589819A810E94B63C1D
:1087D00068E070E08F2D0E9466550E94B53C0E94B3
:1087E000336B6B017C01C8010E947B558823B9F073
:1087F00062E370E080E090E00E94F96A0E94336BCF
:10880000DC01CB018C199D09AE09BF09883E93405C
:10881000A105B10540F3F80184850E94514384E02D
:10882000F80184870F900F90DF91CF911F910F91E6
:10883000FF90EF90DF90CF900895CF93DF9390E07B
:108840000496982F8827EC01C60FD71F0E94E02FAF
:108850008FE00E948B428D2F0E948B428C2F0E94B2
:108860008B4280E00E948B42C82F0E94DE2F8C2F0B
:10887000DF91CF910895CF92DF92FF920F931F93D4
:10888000CF93DF931F921F92CDB7DEB7F82E6B0107
:10889000CE0101960E94765589819A810E94B63C4C
:1088A00068E270E08F2D0E941D44082F10E069E2FD
:1088B00070E08F2D0E941D44702F6627682B21E0E9
:1088C00030E0A6018F2D0E94A4590E94B53C81E0A2
:1088D00090E00F900F90DF91CF911F910F91FF903B
:1088E000DF90CF900895CF93DF931F92CDB7DEB77F
:1088F000FC01218D328D232B49F0BE016F5F7F4F2C
:10890000808D0E943B44898190E002C08FEF9FEFF1
:108910000F90DF91CF9108958F929F92BF92CF9247
:10892000DF92EF92FF920F931F93CF93DF931F92EB
:108930001F92CDB7DEB7B82E6B017A01CE0101963A
:108940000E94765589819A810E94B63C812C912C97
:108950008B2D0E945C308C01892B21F08B2D0E9485
:108960005C304C010815190599F70115110599F4AA
:1089700063E070E08B2D0E941D448431D9F188237F
:10898000C9F101E010E08C3111F400E010E0119524
:10899000019511092FC0E016F1060CF4870110169D
:1089A000110644F568E270E08B2D0E941D44E82E0C
:1089B000F12C69E270E08B2D0E941D44FE2CEE2408
:1089C000E82A9801A601B7018B2D0E94A459E00E58
:1089D000F11E4F2D68E270E08B2D0E9447434E2D13
:1089E00069E270E08B2D0E94474360E470E08B2DBC
:1089F0000E9466550E94B53CC8010F900F90DF9110
:108A0000CF911F910F91FF90EF90DF90CF90BF908B
:108A10009F908F900895CF93DF93FC01218D328D2D
:108A20002115310519F48FEF9FEF11C0EC014217AA
:108A3000530708F0A901888D0E948C441816190666
:108A400094F7298D3A8D281B390B3A8F298FDF91A6
:108A5000CF9108950F931F93CF93DF931F92CDB7BC
:108A6000DEB7FC01218D328D232B61F08C0141E0BA
:108A700050E0BE016F5F7F4F808D0E948C441816BE
:108A800019061CF08FEF9FEF08C0F801818D928DC1
:108A90000197928F818F898190E00F90DF91CF9124
:108AA0001F910F9108950F931F93CF93DF93CDB72D
:108AB000DEB728970FB6F894DEBF0FBECDBF8C018E
:108AC000D80159968D919C915A97892B41F0ED913F
:108AD000FC910284F385E02DC8011995F1CFF801CE
:108AE000808D0E9492421816190654F548E050E015
:108AF000BE016F5F7F4FD80158968C910E948C44C5
:108B000018161906FCF4D801509684E0FE0131963F
:108B100001900D928A95E1F78D8190E0982F88273A
:108B20002E81820F911DF801958B848B8F8190E0AF
:108B3000982F88272885820F911D928F818F02C0E0
:108B400080E090E028960FB6F894DEBF0FBECDBF50
:108B5000DF91CF911F910F9108951F93CF93DF93D2
:108B60001F921F92CDB7DEB7182FCE0101960E943B
:108B7000765589819A810E94B63C63E070E0812F2E
:108B80000E941D44182F0E94B53C812F0F900F901A
:108B9000DF91CF911F910895EF92FF921F93CF9392
:108BA000DF93FC01208D243011F080E01CC07B019C
:108BB000EC0110E0812F0E94AD45811102C0188F99
:108BC00005C08831E1F31F5F1430A1F7888D843030
:108BD00061F3FD86EC861A8E198E20E0A70162E013
:108BE0000E94744381E0DF91CF911F91FF90EF903D
:108BF00008951F93CF93DF931F921F92CDB7DEB7D7
:108C0000FC01108DCE0101960E94765589819A81D2
:108C10000E94B63C60E270E0812F0E94665562E0DF
:108C200070E0812F0E941D4484FD1DC062E070E051
:108C3000812F0E941D4483FF0BC048E162E070E079
:108C4000812F0E9447430E94B53C80E090E015C010
:108C50000E94B53CCE0101960E94765589819A8189
:108C60000E94B63CDCCF40E162E070E0812F0E94C0
:108C700047430E94B53C81E090E00F900F90DF9158
:108C8000CF911F910895CF93DF93C82FD62F472FF1
:108C900060E170E00E9447434D2F61E170E08C2F4E
:108CA000DF91CF910C94474390E0982F882744E0C0
:108CB00050E0845F9B4F0C941230BF92CF92DF92B2
:108CC000EF92FF920F931F93CF93DF9300D000D0CA
:108CD000CDB7DEB7FC01208D243009F04CC06A010D
:108CE0007B018C01B12C63E070E08B2D0E941D4450
:108CF000811103C0F801B08E06C08831D9F3B39456
:108D0000F4E0BF12F0CFF801808D8430A1F196E03D
:108D1000E2E2F3E0DE01119601900D929A95E1F7FF
:108D2000F70193819F779C8394819D8395819E8396
:108D3000B7016E5F7F4F0E945446B601F801808DE7
:108D40000E944346F801808D90E0982F882746E0E6
:108D500050E0BE016F5F7F4F8A5F9B4F0E941230D1
:108D6000F801128E118E20E8A60162E0808D0E942B
:108D7000744381E001C080E026960FB6F894DEBF10
:108D80000FBECDBFDF91CF911F910F91FF90EF905C
:108D9000DF90CF90BF900895DF92EF92FF920F93F4
:108DA0001F93CF93DF931F921F92CDB7DEB7FB01C6
:108DB000DC0157961C921E9256972281211109C000
:108DC0002381211106C02481211103C02581222382
:108DD000F1F041155105D9F07A018F01FC01D08CD9
:108DE000CE0101960E94765589819A810E94B63CF7
:108DF000B8016E5F7F4F8D2D0E945446B7018D2DB7
:108E00000E9443460E94B53C81E090E002C080E0B1
:108E100090E00F900F90DF91CF911F910F91FF90F5
:108E2000EF90DF9008950C94454E66E67FE08FE664
:108E300098E00C94CF5DCF93C1E068EE73E080E0E2
:108E400090E00E94F96A4AE050E06C2F8FE698E0CB
:108E50000E94A05ECF5FC43181F7CF9108950F9338
:108E60001F93CF93DF93CDB7DEB728970FB6F89453
:108E7000DEBF0FBECDBF0E94222A6FEB7DE08FE6E2
:108E800098E00E94CF5DCE0101960E943659CE0136
:108E900001960E94E0580AE113E01A8309831B82BD
:108EA0001C821D821E82CE0107960E9476558F81FC
:108EB00098850E94B63C44E050E0BE016D5F7F4F54
:108EC00081E090E00E94E22F0E94B53CCE01019625
:108ED0000E94E0581A8309831B821C821D821E8215
:108EE000CE0107960E9476558F8198850E94B63CE8
:108EF00044E050E0BE016D5F7F4F85E090E00E944E
:108F0000E22F0E94B53CCE0101960E94E05865EE2A
:108F10007DE08FE698E00E94CF5D28960FB6F8942A
:108F2000DEBF0FBECDBFDF91CF911F910F9108958E
:108F30005F926F927F928F929F92AF92BF92CF92E9
:108F4000DF92EF92FF920F931F93CF93DF93CDB7F2
:108F5000DEB761970FB6F894DEBF0FBECDBF80912C
:108F6000710B9091720B009709F451C469EE74E093
:108F70000E946C389093680B8093670B009709F4FC
:108F8000A9C00E94FA3B082F10E00115110509F451
:108F9000A1C0000F111F000F111F8091620B909153
:108FA000630B892B09F085C0C8010E94A7779093B5
:108FB000630B8093620B1092E00B1092DF0B109208
:108FC0006A0B1092690B1092DE0B1092E20B10925A
:108FD000E10B7801013022E012071CF0E12C72E075
:108FE000F72EC70101960E94A7779093E40B809318
:108FF000E30B9093DD0B8093DC0B8E0D9F1D909304
:10900000D70B8093D60B0E94336B6093D80B709371
:10901000D90B8093DA0B9093DB0B80E090E0E0912A
:10902000E30BF091E40BE80FF91F10820196E816AC
:10903000F906ACF782E090E09093E00B8093DF0BB1
:1090400080E98093C9001092C8001092CD0083E09F
:109050008093CC008EE08093CA00F0920702E092E9
:1090600006022091E30B3091E40B8091060290916F
:109070000702820F931F9093D70B8093D60B232B5D
:1090800009F4CEC26FE87FE08FE698E00E94CF5DE2
:109090004AE050E0B8018FE698E00E94995E8FE6C2
:1090A00098E00E94F25E83E290E29093D50B809369
:1090B000D40B61E870E18FE698E00E94CF5D4AE052
:1090C00050E0B8018FE698E00E94995E8FE698E044
:1090D0000E94F25E6FEE74E08091710B9091720BC2
:1090E0000E946C388C010097A1F10E94FA3B882302
:1090F00081F161E0C8010E945F38FC0101851285A1
:1091000090914F0B992359F0809170008E7F80933E
:10911000700010924F0B109202021092010283E035
:109120008093000291110E94973EC8010E94BF3EA9
:1091300065E670E18FE698E00E94CF5D4AE050E07E
:10914000B8018FE698E00E94995E8FE698E00E9451
:10915000F25E0091710B1091720B63EF74E0C80125
:109160000E946C3890936C0B80936B0B6AEF74E0E9
:10917000C8010E946C3890939F0580939E050097CC
:1091800009F49AC12091A005211196C1DC0116961F
:10919000ED90FC9017978091900590919105892B07
:1091A00009F0C7C068EE7FE08FE698E00E94CF5DCF
:1091B0008FE698E00E94F25E81E190E00E94A7773E
:1091C0008C0188E1F801818312821082108A17864F
:1091D0000E943455109391050093900583E190E02F
:1091E0000E94A777FC0185ED91E4928B818B168319
:1091F00005831482108289E0818311E01283138336
:10920000F0939905E093980580EA90E00E94A77793
:10921000909395058093940588E290E00E94A7774B
:1092200090938F0580938E050E9434558091900510
:10923000909191050E94702481E00E941854811140
:109240006FC065ED7FE08FE698E00E944D38C090DA
:109250009005D0909105C6010E94702440E060EF17
:10926000C6010E94723FC6010E946D24E0919005E4
:10927000F0919105108365EB7FE08FE698E00E9406
:109280004D3880919005909191050E94DE3F882392
:1092900031F069EA7FE08FE698E00E944D38009156
:1092A0009805109199050E94336B4B015C01F0E128
:1092B0008F0EF7E29F1EA11CB11CD8011596ED91EF
:1092C000FC9116978FEF83871486DF0113963B96E8
:1092D0001D92EA17FB07E1F7F801148277247394D3
:1092E000BE01665F7F4FD80115968D919C911697B0
:1092F0000E94AA40181644F40E94336B6815790541
:109300008A059B0508F493C189E798E69093930535
:1093100080939205E0919805F0919905128209C019
:109320006BE97FE08FE698E00E944D3880E090E0A6
:1093300002C081E090E0282F21702093A005892BA6
:1093400031F065E570E18FE698E00E94CF5D109204
:1093500097051092960501E010E0E114F10409F47C
:10936000ABC08091A005882309F4A6C0F7018085D1
:10937000863009F09BC0C080D180CE0101965C018F
:10938000460190E1890E911C3501D6018C910E9415
:10939000C826582EF60181810E94C826529460EF9B
:1093A00056228529D5018D935D01B2E0CB0ED11CEB
:1093B0008C149D0451F78091960590919705843106
:1093C00091050CF073C0880F991FE0918E05F09104
:1093D0008F05E80FF91F11830083A0919605B091C6
:1093E000970533E0AA0FBB1F3A95E1F780919405EA
:1093F00090919505A80FB91F88E0F30101900D9297
:109400008A95E1F7C0909605D090970560E170E1EC
:109410008FE698E00E94CF5D4AE050E0B6018FE60B
:1094200098E00E94995E69E070E18FE698E00E9402
:10943000CF5D809196059091970543E0880F991F25
:109440004A95E1F72091940530919505820F931F7D
:109450000E9408558FE698E00E94F25E60919605A2
:109460007091970553E0660F771F5A95E1F7809149
:10947000940590919505680F791FFB0180818832D2
:1094800061F480919805909199050E94865480918D
:109490009005909191050E949E248091960590914F
:1094A000970501969093970580939605D70112969C
:1094B000ED90FC90139751CFE090710BF090720BF0
:1094C0006DEF74E0C7010E946C388C019093EA0B39
:1094D0008093E90B63E075E0C7010E946C389093BC
:1094E00062068093610610929B0510929A05011501
:1094F000110529F1F801E680F78090E8C92E93E084
:10950000D92E0091E90B1091EA0B0115110571F0AC
:10951000E114F10459F0D70118968C918530A9F720
:10952000C7010E94FA3B823080F306C1D80116962B
:109530008D919C91179790939B0580939A0500912C
:10954000710B1091720B6CEE74E0C8010E946C38C4
:1095500090935E0680935D066AE075E0C8010E9404
:109560006C389093660B8093650B6FE370E18FE628
:1095700098E00E94CF5D67E370E18FE698E00E947B
:10958000CF5D81E02091E90B3091EA0B232B09F4A8
:1095900080E00E943A4E6EE270E18FE698E00E9411
:1095A000CF5D81E020915D0630915E06232B09F4AA
:1095B00080E00E943A4E65E270E18FE698E00E94FA
:1095C000CF5D81E020916B0B30916C0B232B09F464
:1095D00080E00E943A4E6EE170E18FE698E00E94D2
:1095E000CF5D81E02091650B3091660B232B09F450
:1095F00080E00E943A4E65E170E18FE698E00E94BB
:10960000CF5D81E020919E0530919F05232B09F4C9
:1096100080E00E943A4E8FE698E00E94F25EF7C02A
:1096200068E77FE08FE698E00E944D383CCD67E028
:10963000CE010A960E94213F9989891373C063EF76
:1096400073E08FE698E00E94F65EF8018081811158
:1096500038C0858196810E94DE3FBE01665F7F4FE4
:10966000D80115968D919C9116970E94943F40E0E9
:1096700064EBF801858196810E94723FD8011596AE
:10968000CD90DC901697C6010E942E3FC6010E9425
:10969000702467E88AE199E00E94E72360E88AE1A4
:1096A00099E00E94E723C6010E946D24C6010E9432
:1096B0002E3FD82EF801858196810E94DE3FD5FE8F
:1096C00038C0AE014F5F5F4FBE01665F7F4FC8017C
:1096D0000E941340D8011196DC908A85803109F4EC
:1096E00091C0BE01665F7F4FC8010E947C408D150E
:1096F00018F4F80181810BC08A85803111F48CE067
:1097000006C0BE01665F7F4FC8010E947C40D80141
:1097100011968C93119714968C9114978F5F1496D1
:109720008C93DECD69EF73E08FE698E00E94F65EE1
:10973000D7CDD8017C92C5CFDA82C982FC82EB8278
:10974000CE0101960E948221CE0101960E94B12095
:10975000882309F453C060E070E0CE0101960E94B6
:109760001A218C0160E0CE0101960E946F21A82E83
:10977000B12C8985853019F0863049F03FC0A1149D
:10978000B10429F462E0CE0101960E944821C8018B
:1097900017FF03C0919581959109982E092F882E66
:1097A00061E00E94BD6A11E0AA94AB2809F010E0C4
:1097B000612F882D0E946E3660E570E18FE698E09B
:1097C0000E94CF5D4AE050E0692D702F8FE698E04F
:1097D0000E94995E6EE470E18FE698E00E94CF5D92
:1097E000612F70E04AE050E08FE698E00E94995EB9
:1097F0006CE470E18FE698E00E94CF5DF701E280B3
:10980000F3807FCEBCE0BD1508F473CF78CF6196AE
:109810000FB6F894DEBF0FBECDBFDF91CF911F9181
:109820000F91FF90EF90DF90CF90BF90AF909F90FF
:109830008F907F906F905F900895CF92DF92EF921C
:10984000FF920F931F93CF93DF936C01EB0109906D
:109850000020E9F72197C61BD70BC032D10514F0C1
:10986000CFE1D0E08B01E12CF12CEC16FD0664F485
:10987000F80161918F01C7018C0D9D1D0E94F88137
:10988000FFEFEF1AFF0AF1CF60E0C6018C0F9D1FBA
:10989000DF91CF911F910F91FF90EF90DF90CF90CC
:1098A0000C94F881CF93DF931F92CDB7DEB7198266
:1098B000892B21F0FB016281738103C0BE016F5FC0
:1098C0007F4F86E390E00E941D4C6AE271E18FE6D3
:1098D00098E00E94CF5D0F90DF91CF910895CF93D4
:1098E000DF93C0E0D0E060E0CE010E94F8812196D5
:1098F000C11582E0D807B9F76AE171E18FE698E017
:10990000DF91CF910C94CF5D0F931F93CF93DF9393
:10991000EB018FEC97E09F938F938EEC97E09F93F2
:109920008F938DEC97E09F938F938CEC97E09F93B0
:109930008F938BEC97E09F938F938AEC97E09F93A4
:109940008F938FE095E09F938F938B818F938A8184
:109950008F930E9497872DB73EB7205F3F4F0FB67A
:10996000F8943EBF0FBE2DBF069794F40A80DB81AA
:10997000C02D6CE371E18FE698E00E94CF5DBE01DF
:109980008FE698E0DF91CF911F910F910C94F65ED6
:109990000E948D660AEC17E0C0E0D0E0F80161910A
:1099A0008F01CE010E94F8812196C630D105B1F712
:1099B0006EE471E18FE698E0DF91CF911F910F91F6
:1099C0000C94CF5D0F931F93CF93DF93CDB7DEB78A
:1099D0002C970FB6F894DEBF0FBECDBF8B012AE1E6
:1099E00033E03A8329831B821C821D821E823887C2
:1099F0002F8319861A861B861C8683309105B9F140
:109A000044F48130910509F454C0029709F443C02D
:109A100057C084309105B9F0059709F051C0BE01D7
:109A2000695F7F4FF801808591850E94AE33BE014A
:109A3000892B19F0695F7F4F02C06F5F7F4F82E112
:109A400090E00E948F33BE01695F7F4FF8018681ED
:109A500097810E94AE33BE01892B19F0695F7F4F59
:109A600002C06F5F7F4F8EE090E00E948F33BE0197
:109A7000695F7F4FF801848195810E94AE33BE01FA
:109A8000892B19F0695F7F4F02C06F5F7F4F8AE0BB
:109A900090E00E948F33BE01695F7F4FF8018281A1
:109AA00093810E94AE33BE01892B21F0695F7F4F05
:109AB00003C0BE016F5F7F4F86E090E00E948F334E
:109AC00063E171E18FE698E00E94CF5D2C960FB6BE
:109AD000F894DEBF0FBECDBFDF91CF911F910F91E4
:109AE0000895CF93DF93CDB7DEB72C970FB6F894D8
:109AF000DEBF0FBECDBF1C821B821E821D828FEF78
:109B00009FEF98878F8384E593E09A83898386E427
:109B100090E09A8789871C861B8669EF70E18FE643
:109B200098E00E94CF5D6091710B7091720BCE0135
:109B300001960E94FB2C6FEFCE0101960E94DC2B58
:109B400069EE70E18FE698E00E94CF5D2C960FB62B
:109B5000F894DEBF0FBECDBFDF91CF910895CF93B4
:109B6000DF93CDB7DEB769970FB6F894DEBF0FBEAF
:109B7000CDBF8FE290E09A838983FE01339687E11F
:109B8000DF011D928A95E9F764ED70E18FE698E0B8
:109B90000E94CF5DAE014E5F5F4F66E08AEC97E0BA
:109BA0000E94D9261E8664E275E0CE0101960E94CD
:109BB000D886BE016F5F7F4F8FE698E00E94F65E09
:109BC000CE0101960E9421331E866CE275E0CE0123
:109BD00001960E94D886BE016F5F7F4F8FE698E0A6
:109BE0000E94F65E66E375E0CE0101960E946A650A
:109BF00069960FB6F894DEBF0FBECDBFDF91CF914F
:109C00000895AF92BF92CF92DF92EF92FF920F939F
:109C10001F93CF93DF936C017B018A010E94F08137
:109C200081508E3FA0F45701C0E0D0E001501109EF
:109C3000C017D1077CF4C6018C0F9D1F0E94F081D4
:109C4000F50181935F01882329F02196F1CF80E00F
:109C500090E005C0CE0DDF1D188281E090E0DF911D
:109C6000CF911F910F91FF90EF90DF90CF90BF9019
:109C7000AF900895882319F067E571E102C069E5A6
:109C800071E18FE698E00C94CF5DCF93DF93CDB771
:109C9000DEB72C970FB6F894DEBF0FBECDBF65ECD4
:109CA00070E18FE698E00E94CF5D86E490E00E942C
:109CB000F0818B37A1F51C821B821E821D828FEFE3
:109CC0009FEF98878F8384E593E09A83898386E466
:109CD00090E09A8789871C861B868091710B9091F2
:109CE000720B0E947565CE0101960E94F753909306
:109CF000720B8093710B892B19F464EA70E111C027
:109D00006BE970E18FE698E00E94CF5D0E94984772
:109D100081EE9AE00E94CE4381E090E008C062EBC1
:109D200070E18FE698E00E94CF5D80E090E02C9695
:109D30000FB6F894DEBF0FBECDBFDF91CF9108956F
:109D4000AF92BF92CF92DF92EF92FF920F931F9349
:109D5000CF93DF93CDB7DEB7C856D1090FB6F894CD
:109D6000DEBF0FBECDBF1AA619A6FE01BB962EE11F
:109D7000DF011D922A95E9F78E01075D1F4F0297BB
:109D800074F0FB01628173814FE150E0C8010E94D1
:109D90001C87B80186E190E00E941D4C10C040E293
:109DA00050E0B80186E190E00E94014E892B39F421
:109DB00040E250E065E372E1C8010E94B77A809109
:109DC000CF071F928F938091CE071F928F93809120
:109DD000CD071F928F938091CC071F928F93809114
:109DE000CB071F928F938091CA071F928F9388E3AE
:109DF00095E09F938F931F9288E28F93CE010196F7
:109E00006C019F938F930E942B8761E272E18FE632
:109E100098E00E94CF5DB8018FE698E00E94F65E60
:109E2000B6018FE698E00E94F65E8FE698E00E9409
:109E3000F25E0FB6F894A8958091600088618093D7
:109E40006000109260000FBE7E0199E4E90EF11CE3
:109E5000D70113961C921E92129788EE93E0A0E011
:109E6000B0E0F70184839583A683B78384E0848779
:109E700084EF92E09183808316870587108A178686
:109E800080E590E0928B818B158A67E67CE285E223
:109E90009FE20E94357B8C010FB6F894DEBF0FBEA7
:109EA000CDBF892BE1F183E090E00E94A777D80134
:109EB0001D969C938E931C97FC01F182E082128286
:109EC000C7010E946742882319F0C7010E94CE4350
:109ED000D7011F966D917C9150975196AD90BC9093
:109EE00052976115710569F0CE01815A9F4F0E940A
:109EF000F85EA501BE01615A7F4FC7010E94443D33
:109F000007C0F70165857685A501C7010E946A41F2
:109F1000181619060CF4A0C0C8010E94FE2E00E01D
:109F200010E0F701E388F48899E288E10FB6F8942D
:109F3000A895809360000FBE9093600001151105F5
:109F400009F46BC0F8ECEF16F10409F058C065E1B4
:109F500072E18FE698E00E94CF5DA3961FAE1EAE21
:109F6000A397A5961FAE1EAEA5978FEF9FEFA7965E
:109F70009FAF8EAFA7978AE693E0A1969FAF8EAF73
:109F8000A197A9961FAF0EAFA997F8948091710B76
:109F90009091720B0E947565CE01815A9F4F0E946D
:109FA000F7539093720B8093710B7894C8010E94C1
:109FB000FE2E8091710B9091720B892B79F46EEFCC
:109FC00071E18FE698E00E94CF5D0E94336BDC0167
:109FD000CB018856954CAF4FBF4F33C063EF71E153
:109FE0008FE698E00E94CF5D0E9498476CEE71E189
:109FF0008FE698E00E94CF5D82E090E0CDC064EDF6
:10A0000071E18FE698E00E94CF5D4AE050E0B70131
:10A010008FE698E00E94995E0CC062EC71E18FE6D9
:10A0200098E00E94CF5D69EA71E18FE698E00E94B6
:10A03000CF5D0E94336BDC01CB0188579C4EAF4F44
:10A04000BF4F80936D0B90936E0BA0936F0BB093EB
:10A05000700B85EF9FEFA0C0D7011D96BC901D9798
:10A060001E96AC90DF92CF9285EA91E19F938F93F9
:10A070001F930F930E94BE7BDF92CF9280EA91E103
:10A080009F938F931F930F930E94BE7BD8011C96C2
:10A09000ED91FC911D9781E08283DF92CF928DE953
:10A0A00091E19F938F931F930F930E94BE7BD801E2
:10A0B0001C96ED91FC911D971282AF92BF9287E69C
:10A0C00091E19F938F931F930F930E94BE7B82EA2F
:10A0D00091E19F938F931F930F930E94BE7BF70193
:10A0E000148A138AD8011C96ED91FC911D97A080CB
:10A0F000B1800FB6F894DEBF0FBECDBF83E3C82E8C
:10A10000D12CD501ED91FC910084F185E02DC501A4
:10A11000199541975CF4B1E0CB1AD10839F064E1AC
:10A1200070E080E090E00E94F96AEBCF6E01FFE5FD
:10A13000CF0ED11CDF92CF928BE591E19F938F934D
:10A140001F930F930E94DB7B0F900F900F900F9047
:10A150000F900F90019709F0E4CEF6018081918174
:10A16000D70154969C938E935397D12C80E08A30DC
:10A1700039F4BAE0DB1609F4D4CE9AE0D92E03C044
:10A180008D3009F0D82EC8010E94807B8F3F79F76F
:10A19000C8010E94FE2EC5CEC859DF4F0FB6F894F5
:10A1A000DEBF0FBECDBFDF91CF911F910F91FF900A
:10A1B000EF90DF90CF90BF90AF9008950E94A04E97
:10A1C00090939D0580939C0581EE9AE00C94CE437C
:10A1D0002F923F924F925F926F927F928F929F92B7
:10A1E000AF92BF92CF92DF92EF92FF920F931F93A5
:10A1F000CF93DF93CDB7DEB728970FB6F894DEBFC5
:10A200000FBECDBF8C016B010E94192E019609F47F
:10A21000D3C2D801ED91FC910284F385E02DC801F1
:10A2200019957C018F3FBFEF9B0709F4C5C2D80188
:10A23000ED91FC910684F785E02D682FC8011995F2
:10A24000B2E2EB16F10429F4B601C8010E943A2EDD
:10A25000B5C2EDE2EE16F10429F0C701C0970A97E6
:10A2600008F044C1D801ED91FC910284F385E02D02
:10A27000C80119957C018F3FBFEF9B0709F49CC271
:10A280008D9789F4D801ED91FC910284F385E02D3E
:10A29000C80119957C01019609F48EC2EFEFFFEF1A
:10A2A000F887EF8304C021E030E038872F83C701AF
:10A2B000C097A12CB12C0A97C8F49AE0992E9A9CC9
:10A2C000C0019B9C900D1124B701605371095B0183
:10A2D000A80EB91ED801ED91FC910284F385E02D02
:10A2E000C80119957C01C0970A9748F3BEE2EB16A6
:10A2F000F104D1F0C7018F7D85349105A9F0EF817C
:10A30000F885AE9EC001AF9E900DBE9E900D1124AB
:10A31000092E000CAA0BBB0BF60181879287A3873D
:10A32000B48782E08087D8C0B501BB0C880B990B3D
:10A330000E94DB832B013C01FEE2EF16F104A1F544
:10A34000D801ED91FC910284F385E02DC8011995A7
:10A350007C01212C312C20E030E040E251E4C301AB
:10A36000B2010E9490844B015C01B70160537109F6
:10A37000072E000C880B990B0E94DB83A50194012A
:10A380000E94C0822B013C01B1E02B1A3108D80198
:10A39000ED91FC910284F385E02DC80119957C01B3
:10A3A000C0970A97C0F202C0212C312CC7018F7DC3
:10A3B0008534910509F042C0D801ED91FC910284E9
:10A3C000F385E02DC80119957C018B32910559F474
:10A3D000D801ED91FC910284F385E02DC801199517
:10A3E0007C01B1E00CC08D9761F4D801ED91FC9136
:10A3F0000284F385E02DC80119957C01BFEFBE836F
:10A4000002C0E1E0EE83A12CB12C8AE0982EC701B6
:10A41000C0978A309105B0F49A9C90019B9C300DB6
:10A4200011245C01A20EB31ED801ED91FC910284AF
:10A43000F385E02DC80119957C01E9CFB1E0BE8319
:10A44000A12CB12CEF81F885BF01FF0F880B990B70
:10A450000E94DB83A30192010E9490842B013C01A6
:10A46000B501BB0C880B990B0E94DB834B015C018F
:10A47000FE816F2FFF0F770B880B990B0E94DB83F8
:10A480009B01AC01C501B4010E9490844B015C01A9
:10A49000B101330C880B990B0E94DB839B01AC014B
:10A4A000C501B4010E94C0829B01AC0160E070E074
:10A4B00080E291E40E94FD849B01AC01C301B201E2
:10A4C0000E949084D60119966D937D938D939C93F1
:10A4D0001C9783E018968C93D801ED91FC9106842B
:10A4E000F785E02D6E2DC801199522C0BBE5EB164E
:10A4F000F10409F060C0D801ED91FC910284F3856C
:10A50000E02DC80119958B35910509F055C185E0FD
:10A51000F6018087C8010E94192ED801ED91FC91A7
:10A520000284F385E02DC80119958D35910519F444
:10A5300080E090E043C1D801ED91FC910684F7855D
:10A54000E02D682FC8011995BB24BA940E94F22E01
:10A550007C01009709F430C1BB2021F0F6019783FC
:10A56000868308C0D40113969C938E931297FC01A6
:10A5700095828482C8010E94192EB701C8010E94E9
:10A58000E850892B09F018C1C8010E94192ED80182
:10A59000ED91FC910284F385E02DC8011995B12C51
:10A5A00047018C32910591F221E030E08D35910523
:10A5B00009F089C086C0BBE7EB16F10409F088C03A
:10A5C000D801ED91FC910284F385E02DC801199525
:10A5D0008B37910509F0F0C086E0F6018087C8014D
:10A5E0000E94192ED801ED91FC910284F385E02D93
:10A5F000C80119958D37910509F49ACFD801ED91CD
:10A60000FC910684F785E02D682FC80119959924DF
:10A610009A940E94F22E7C01009709F4CDC09920F3
:10A6200021F0F6019783868308C0D50113969C9389
:10A630008E931297FC01B582A482C8010E94192E44
:10A64000B701C8010E943A2E019609F4B5C0C801AD
:10A650000E94192ED70119968D919C911A971196E7
:10A660009C938E931A961C921E921997D801ED9185
:10A67000FC910284F385E02DC8011995CA9709F071
:10A680009BC0C8010E94192EB701C8010E94E85062
:10A69000019609F491C0C8010E94192ED801ED91CC
:10A6A000FC910284F385E02DC8011995912C570186
:10A6B0008C32910509F4ADCF21E030E08D37910562
:10A6C00011F420E030E088279927821B930B76C095
:10A6D000BEE6EB16F10411F519821A821B821C8268
:10A6E000D801ED91FC910484F585E02D44E050E023
:10A6F000BE016F5F7F4FC8011995049709F05CC0D8
:10A7000044E050E067EA74E0CE0101960E940E87B3
:10A71000009709F051C0F601108650C0F6E6EF161A
:10A72000F10421F59E012F5F3F4F790185E0D901AA
:10A730001D928A95E9F7D801ED91FC910484F58585
:10A74000E02D45E050E0B901C80119950597A1F544
:10A7500045E050E061EB74E0C7010E940E8700976E
:10A7600059F521E0F6012087118628C0F4E7EF169D
:10A77000F10411F519821A821B821C82D801ED9115
:10A78000FC910484F585E02D44E050E0BE016F5F4C
:10A790007F4FC8011995049779F444E050E06CEAC2
:10A7A00074E0CE0101960E940E87009729F421E003
:10A7B000F6012087218702C08FEF9FEF28960FB602
:10A7C000F894DEBF0FBECDBFDF91CF911F910F91E7
:10A7D000FF90EF90DF90CF90BF90AF909F908F90C1
:10A7E0007F906F905F904F903F902F9008950F93C0
:10A7F0001F93CF93DF93009791F08C010E94F22E6C
:10A80000EC01892B61F0C8010E94192EBE01C8011C
:10A810000E94E850019631F4CE010E94756580E0F7
:10A8200090E001C0CE01DF91CF911F910F9108956B
:10A83000282F3091D30B313208F04AC08091AF0BF2
:10A840008111FCCF9091D20B42E04093AF0B20934B
:10A85000AE0B2FEF2093AD0B1092AC0B3093AB0BE4
:10A86000E2EBFBE0ABE8BBE020E0321721F04191E6
:10A870004D932F5FFACF10928A0B20918A0B990F7C
:10A88000922B90938A0B9091890B913061F41092E6
:10A89000890B90918A0B9093BB009091BC0093FD23
:10A8A000F8CF95EC01C095EE9093BC009091AF0B62
:10A8B0009230E1F39091AD0B9F3F79F08091AD0B19
:10A8C000803241F08091AD0B803331F084E005C0DF
:10A8D00081E003C082E001C083E01092B10B1092CE
:10A8E000D30B1092B00B08950F931F93CF93DF9368
:10A8F000EC010E94F35D8C01CE010E94F25E800F9C
:10A90000911FDF91CF911F910F910895DF92EF92E8
:10A91000FF920F931F93CF93DF93CDB7DEB72997A5
:10A920000FB6F894DEBF0FBECDBF8C017B01AE0128
:10A930004F5F5F4F0E946940D82E882309F459C0A9
:10A94000F7018081803109F454C08FE78D83F801CD
:10A95000858196810E94DE3FB701F801858196814D
:10A960000E94943F40E06EE4F801858196810E9448
:10A97000723F40E06B81F801858196810E94723FB1
:10A9800040E06C81F801858196810E94723FF70159
:10A990008081803139F040E06D81F80185819681B8
:10A9A0000E94723FF801858196810E94DE3FB701C7
:10A9B000F801858196810E94943FF801408168E406
:10A9C000858196810E94723F64E170E080E090E0B2
:10A9D0000E94F96AF8018081882331F06AE070E012
:10A9E00080E090E00E94F96AF801858196810E94DA
:10A9F000DE3F8D2D29960FB6F894DEBF0FBECDBF7A
:10AA0000DF91CF911F910F91FF90EF90DF9008950C
:10AA1000EF92FF920F931F93CF93DF93EC018C0182
:10AA2000085F1F4F7E01699170E084E0759567951E
:10AA30008A95E1F740E150E08FE698E00E94995E48
:10AA4000F70160816F7070E040E150E08FE698E0C0
:10AA50000E94995EC017D10729F7DF91CF911F910E
:10AA60000F91FF90EF9008951092880B1092870B32
:10AA70001092B10B1092D30B1092AF0B81E0809328
:10AA8000AE0B1092890B61E084E10E946E3661E0AA
:10AA900085E10E946E36E9EBF0E080818E7F808355
:10AAA00080818D7F808388E48093B80085E48093E3
:10AAB000BC008DE893E29093860B8093850B8EE823
:10AAC00093E29093840B8093830B0895CF93C82FC8
:10AAD000462F61E070E00E94474361E070E08C2FF8
:10AAE0000E941D448111F9CFCF91089520E5FC010A
:10AAF000208311820895FC018485843011F00C9428
:10AB0000AD4580E008958F929F92AF92BF92CF9211
:10AB1000DF92EF92FF920F931F93CF93DF936B011E
:10AB20007C01142F9B01AC010E944D85882319F0F4
:10AB300063E675E027C046015701E894B7F82FEFA8
:10AB40003FEF4FE75FE7C501B4010E944D858111DA
:10AB50000DC02FEF3FEF4FE75FE7C501B4010E9443
:10AB60002C8318161CF467E675E00CC02FEF3FEF3E
:10AB70004FE75FE4C701B6010E948B84181694F476
:10AB80006BE675E08FE698E0DF91CF911F910F9112
:10AB9000FF90EF90DF90CF90BF90AF909F908F90FD
:10ABA0000C94F35D2FEF3FEF4FE75FECC701B60169
:10ABB0000E942C8387FDE4CF20E030E0A901C7018B
:10ABC000B6010E942C8387FF0BC06DE28FE698E0F0
:10ABD0000E94C85DEC01F7FAF094F7F8F09402C017
:10ABE000C0E0D0E000E060E070E080E09FE310179C
:10ABF00041F020E030E040E251E40E9431830F5FF9
:10AC0000F6CFA70196010E94C0826B017C010E94D1
:10AC1000AA834B015C012AE0AB01BC018FE698E0FE
:10AC20000E94085EC80FD91F1123C9F1C501B401E4
:10AC30000E94D9839B01AC01C701B6010E94BF826B
:10AC40006B017C016EE28FE698E00E94C85DC80F40
:10AC5000D91F20E030E040E251E4C701B6010E9474
:10AC600090844B015C010E94AA836B01E12CF12CC2
:10AC70002AE0B701A6018FE698E00E94085EC80F9F
:10AC8000D91FC701B6010E94D9839B01AC01C50140
:10AC9000B4010E94BF826B017C011150D1F6CE013C
:10ACA000DF91CF911F910F91FF90EF90DF90CF90A8
:10ACB000BF90AF909F908F900895CF92DF92EF92C8
:10ACC000FF92CF93DF93EC010E94336B6B017C0109
:10ACD00080912A0990912B09DC01ED91FC9100846F
:10ACE000F185E02D1995892B79F40E94336BDC01F5
:10ACF000CB018C199D09AE09BF0988399A43A1057A
:10AD0000B10530F380E00DC080912A0990912B09A4
:10AD1000DC01ED91FC910284F385E02D1995888387
:10AD200081E0DF91CF91FF90EF90DF90CF90089579
:10AD30004F925F926F927F928F929F92AF92BF924B
:10AD4000CF92DF92EF92FF920F931F93CF93DF93F7
:10AD50001F921F92CDB7DEB75C018CE299E00E9492
:10AD60005D5681113AC036C08C01CE0101960E9419
:10AD70005D56882379F1C80101962981F701219355
:10AD80007F01422F4F7750E0449DB001459D700DEB
:10AD9000549D700D1124C60ED71E47E0440C551C5F
:10ADA000661C771C4A95D1F727FF27C0853091058F
:10ADB000D9F68FEF9FEF9093C6098093C5098091D4
:10ADC0002A0990912B09DC01ED91FC910488F58909
:10ADD000E02D199580E090E08EC090902C091982AA
:10ADE0008DE2E82E89E0F82E01E010E0C12CD12C94
:10ADF000412C512C32014394B8CFF92DF07FFA83C6
:10AE00002FEF280FD5012C93F03319F5845D964F61
:10AE10000E945D568823F1F2C801825D964F0E9420
:10AE20005D568823B9F2C8010396D501EC91F0E094
:10AE3000EA5DF64FE780F12CFE2CEE242085E20E31
:10AE4000F11C20912C0921FF08C0B2E0EB0EF11C8F
:10AE500004C020E0E12CF12C01C022E0422E512C54
:10AE6000FC01EA5DF64F4F018C01481A590A2EEF9A
:10AE7000622E77247A94C801840D951D8C159D054A
:10AE800078F5CE0101960E945D56882309F4A2CF81
:10AE90008091C3099091C4090097B1F0FA81F03311
:10AEA00099F4D5012C91F301E21BF1099F01200FC8
:10AEB000311FE216F30640F4DC01ED91FC910190A4
:10AEC000F081E02D698119950038110518F4898108
:10AED000F40186830F5F1F4FFFEF8F1A9F0ACBCFBE
:10AEE0008091C3099091C409892B21F4013811057F
:10AEF00008F070CFC8010F900F90DF91CF911F9194
:10AF00000F91FF90EF90DF90CF90BF90AF909F9008
:10AF10008F907F906F905F904F9008952F923F9207
:10AF20004F925F926F927F928F929F92AF92BF9259
:10AF3000CF92DF92EF92FF920F931F93CF93DF9305
:10AF40001F92CDB7DEB70E943C63382E882309F4E8
:10AF500022C10E94336B2B013C018091B209909178
:10AF6000B309A091B409B091B509A3019201281BBE
:10AF7000390B4A0B5B0BDA01C90189399A43A105E8
:10AF8000B105A8F48091AE099091AF09A091B009E4
:10AF9000B091B109A3019201281B390B4A0B5B0B3D
:10AFA000DA01C90189399A43A105B105C8F1209197
:10AFB000B60980912A0990912B09222371F02CEF78
:10AFC0003FEF3093C6092093C509DC01ED91FC9158
:10AFD0000488F589E02D1995DDC020EC20932C091B
:10AFE00010922D09DC01ED91FC910280F381E02D9E
:10AFF00042E050E06CE279E019954092AE0950923F
:10B00000AF096092B0097092B1094092B2095092B2
:10B01000B3096092B4097092B50981E08093B609D2
:10B0200080912A0990912B09DC01ED91FC9100841B
:10B03000F185E02D1995892B09F4ADC0CE0101965B
:10B040000E9498565C01892B09F4A0C04092B20975
:10B050005092B3096092B4097092B50980912C099D
:10B06000807F803309F076C08091B7099091B8094C
:10B07000892B09F490C0E980F12CF701EA5DF64FC5
:10B08000078110E0102F00278085080F111D970100
:10B09000225D364F4901B701615D764FA801C901B4
:10B0A0000E94B386B8016E0D7F1DDB01AA5DB64F0D
:10B0B00018961C92189780912C098670282EE09182
:10B0C000B709F091B80932E0831337C01996CC90D4
:10B0D0001997D12CDC2CCC241A968C91C80ED11C3B
:10B0E0004BEF5FEF4E195F09401B510B4A0D5B1D83
:10B0F0006F5C764FC401199580E480932C092092EF
:10B100002D09D0922E09C0922F0980912A09909181
:10B110002B09DC01ED91FC910280F381E02D44E0EC
:10B1200050E06CE279E019954092AE095092AF0977
:10B130006092B0097092B1092EC04DEF5FEF4E19C9
:10B140005F09401B510B4A0D5B1D615D764FC401C9
:10B15000199521C0803CA9F480ED80932C091092B0
:10B160002D0980912A0990912B09DC01ED91FC9128
:10B170000280F381E02D42E050E06CE279E0199525
:10B180000AC0803D41F41092B60905C00E943C639C
:10B19000811101C0312C832D0F90DF91CF911F9130
:10B1A0000F91FF90EF90DF90CF90BF90AF909F9066
:10B1B0008F907F906F905F904F903F902F90089569
:10B1C000AF92BF92CF92DF92EF92FF921F93CF93F5
:10B1D000DF9300D000D0CDB7DEB76C017C0110E06A
:10B1E0008AE0A82EB12C1330A9F0F701828190E0FB
:10B1F000A0E0B0E089839A83AB83BC83BE82AD823A
:10B20000BE016F5F7F4F8FE698E00E94DC2164E40F
:10B2100072E114C0F601858190E0A0E0B0E089837E
:10B220009A83AB83BC83BE82AD82BE016F5F7F4FCA
:10B230008FE698E00E94DC2161E472E10E94CF5D1C
:10B240001F5FFFEFEF1AFF0A143069F626960FB65C
:10B25000F894DEBF0FBECDBFDF91CF911F91FF905D
:10B26000EF90DF90CF90BF90AF9008950F931F9312
:10B27000CF93DF931F921F92CDB7DEB78C018AE187
:10B2800093E0F801918380831282138214821582E5
:10B29000CE0101960E94765589819A810E94B63C22
:10B2A000B8016E5F7F4F44E050E08FE090E00E9475
:10B2B000E22F0E94B53CC8010F900F90DF91CF9113
:10B2C0001F910F910895CF93DF93C6E2D9E080EEEE
:10B2D0008E831F828C819D81DC01ED91FC91028027
:10B2E000F381E02D42E050E06CE279E019958FEFB8
:10B2F0009FEF9093C6098093C5098C819D81DC01E5
:10B30000ED91FC910680F781E02D19958C819D814E
:10B31000DC01ED91FC910488F589E02D19950E94DE
:10B32000336B6093AE097093AF098093B00990932B
:10B33000B1096093B2097093B3098093B4099093F3
:10B34000B509DF91CF910895AF92BF92CF92DF926E
:10B35000EF92FF920F931F93CF93DF931F921F9251
:10B36000CDB7DEB77A836983BA01A901E981FA8191
:10B37000F770082F10E0000F111F0558144FD80167
:10B380008D919C918E0F9F1F9F01240F351F21309F
:10B390003840A0F07A015B0160E078E06B01CE1AE2
:10B3A000DF0AA601B5010E94E22FA7014C195D0931
:10B3B000B5016C0D7D1DF801808191810F900F907A
:10B3C000DF91CF911F910F91FF90EF90DF90CF9081
:10B3D000BF90AF900C94E22F9F92AF92BF92CF920A
:10B3E000DF92EF92FF920F931F93CF93DF93982EEC
:10B3F0008B015A01690164E270E00E941D44E82E4D
:10B40000F12C65E270E0892D0E941D44FE2CEE2493
:10B41000E82AE801CE0DDF1D9E013770E92CF12CE2
:10B42000C701880F991FAC014D58544F7A01FA019A
:10B4300080819181820F931FA9014C0D5D1D4130C8
:10B44000584090F000E018E0021B130BA801B50172
:10B450000E941230A601401B510BB501600F711FF5
:10B46000F7018081918102C0A601B5010E941230CE
:10B47000CC0DDD1D4D2F64E270E0892D0E94474305
:10B480004C2F65E270E0892DDF91CF911F910F91D4
:10B49000FF90EF90DF90CF90BF90AF909F900C9473
:10B4A0004743FF920F931F93CF93DF93F82E00E053
:10B4B00010E08F2D0E947430EC01892B21F08F2D2C
:10B4C0000E9474308C01C017D10799F7CE01DF912B
:10B4D000CF911F910F91FF90089520E3FC012083ED
:10B4E0003296862F82958F7090E1899F6019112482
:10B4F0006A3014F4605D01C0695C6293682F811149
:10B50000F0CF08952F923F924F925F926F927F9269
:10B510008F929F92AF92BF92CF92DF92EF92FF9263
:10B520000F931F93CF93DF93CDB7DEB7E2970FB69C
:10B53000F894DEBF0FBECDBF7C012A013B0169013B
:10B540000E94336B4B015C0187010D5B1F4FC801EB
:10B550000E94534518161906A4F00E94336BDC01B3
:10B56000CB0188199909AA09BB09481659066A0628
:10B570007B06D8F062E370E080E090E00E94F96A18
:10B58000E6CF42E250E0BE016F5F7F4FC8010E94EC
:10B590000B458981823011F080E060C1F801848917
:10B5A000958983349105C1F702C08FEF57C16D8132
:10B5B0007E818F8198850E9495824B015C01F60106
:10B5C000608371838283938346E050E0B701685FB4
:10B5D0007F4FCE014D960E94A686892BE9F6F70192
:10B5E00080819181A281B38188169906AA06BB0643
:10B5F00098F284819581A681B78188159905AA055D
:10B60000BB0550F289899A89AB89BC89868797875F
:10B61000A08BB18B8EECC82ED12CC8010E942A457C
:10B62000F1E0CF1AD108C9F7712CC70182969AA709
:10B6300089A7F701B696FCA7EBA708969EA78DA74A
:10B640003C974F01899698AB8FA73897FAABE9AB37
:10B650001701F6E12F0E311C27018EE1480E511C17
:10B66000F801818D928D181619060CF0F6C0C801EC
:10B670000E942A458333910509F4C9C0F4F481304E
:10B680009105B9F11CF4892B59F3DBC08330910586
:10B69000C1F1069709F0D5C0C8010E942A456C0186
:10B6A00044E050E0B201C8010E940B45A12CB12C2E
:10B6B000DD2494E0C91AD1083FC08A33910509F40A
:10B6C0007AC03CF48533910561F0C69709F43FC018
:10B6D000B8C08B33910509F484C08F3F910501F206
:10B6E000B0C0C8010E942A45C8010E942A45782E90
:10B6F000B7CFC8010E942A4544E050E069A97AA961
:10B700003AC0C8010E942A456C0144E050E0B101F2
:10B71000C8010E940B45A12CB12CDD24F4E0CF1A06
:10B72000D108AC14BD040CF09BCFC8010E942A457F
:10B730008FEFA81AB80AF5CFAC14BD040CF090CF67
:10B74000C8010E942A45EFEFAE1ABE0AF5CFC80124
:10B750000E942A45682EF701828D811110C0838DC9
:10B7600081110DC0848D81110AC0858D811107C0A2
:10B7700044E050E0B401C8010E940B4571CFEFA531
:10B78000F8A9A080B180C280D380B401CE01839695
:10B790000E94F85E8DA19EA1AFA1B8A5A816B9061A
:10B7A000CA06DB0629F3662009F45ACFC8010E94B5
:10B7B0002A456A94F8CFC8010E942A4544E050E027
:10B7C0006BA57CA5C8010E940B45F70166A177A176
:10B7D00080A591A50E94958266A377A380A791A7D3
:10B7E0003FCFC8010E942A4544E050E06DA57EA5E8
:10B7F000C8010E940B45F70162A573A584A595A514
:10B800000E94958262A773A784A795A729CFC80134
:10B810000E942A4544E050E069A57AA5C8010E942B
:10B820000B45F70162A173A184A195A10E949582A5
:10B8300062A373A384A395A366A777A780AB91ABFC
:10B840000FCFC8010E942A45D82EDD2009F408CF69
:10B85000C8010E942A45DA94F8CF872DE2960FB6E8
:10B86000F894DEBF0FBECDBFDF91CF911F910F9136
:10B87000FF90EF90DF90CF90BF90AF909F908F9010
:10B880007F906F905F904F903F902F900895CF9250
:10B89000DF92EF92FF920F931F93CF93DF936C0190
:10B8A0007A018B01C0E0D0E0CE15DF0581F0D80130
:10B8B0006D918D01D601ED91FC910190F081E02D0B
:10B8C000C6011995892B11F02196EECF7E01C70193
:10B8D000DF91CF911F910F91FF90EF90DF90CF906C
:10B8E0000895FC01538D448D252F30E0842F90E086
:10B8F000821B930B541710F0CF960895019708956B
:10B90000FC01918D828D981761F0828DDF01A80F67
:10B91000B11D5D968C91928D9F5F9F73928F90E089
:10B9200008958FEF9FEF0895FC01918D828D9817F8
:10B9300031F0828DE80FF11D858D90E008958FEF35
:10B940009FEF0895FC01918D228D892F90E0805CFE
:10B950009F4F821B91098F739927089582ED97E07D
:10B960000E94A25C21E0892B09F420E0822F089537
:10B970008FE698E00E94A25C21E0892B09F420E088
:10B98000822F0895FC01848DDF01A80FB11DA35AF9
:10B99000BF4F2C91848D90E001968F739927848FEF
:10B9A000A689B7892C93A089B1898C918370806412
:10B9B0008C93938D848D981306C00288F389E02DB3
:10B9C00080818F7D80830895EF92FF920F931F9364
:10B9D000CF93DF93EC0181E0888F9B8D8C8D981342
:10B9E00005C0E889F989808185FD26C0F62E0B8D7A
:10B9F00010E00F5F1F4F0F731127E02E8C8DE812A0
:10BA00000CC00FB607FCFACFE889F989808185FF61
:10BA1000F5CFCE010E94C25CF1CF8B8DFE01E80F05
:10BA2000F11DE35AFF4FF0829FB7F8940B8FEA891C
:10BA3000FB89808180620AC09FB7F894EE89FF89F4
:10BA40006083E889F98980818370806480839FBFE7
:10BA500081E090E0DF91CF911F910F91FF90EF90E7
:10BA60000895CF93DF93EC01888D8823C9F0EA898C
:10BA7000FB89808185FD05C0A889B9898C9186FDE7
:10BA80000FC00FB607FCF5CF808185FFF2CFA889E4
:10BA9000B9898C9185FFEDCFCE010E94C25CE7CFC2
:10BAA000DF91CF91089580E090E0892B21F00E94F2
:10BAB000B85C811121C080E090E0892B41F080E0EA
:10BAC00090E0892B21F00E940000811118C080E0D5
:10BAD00090E0892B21F00E94AE5C811113C080E0C0
:10BAE00090E0892BA1F080E090E0892B81F00E940A
:10BAF000000081110AC008950E940000DCCF0E945E
:10BB00000000E5CF0E940000EACF0C9400000895E9
:10BB10000E948786EF92FF920F931F93CF93DF933C
:10BB2000EC018B017A010E94336BFE01E857FF4F55
:10BB300060837183828393838C819D81DC01ED918D
:10BB4000FC910280F381E02DA701B801DF91CF9134
:10BB50001F910F91FF90EF9019941F93CF93DF9354
:10BB6000EC01162F0E94336BFE01E857FF4F6083F4
:10BB70007183828393838C819D81DC01ED91FC91A3
:10BB80000190F081E02D612FDF91CF911F911994E9
:10BB9000DC01ED91FC910190F081E02D1994EF9280
:10BBA000FF920F931F93CF93DF938C017B01C0E033
:10BBB000D0E0F701EC0FFD1F6491662361F0D8011E
:10BBC000ED91FC910190F081E02DC8011995892B30
:10BBD00011F02196EECFCE01DF91CF911F910F9101
:10BBE000FF90EF9008956115710579F0FB010190C8
:10BBF0000020E9F73197AF01461B570BDC01ED91AF
:10BC0000FC910280F381E02D199480E090E008958A
:10BC10008F929F92AF92BF92EF92FF920F931F93DA
:10BC2000CF93DF93CDB7DEB7A1970FB6F894DEBF01
:10BC30000FBECDBF7C01FA01CB0119A2223008F45E
:10BC40002AE08E010F5D1F4F822E912CA12CB12C6A
:10BC5000BF01A50194010E941682F901CA01015099
:10BC600011096A3014F4605D01C0695CD8016C93FD
:10BC7000232B242B252B61F7B801C7010E94F35D0C
:10BC8000A1960FB6F894DEBF0FBECDBFDF91CF9166
:10BC90001F910F91FF90EF90BF90AF909F908F906A
:10BCA0000895CF92DF92EF92FF920F931F93CF935D
:10BCB000DF932115310581F4DC01ED91FC910190B8
:10BCC000F081E02D642FDF91CF911F910F91FF90B4
:10BCD000EF90DF90CF9019942A30310501F577FF6E
:10BCE0001DC06A017B01EC016DE20E94C85D8C0100
:10BCF00044275527BA014C195D096E097F092AE0CE
:10BD0000CE010E94085E800F911FDF91CF911F919D
:10BD10000F91FF90EF90DF90CF9008952AE0DF9190
:10BD2000CF911F910F91FF90EF90DF90CF900C94E7
:10BD3000085E9A01AB01770F660B770B0C94515E8E
:10BD40009A01452B39F4DC01ED91FC910190F081D1
:10BD5000E02D1994462F50E060E070E00C94085EEE
:10BD60008F929F92AF92BF92CF92DF92EF92FF920B
:10BD70000F931F93CF93DF937C018B014C0182E0E3
:10BD8000880E911C5701E5E0AE0EB11CC0E0D0E07A
:10BD9000F40161914F014AE050E0C8010E94A05EA9
:10BDA0006C016EE2C8010E94C85D8C0D9D1DC80F1C
:10BDB000D91F8A149B0461F74AE050E0F7016581BE
:10BDC000C8010E94A05E8C0F9D1FDF91CF911F9133
:10BDD0000F91FF90EF90DF90CF90BF90AF909F902A
:10BDE0008F9008956AEE73E00C94F35D0C94F35D0C
:10BDF000DC018AE193E08D939D9384E0FB01019047
:10BE00000D928A95E1F708951F920F920FB60F9247
:10BE100011240BB60F922F933F934F935F936F9321
:10BE20007F938F939F93AF93BF93EF93FF9382ED95
:10BE300097E00E94C25CFF91EF91BF91AF919F91FB
:10BE40008F917F916F915F914F913F912F910F90C3
:10BE50000BBE0F900FBE0F901F9018951F920F9260
:10BE60000FB60F9211240BB60F922F938F939F93BF
:10BE7000EF93FF93E091E207F091E3078081E09177
:10BE8000E807F091E90782FD12C090818091EB07ED
:10BE90008F5F8F732091EC07821751F0E091EB07D1
:10BEA000F0E0EE52F84F958F8093EB0701C0808150
:10BEB000FF91EF919F918F912F910F900BBE0F905B
:10BEC0000FBE0F901F9018951F920F920FB60F92F2
:10BED00011240BB60F922F933F934F935F936F9361
:10BEE0007F938F939F93AF93BF93EF93FF938FE6CF
:10BEF00098E00E94C25CFF91EF91BF91AF919F913A
:10BF00008F917F916F915F914F913F912F910F9002
:10BF10000BBE0F900FBE0F901F9018951F920F929F
:10BF20000FB60F9211240BB60F922F938F939F93FE
:10BF3000EF93FF93E0917F08F09180088081E0917A
:10BF40008508F091860882FD12C090818091880852
:10BF50008F5F8F7320918908821751F0E0918808D4
:10BF6000F0E0E159F74F958F8093880801C08081F8
:10BF7000FF91EF919F918F912F910F900BBE0F909A
:10BF80000FBE0F901F9018951F920F920FB60F9231
:10BF900011240BB60F922F933F934F935F938F9380
:10BFA0009F93EF93FF932091E30B3091E40B8091EB
:10BFB000E10B9091E20BAC014F5F5F4F5093E20BAE
:10BFC0004093E10BF901E80FF91F80818093CE00C7
:10BFD00080910602909107022091E10B3091E20BD3
:10BFE0008217930748F48FEF9FEF9093E20B8093B3
:10BFF000E10B88E48093C900FF91EF919F918F91AD
:10C000005F914F913F912F910F900BBE0F900FBEFC
:10C010000F901F9018951F920F920FB60F92112438
:10C020002F933F938F939F932091DF0B3091E00BE1
:10C030008091E10B9091E20B21303105A9F48F3F03
:10C040002FEF920789F41092C8001092CD0089E07A
:10C050008093CC0086E28093CA001092CE001092AA
:10C06000E20B1092E10B17C0892BA9F41092C800C3
:10C070001092CD0083E08093CC008EE08093CA00C4
:10C0800088E28093C9001092CE0081E090E0909306
:10C09000E20B8093E10B9F918F913F912F910F9035
:10C0A0000FBE0F901F9018951F920F920FB60F9210
:10C0B00011240BB60F922F933F934F935F936F937F
:10C0C0007F938F939F93AF93BF93EF93FF93909141
:10C0D000C8008091CE0094FF08C081E08093DE0B01
:10C0E0008091E30B9091E40B57C09091DE0B91305F
:10C0F00099F481110EC082E08093DE0B0E94336BB5
:10C100006093D80B7093D90B8093DA0B9093DB0B71
:10C110003EC01092DE0B44C0923009F041C0E09165
:10C12000DC0BF091DD0B9081891721F091E0909369
:10C13000050280832091DC0B3091DD0B8091D60BC2
:10C140009091D70B2817390711F51092DE0B8091CB
:10C1500005028823D1F08091D40B9091D50B892BC7
:10C16000A1F01092C900E091D40BF091D50B199574
:10C1700080E98093C9001092C8001092CD0083E03E
:10C180008093CC008EE08093CA00109205028091CB
:10C19000DC0B9091DD0B01969093DD0B8093DC0B13
:10C1A000FF91EF91BF91AF919F918F917F916F918F
:10C1B0005F914F913F912F910F900BBE0F900FBE4B
:10C1C0000F901F901895CF92DF92EF92FF920F93EE
:10C1D0001F93CF93DF936C018B0186E090E00E9468
:10C1E000A777EC019093E60B8093E50BF6010190A5
:10C1F0000020E9F7CF018C199D090E94A7777C01E7
:10C20000B6010E94F786F60101900020E9F7319708
:10C21000EC19FD09EE0DFF1D1082F982E8821B83E7
:10C220000A8380918C0590918D059D838C83D0939A
:10C230008D05C0938C05DF91CF911F910F91FF90D9
:10C24000EF90DF90CF900895CF92DF92EF92FF9220
:10C250000F931F93CF93DF93CDB7DEB7EC970FB655
:10C26000F894DEBF0FBECDBFDC012C91222309F470
:10C2700051C065E274E00E94C67A9A8389837E0188
:10C28000B3E0EB0EF11C01E010E0D02EC12E65E210
:10C2900074E080E090E00E94C67AF7018193919368
:10C2A0007F010E31110539F40091E50B1091E60B79
:10C2B000E980FA8008C00F5F1F4F892B31F7F4CF58
:10C2C000F8010481158101151105A1F0D8016D91C6
:10C2D0007C91C7010E94EE86892B91F7D8011296B6
:10C2E000ED91FC911397BE016F5F7F4F8D2D9C2DBB
:10C2F000199506C06AE472E18FE698E00E944D3815
:10C300008FE698E00E94F25E66E472E18FE698E0C4
:10C310000E94CF5DEC960FB6F894DEBF0FBECDBF86
:10C32000DF91CF911F910F91FF90EF90DF90CF9011
:10C330000895FB01248135814281538124173507FB
:10C3400058F440815181DA01A20FB31F8C9384818C
:10C35000958101969583848380E00895CF93DF9340
:10C36000EC0180E893E0998388836115710559F0A9
:10C370008091E90B9091EA0B009729F00E946C38AC
:10C380009B838A8302C01B821A82CE01DF91CF91E8
:10C390000C9482216F927F928F929F92AF92BF9264
:10C3A000CF92DF92EF92FF920F931F93CF93DF9381
:10C3B000CDB7DEB72C970FB6F894DEBF0FBECDBF5A
:10C3C0004C01762E672E6A0159018091E70B9091FE
:10C3D000E80B892BA1F06AE872E18FE698E00E94F1
:10C3E000CF5D60E4C4010E944821A701FF0C660BE9
:10C3F000770BC4010E94BE208FEF9FEF9FC081E0AA
:10C4000090E09093E80B8093E70B26E240E855E23A
:10C4100060E070E082ED97E00E94DE387092C9091A
:10C4200082ED97E09093C8098093C7091092D40ACF
:10C430001092D60A1092D50A0115110541F001306B
:10C44000110539F4FE2CEE24EE24EA9402C0FF24F8
:10C45000FA94C701A0E0B0E08F839887A987BA87D4
:10C4600080E190E09C878B87A60160E070E04983C3
:10C470005A836B837C839E838D834AE050E0672DD3
:10C48000762D8FE698E00E94995E67E872E18FE66C
:10C4900098E00E94CF5DBE016F5F7F4F8FE698E00E
:10C4A0000E94DC218C0163E872E10E94CF5D4AE0CA
:10C4B00050E0B501C8010E94995E60E872E1C801D0
:10C4C0000E94CF5DBE01695F7F4FC8010E94DC21E1
:10C4D0000E94F25EA114B10491F082E0A816B104AA
:10C4E00009F5D0924F0AC0924E0A1092510A10924A
:10C4F000500AF092530AE092520A86E010C0D0929D
:10C500004F0AC0924E0AE11003C080E090E002C0E2
:10C5100080E09FEF9093510A8093500A85E00E943B
:10C52000433906C068E672E18FE698E00E94CF5D6D
:10C530001092E80B1092E70B80E090E02C960FB67B
:10C54000F894DEBF0FBECDBFDF91CF911F910F9149
:10C55000FF90EF90DF90CF90BF90AF909F908F9023
:10C560007F906F900895CF93DF93EC01FA0132969C
:10C57000E60FF71FDC01AD014C1B5D0BCF01861BE5
:10C58000970B2D91222311F02193F5CF9C01241BB1
:10C59000350B620F731FFB01329750833196408336
:10C5A000DF91CF910895EF92FF920F931F93CF9356
:10C5B000DF9300D01F92CDB7DEB77B01BA0130E028
:10C5C000962F9F77660F672F661F770B7195611502
:10C5D000710509F0906821E0230FE1E0F0E0EC0F35
:10C5E000FD1FE30FF11D90836115710511F0322FCE
:10C5F000E7CF30E0B701621B730B6C5F7F4FDB014D
:10C600008C93DE011196F701E21BF30B359685E062
:10C61000E80EF11CEE16FF0619F08D918193FACF0A
:10C6200080912A0990912B092F5F3F4F8901040FB8
:10C63000151FDC01ED91FC910280F381E02DA80132
:10C6400019957C010E94336B6093AE097093AF091A
:10C650008093B0099093B10981E00E151F0509F090
:10C6600080E00F900F900F900F90DF91CF911F916E
:10C670000F91FF90EF900895CF9380912A099091A8
:10C680002B09009771F1DC01ED91FC910688F78987
:10C69000E02D1995C1E0811125C0C0E08091C50948
:10C6A0009091C609892BF1F48DEF9FEF9093C60905
:10C6B0008093C50980912A0990912B09DC01ED91A5
:10C6C000FC910680F781E02D199580912A099091BF
:10C6D0002B09DC01ED91FC910488F589E02D199579
:10C6E00001C0C0E08C2FCF910895DF92EF92FF92AE
:10C6F0000F931F93CF93DF938C01D62EE72EEA0181
:10C70000F22E0E943C638823B9F1F80101900020C9
:10C71000E9F73197E01BF10BCE010796E80FF91FFF
:10C72000E138F10548F545E050E06CE279E0C801F8
:10C730000E94B362AC01ED2DFE2DDC01A45DB64F6D
:10C740009F012C0F3D1FE217F30719F081918D9384
:10C75000FACF2597FF2011F081E301C080E34C0F51
:10C760005D1F6CE279E0DF91CF911F910F91FF90F7
:10C77000EF90DF900C94D36280E0DF91CF911F9116
:10C780000F91FF90EF90DF900895FB010190002042
:10C79000E9F73197AF01461B570B21E00C94756305
:10C7A000CF92DF92EF92FF920F931F93CF93DF937D
:10C7B0001F921F92CDB7DEB76C0161E00E946F211E
:10C7C000182F86FF1BC0C6010E94F6207A8369835A
:10C7D0006AE572E18FE698E00E94CF5D612F70E01C
:10C7E0006F7BE12CF12C01E09E012F5F3F4F41E078
:10C7F00050E0C6010E94B90981E001C080E00F90BD
:10C800000F90DF91CF911F910F91FF90EF90DF90EC
:10C81000CF9008958F929F92AF92BF92CF92DF9266
:10C82000EF92FF920F931F93CF93DF931F921F926C
:10C83000CDB7DEB76C017B0162E070E00E941A2187
:10C840008C0197FF03C080E090E099C063E070E046
:10C85000C6010E941A21AC011816190614F04FE304
:10C8600050E0E982FA820130110531F48F2D880FF2
:10C87000880BF9828A8303C0023011052CF4898168
:10C880009A8199279A838983A981BA8124E630E025
:10C890000E94A4829A01550F440B550B0E943882C6
:10C8A00049015A0189013A83298360E0C6010E9447
:10C8B0006F21E82EF12CC6010E94F620092C000CF5
:10C8C000AA08BB08681579058A059B0559F4012B50
:10C8D000E9F182E0E816F10459F085E0E816F10488
:10C8E000A9F506C0012B71F182E0E816F10479F593
:10C8F00000E020E030E040E050E061E070E0C601A0
:10C900000E94E76600E09E012F5F3F4F41E050E04C
:10C9100060E070E0C6010E94E76686E0E816F10478
:10C9200039F0EA94EF2821F061E0C6010E94482125
:10C9300049815A81052E000C660B770BC6010E94B7
:10C94000BE2004C085E0E816F10431F418C085E08B
:10C95000E816F104B9F6CCCF82E0E816F104B1F3A1
:10C9600062E0C6010E94482100E020E030E040E0A3
:10C9700050E062E070E0C6010E94E766E7CF0F90EA
:10C980000F90DF91CF911F910F91FF90EF90DF906B
:10C99000CF90BF90AF909F908F900895CF92DF92ED
:10C9A000EF92FF920F93CF93DF9300D000D0CDB7DB
:10C9B000DEB77C0161E00E946F2185FF40C0C82E78
:10C9C000D12CC7010E94F620382F292FF70180852E
:10C9D00090E08A30910528F5FC018827E852FF4F46
:10C9E0008F4F0C948D8269837A83832F330F990B39
:10C9F0009C838B83822F220F990B9E838D8300E073
:10CA00009E012F5F3F4F43E050E008C07A83698367
:10CA100000E09E012F5F3F4F41E050E060E070E09A
:10CA200006C000E020E030E040E050E0B601C70181
:10CA30000E94E766B6016F7DC7010E9448212696D5
:10CA40000FB6F894DEBF0FBECDBFDF91CF910F912F
:10CA5000FF90EF90DF90CF9008958F929F92AF92CA
:10CA6000BF92EF92FF920F931F93CF93DF938C01AE
:10CA70007B0149015A010E94F22EEC01892BF9F049
:10CA800083E0888789869A86AB86BC86888199816F
:10CA9000009711F00E943F78C7010E948C8699830D
:10CAA0008883BE01C801DF91CF911F910F91FF9044
:10CAB000EF90BF90AF909F908F900C948738DF914C
:10CAC000CF911F910F91FF90EF90BF90AF909F90EB
:10CAD0008F900895FB0101900020E9F73197AF0195
:10CAE000461B570B20E00C9475630F931F93CF9355
:10CAF000DF93EC012097F9F00A811B81888587FD7F
:10CB000006C08E819F81009711F00E94756588850F
:10CB1000843031F489859A85009711F00E943F781E
:10CB200088819981009711F00E943F78CE010E9480
:10CB30003F78E801DFCFDF91CF911F910F910895EA
:10CB4000FC01848195810895089580E090E0089526
:10CB50008F929F92AF92BF92CF92DF92EF92FF920D
:10CB60000F931F93CF93DF93CDB7DEB7C154D10995
:10CB70000FB6F894DEBF0FBECDBF5C016B018A011A
:10CB80006BEE72E18FE698E00E94CF5DB5018FE613
:10CB900098E00E94F65E68EE72E18FE698E00E94EF
:10CBA000CF5DC114D10409F4A4C00C0D1D1DF80102
:10CBB00010829E012F5F3F4F79018091F60B90917B
:10CBC000F70B009711F482E09CE0F701E81BF90BEA
:10CBD000EA3FF1051CF463EE72E149C0460180169C
:10CBE000910641F0F40161914F018FE698E00E94B7
:10CBF000C85DF5CF8FE698E00E94F25E80919C05BB
:10CC000090919D0520E030E0049719F443E050E056
:10CC100019C042E050E061E4C7010E943726F701E5
:10CC200001900020E9F731978F010E191F09A80123
:10CC3000B701C5010E940E870097A9F020E030E0FF
:10CC400041E050E061E4C7010E943726F7010190FE
:10CC50000020E9F731978F010E191F09A801B701CC
:10CC6000C5010E940E87892B39F068ED72E18FE6CD
:10CC700098E00E94CF5D3DC00A0D1B1D6FE675E078
:10CC8000C8010E94EE86892B21F4C6010E9424610E
:10CC900030C06FE270E0C8010E94E3865C0100973B
:10CCA00041F0FC0110828181843219F1FFEFAF1A4B
:10CCB000BF0AF80180818432E1F0B801C7010E9407
:10CCC000AE61C7010E94B120882399F02985809127
:10CCD0009C0590919D05273019F48430910549F009
:10CCE00041E0049709F440E09501B601C7010E94B4
:10CCF000CA1CCF5BDF4F0FB6F894DEBF0FBECDBFAF
:10CD0000DF91CF911F910F91FF90EF90DF90CF9027
:10CD1000BF90AF909F908F900895CF92DF92EF9247
:10CD2000FF921F93CF93DF9300D000D0CDB7DEB733
:10CD300060EF72E18FE698E00E94CF5D8AECE82E0A
:10CD400087E0F82E10E090E1C92ED12C1530B9F013
:10CD5000F701808190E0A0E0B0E089839A83AB8303
:10CD6000BC83DE82CD82BE016F5F7F4F8FE698E08D
:10CD70000E94DC216EEE72E10E94CF5D14C08091B2
:10CD8000CF0790E0A0E0B0E089839A83AB83BC83B7
:10CD9000DE82CD82BE016F5F7F4F8FE698E00E94FA
:10CDA000DC210E94F25E1F5FFFEFEF1AFF0A1630D0
:10CDB00069F626960FB6F894DEBF0FBECDBFDF91A1
:10CDC000CF911F91FF90EF90DF90CF9008955F92E9
:10CDD0006F927F928F929F92AF92BF92CF92DF928B
:10CDE000EF92FF920F931F93CF93DF93CDB7DEB7F0
:10CDF000E4970FB6F894DEBF0FBECDBF6C017B0188
:10CE00003A01590161E00E946F21002361F0682F0F
:10CE10006062C6010E94482167EC72E18FE698E0EB
:10CE20000E94CF5DB8C01AA219A2FE01B3968EE08F
:10CE3000DF011D928A95E9F720E030E043E050E001
:10CE400060E2CE0101960E943726D6011296ED913E
:10CE5000FC9113976081718140E250E0CE01019610
:10CE60000E94FE86B2E0EB16F104C9F03CF4E11436
:10CE7000F104E1F0EA94EF2879F05FC086E0E8166B
:10CE8000F10451F09EE0E916F10481F0A5E0EA1604
:10CE9000F10409F052C003C06AE874E002C06DE812
:10CEA00074E0CE0181960E94F78650C0A114B104AF
:10CEB00009F44CC08501C12CD12C88E7A82E85E04F
:10CEC000B82E94E0592E7E01B1E3EB0EF11C430124
:10CED000E1E08E1A9108C614D704C4F5D8018C91EC
:10CEE00011969C910E5F1F4F9F938F93BF92AF92AD
:10CEF0001F925F92FF92EF920E942B8740E150E0D9
:10CF0000B701CE0181960E94FE860FB6F894DEBF6F
:10CF10000FBECDBFC814D90461F06BE775E0C7013F
:10CF20000E94F78640E150E0B701CE0181960E9451
:10CF3000FE86FFEFCF1ADF0ACECF69EB72E18FE6F4
:10CF400098E00E94CF5D8FEF9FEF27C063EB72E107
:10CF50008FE698E00E94CF5DBE016F5F7F4F8FE646
:10CF600098E00E94F65E60EB72E18FE698E00E9426
:10CF7000CF5DBE016F5D7F4F8FE698E00E94F65E49
:10CF80008FE698E00E94F25EBE016F5D7F4FCE019A
:10CF900001960E94C56380E090E0E4960FB6F89495
:10CFA000DEBF0FBECDBFDF91CF911F910F91FF90DC
:10CFB000EF90DF90CF90BF90AF909F908F907F9039
:10CFC0006F905F900895FF920F931F93CF93DF931D
:10CFD000CDB7DEB729970FB6F894DEBF0FBECDBF31
:10CFE0008C010E94B120882309F46BC060E0C80165
:10CFF0000E946F21D8011896FC90B7E0FB1671F0E3
:10D00000823009F45CC020F4813009F45DC006C0B0
:10D01000853009F454C0863009F456C0C8010E9416
:10D02000F620362F272F4F2D50E04A30510508F0BB
:10D0300046C0FA018827EE51FF4F8F4F0C948D8226
:10D04000D8011496ED91FC91159780858530B9F53E
:10D0500064EA72E18FE698E00E94CF5DD8011496F1
:10D06000ED91FC911597068117810115110539F194
:10D07000F80161857285CE0101960E94AE61CE01F4
:10D0800001960E94B120882311F1CE0101960E94E1
:10D09000E367892BE1F06CE972E18FE698E00E948A
:10D0A000CF5D12C0292F990F330B03C0832F922F0E
:10D0B0009C0181E090E0232B81F480E00EC080E0B1
:10D0C00004C08FEF9FEF09C081E090E006C0D80157
:10D0D00012960D911C911397C8CF29960FB6F8940C
:10D0E000DEBF0FBECDBFDF91CF911F910F91FF909B
:10D0F00008952F923F924F925F926F927F928F92FC
:10D100009F92AF92BF92CF92DF92EF92FF920F93D6
:10D110001F93CF93DF93CDB7DEB7E0970FB6F894A8
:10D12000DEBF0FBECDBF8B0169017A0194E0E4E858
:10D13000F3E0DE01119601900D929A95E1F7FE0160
:10D1400035968CE1DF011D928A95E9F794E0E4E8D9
:10D15000F3E0DE01919601900D929A95E1F7FE01C0
:10D16000B5968CE0DF011D928A95E9F7AE014F5F1D
:10D170005F4F68E0C8010E94D9261A8AC701B6012C
:10D180000E94A3831B013F926F9388E795E09F93D2
:10D190008F938E010F5D1F4F1F930F930E9468871F
:10D1A0000F900F900F900F900F900F9020E030E0B5
:10D1B000A901C701B6010E948B8426013701181608
:10D1C00024F077FA709477F87094F80101900020B9
:10D1D000E9F731975F01A01AB10A8EE2808382E2FB
:10D1E000882E912C8C0E9D1E8A0C9B1CB10137FE43
:10D1F00003C0719561957109072E000C880B990B7E
:10D200000E94DB839B01AC01C301B2010E94BF827B
:10D2100020E030E040E251E40E9490840E94A38329
:10D22000605DF4016083FE01EA0DFB1D13A28FE631
:10D2300098E00E94F25E66E073E18FE698E00E945B
:10D24000CF5DB8018FE698E00E94F65E64E073E17E
:10D250008FE698E00E94CF5DBE016F5F7F4F8091A7
:10D260009E0590919F050E946C385C01009709F41F
:10D27000DFC065E874E00E946C38DC0119968D907F
:10D280009C901A97B4018FE698E00E94F65E62E0E7
:10D2900073E18FE698E00E94CF5D8FE698E00E94F0
:10D2A000F25E20E030E04EEF52ECC701B6010E9482
:10D2B0002C83882309F4CDC020E030E04AEA52E410
:10D2C000C701B6010E942C83882309F4C2C020E064
:10D2D00030E0A901C701B6010E942C83882309F41C
:10D2E000B8C081149104A9F020E030E043E050E0A0
:10D2F00060E2CE0101960E94372640E250E0B40180
:10D30000CE0101960E94FE86B801CE0101960E94D0
:10D310006A6566E774E0C5010E946C38FC016185AE
:10D3200072856115710509F494C0DB018C91882325
:10D3300009F48FC08091E90B9091EA0B009709F4F2
:10D3400088C00E946C388C01009709F482C064E0A8
:10D3500070E00E940427882309F47BC0C8010E9462
:10D36000FA3B8430A9F50E94F22E5C01892B19F05A
:10D3700085E0F50180870E94F22E4C01892B49F04F
:10D3800083E0D40118968C93F401C186D286E3869B
:10D39000F4860E94F22E7C01892B69F082E0D7018D
:10D3A00018968C9388EC90E0A0E0B0E0F7018187BC
:10D3B0009287A387B487B401C5010E948738B7015B
:10D3C000C5010E948738B501C8010E94873841C055
:10D3D00064E0C8010E945F384C010097D1F161E020
:10D3E0000E945F385C0160E0C4010E945F38DC018C
:10D3F0001996CD92DD92ED92FC921C97F5018185F4
:10D400009285A385B485892B8A2B8B2B39F4D8017F
:10D410006D917C918DE795E00E946A6588EC90E0C3
:10D42000A0E0B0E0F50181879287A387B48711C09F
:10D43000BE016F5F7F4F8FE698E00E94F65E60E06E
:10D4400073E18FE698E00E94CF5D8FE698E00E943E
:10D45000F25EE0960FB6F894DEBF0FBECDBFDF914F
:10D46000CF911F910F91FF90EF90DF90CF90BF90E1
:10D47000AF909F908F907F906F905F904F903F9074
:10D480002F9008953FB7F8948091F00B9091F10B95
:10D49000A091F20BB091F30B26B5A89B05C02F3FCE
:10D4A00019F00196A11DB11D3FBFBA2FA92F982FCA
:10D4B0008827820F911DA11DB11DBC01CD0142E045
:10D4C000660F771F881F991F4A95D1F7089590E03E
:10D4D000FC013197E231F10508F04EC08827E45194
:10D4E000FF4F8F4F0C948D82809180008F7703C007
:10D4F000809180008F7D80938000089580918000CE
:10D50000877FF9CF84B58F7702C084B58F7D84BDC6
:10D5100008958091B0008F7703C08091B0008F7D17
:10D520008093B0000895809190008F7707C080911C
:10D5300090008F7D03C080919000877F8093900042
:10D5400008958091A0008F7707C08091A0008F7D03
:10D5500003C08091A000877F8093A00008958091F0
:10D5600020018F7707C0809120018F7D03C08091BB
:10D570002001877F809320010895CF93DF9390E06F
:10D58000FC01E65EF34F2491FC01E05AF34F8491D5
:10D59000882361F190E0880F991FFC01E050F44F5F
:10D5A000C591D491FC01E056F44FA591B49161115D
:10D5B00009C09FB7F8948881209582238883EC91D5
:10D5C0002E230BC0623061F49FB7F8948881322F0C
:10D5D000309583238883EC912E2B2C939FBF06C01C
:10D5E0008FB7F894E8812E2B28838FBFDF91CF91DE
:10D5F00008958F929F92AF92BF92CF92DF92EF9257
:10D60000FF926B017C010E94426A4B015C01C114D4
:10D61000D104E104F104F1F00E94426ADC01CB0183
:10D6200088199909AA09BB09883E9340A105B1054B
:10D6300070F321E0C21AD108E108F10888EE880EE3
:10D6400083E0981EA11CB11CC114D104E104F104B3
:10D6500019F7DDCFFF90EF90DF90CF90BF90AF90A4
:10D660009F908F9008952FB7F8946091EC0B709174
:10D67000ED0B8091EE0B9091EF0B2FBF08951F9251
:10D680000F920FB60F9211242F933F938F939F9376
:10D69000AF93BF938091EC0B9091ED0BA091EE0BAB
:10D6A000B091EF0B3091EB0B23E0230F2D3720F4DB
:10D6B0000196A11DB11D05C026E8230F0296A11DEC
:10D6C000B11D2093EB0B8093EC0B9093ED0BA0938B
:10D6D000EE0BB093EF0B8091F00B9091F10BA091BA
:10D6E000F20BB091F30B0196A11DB11D8093F00BCD
:10D6F0009093F10BA093F20BB093F30BBF91AF910A
:10D700009F918F913F912F910F900FBE0F901F907F
:10D710001895CF93DF93CDB7DEB7CE56D1090FB6AC
:10D72000F894DEBF0FBECDBF789484B5826084BD0F
:10D7300084B5816084BD85B5826085BD85B5816015
:10D7400085BD80916E00816080936E001092810093
:10D75000809181008260809381008091810081604E
:10D76000809381008091800081608093800080910F
:10D77000B10084608093B1008091B000816080939B
:10D78000B00080919100826080939100809191001F
:10D7900081608093910080919000816080939000DF
:10D7A0008091A10082608093A1008091A10081609E
:10D7B0008093A1008091A00081608093A00080915F
:10D7C00021018260809321018091210181608093F9
:10D7D00021018091200181608093200180917A0055
:10D7E000846080937A0080917A00826080937A00CE
:10D7F00080917A00816080937A0080917A008068BD
:10D8000080937A001092C1001092DD0510928D0570
:10D8100010928C0526E040E052EC61E070E08FE66B
:10D8200098E00E94DE386EE175E08FE698E00E9495
:10D83000CF5D6FE277E486EB93E00E94E36061E7FF
:10D840007DE48BEB93E00E94E36063E177E480EC9E
:10D8500093E00E94E3606EED70E585EC93E00E943A
:10D86000E36064E87CE489EC93E00E94E3606BE1B0
:10D8700077E48DEC93E00E94E3606FEA7DE482ED53
:10D8800093E00E94E36062EE7CE486ED93E00E9408
:10D89000E36062E57CE489ED93E00E94E3606FE67B
:10D8A0007CE48DED93E00E94E36065E177E483EE34
:10D8B00093E00E94E3600E94222A8E010F5F1F4FB7
:10D8C0007E0127E0E20EF11C54EAC52E53E0D52E6E
:10D8D000180140E150E060E070E0C6010E946A7902
:10D8E000F80161938F016AE370E0C6010E94E3864C
:10D8F000009759F0FC012081222339F06C01FFEFE1
:10D90000CF1ADF0A0E151F0521F74AECE42E47E077
:10D91000F42ED12C00E010E0C8010E94F081F70144
:10D9200081937F0181508E3F10F4DD24D3940F5FEB
:10D930001F4F0630110581F7D1100EC062E275E06D
:10D940008FE698E00E94CF5D86E0F101AAECB7E097
:10D9500001900D928A95E1F70E948D660E94454ED6
:10D9600061E08DE00E94BD6A26E040E855E260E09B
:10D9700070E082ED97E00E94DE3887E19AE29093B2
:10D98000DC0A8093DB0A8CE194E29093DE0A8093B8
:10D99000DD0A88E194E29093E00A8093DF0A64E173
:10D9A00070E080E090E00E94F96AE0919005F091CB
:10D9B0009105309721F086E194E2908B878788EA81
:10D9C00095E69093B8098093B70964EF71E080E021
:10D9D00090E00E94F96A9E01265A3F4FA0963FAF01
:10D9E0002EAFA097A8958FE698E00E94A25C892BA5
:10D9F000F1F18FE698E00E94805C182F8A3029F0C0
:10DA00008D3019F0883009F513C0E091DD05F0E0A4
:10DA1000EF55FA4F10826AEE73E08FE698E00E94AD
:10DA2000F65E81EA95E00E9424611092DD05DBCF6D
:10DA300068E08FE698E00E94C85D8091DD0588234C
:10DA400091F281508093DD05CECF682F8FE698E06C
:10DA50000E94C85DE091DD05EB3328F681E08E0F72
:10DA60008093DD05F0E0EF55FA4F1083BCCF0E94A4
:10DA70005B12029714F00E948E578091A0058823B4
:10DA800009F4ECC180919E0590919F05892B09F4C2
:10DA9000E5C10E94336B0091E0051091E1052091F2
:10DAA000E2053091E305601771078207930708F4D8
:10DAB000D5C10E94336BA4966CAF7DAF8EAF9FAF84
:10DAC000A4978091980590919905009709F4AEC1AB
:10DAD0002091DE053091DF056091960570919705E4
:10DAE000261737070CF49FC00E94336B2B013C01B3
:10DAF00038E8430E33E1531E611C711C62E775E088
:10DB00008FE698E00E944D38E0919005F0919105E4
:10DB1000309751F08FEF83871486DF0113963B9681
:10DB20001D92AE17BF07E1F7E0918E05F0918F05CA
:10DB300020E030E0809196059091970528173907ED
:10DB40000CF044C0808191818E7F819391932F5FEF
:10DB50003F4FF0CF8FEFE81AF80AE814F9040CF001
:10DB600028C748E050E0B501C6010E94A68658E0EB
:10DB7000C50ED11C892B71F7EE0CFF1CE0918E05B0
:10DB8000F0918F05EE0DFF1D808191818160918361
:10DB900080836BE675E08FE698E00E94CF5D809110
:10DBA00096059091970523E0880F991F2A95E1F734
:10DBB0002091940530919505820F931F0E9408557E
:10DBC00064E675E08FE698E00E944D3880919005FC
:10DBD00090919105009709F458C76091960570914E
:10DBE000970533E0660F771F3A95E1F7209194058A
:10DBF00030919505620F731F0E94AA4018160CF011
:10DC000044C7809096059090970544E1841691044E
:10DC10000CF03BC70E94336B6415750586059705AC
:10DC200008F4B0C632C70091940510919505A9017A
:10DC3000E3E0440F551FEA95E1F7040F151FF801C3
:10DC40004081483209F0E7C0A101B8010E94694053
:10DC5000882369F12A8130E0C901982F8827990F1C
:10DC6000990F990F6981F8E06F9FB00111249C0111
:10DC7000262B372BF80180818031E1F4688570E034
:10DC80008F81AB01481B5109CA019695982F8827AF
:10DC9000979587950E94798260517109207F13E0E2
:10DCA000220F331F1A95E1F7620F731F04C060E85B
:10DCB00074EE01C0B901613854EE75077CF0072E8F
:10DCC000000C880B990B0E94DB8320E030E040E0E1
:10DCD0005CE30E9490849B01AC0104C020E030E032
:10DCE0004EEF52ECE0919205F0919305309789F058
:10DCF0008091DE059091DF05BC01A3E0660F771FE0
:10DD0000AA95E1F7A0919405B09195056A0F7B1F44
:10DD10001995E090DE05F090DF0543E0EE0CFF1C66
:10DD20004A95E1F78091940590919505E80EF91ECA
:10DD3000C0909805D0909905F7018081803149F015
:10DD4000B701C6010E947C40182F882309F457C0F0
:10DD500001C01CE0F601858196810E94DE3F882388
:10DD600009F44DC0B701F601858196810E94943F68
:10DD7000F601408164E4858196810E94723FF6013C
:10DD800082818823E1F11950133048F4E12FF0E04B
:10DD9000EE0FFF1FEE5EFD4F0081118102C00EEEFF
:10DDA00012E0E114F10429F1F6018381882309F1DD
:10DDB000808181111EC00E94336B2B013C01480100
:10DDC000110FAA08BB08A101B701C6010E941340A8
:10DDD0008981811114C00E94336BDC01CB01881949
:10DDE0009909AA09BB0984159505A605B70558F335
:10DDF00006C0B801110F880B990B0E94F96A809137
:10DE0000DE059091DF0501969093DF058093DE0596
:10DE100064EC79E00DC02F5F3F4F3093DF05209316
:10DE2000DE0580ED97E00E94798202C06FEF7FEF00
:10DE3000CB01770FAA0BBB0BA4962CAD3DAD4EAD1D
:10DE40005FADA497820F931FA41FB51F8093E005B9
:10DE50009093E105A093E205B093E3050E94CB22E5
:10DE60008091E90B9091EA0B892B09F486C580918A
:10DE70009C0590919D05049709F4C2C30E94336BE1
:10DE80000091E4051091E5052091E6053091E70544
:10DE9000061717072807390708F0B2C320E0E091FA
:10DEA0009A05F0919B05309709F4AAC32111A8C3E4
:10DEB0008085853009F08DC340E853E063965FAFFD
:10DEC0004EAF63976596FFAFEEAF6597CE018F5A61
:10DED0009F4F0E9482210E94336B2B013C016A9666
:10DEE0008FAD6A97843061F008F45BC3883009F421
:10DEF00058C3893009F4D7C0853009F057C351C3DE
:10DF00008091E70B9091E80B892B09F0C4C0CE01FA
:10DF10008F5A9F4F0E94D0638111BDC06796AEACEF
:10DF2000BFAC6797F5018085853009F0C6C5C5018E
:10DF30000E94FA3BC82ED12CF2E0CF16D1040CF48B
:10DF4000BCC521E030E03093E80B2093E70B60E0A4
:10DF500070E0CE018F5A9F4F0E941A214C0161E060
:10DF600070E0CE018F5A9F4F0E941A217C0135E04C
:10DF7000C316D1040CF410C664E0C5010E945F38DA
:10DF8000FC010185128526E240E855E260E070E080
:10DF900082ED97E00E94DE388092C90982ED97E019
:10DFA0009093C8098093C7091092D40A1092D60A98
:10DFB0001092D50A0130110509F4A3C50CF484C5EB
:10DFC0000230110509F08EC5F092CB09E092CA0922
:10DFD00021E030E03093CD092093CC0983E00E940A
:10DFE0004339A7968FAFA797A7969FADA797911193
:10DFF00099C5E091CE09F091CF09A996FFAFEEAF98
:10E00000A997CF01FF0FAA0BBB0B89839A83AB8320
:10E01000BC8320E130E03E832D836596EEADFFADFD
:10E020006597008111816DED75E08FE698E00E94A3
:10E03000CF5DB8018FE698E00E94F65E66ED75E070
:10E040008FE698E00E94CF5DB1018FE698E00E94D4
:10E05000DC210E94F25EA9966EAD7FADA997CE013C
:10E060008F5A9F4F0E940A641092E80B1092E70BA0
:10E0700000919A0510919B05F8018281938120E817
:10E0800033E03A8329839C838B83C1010E948221E0
:10E09000012B09F064C5CE018F5A9F4F0E94CE64B8
:10E0A00080ED97E085C28091E70B9091E80B892B7A
:10E0B00091F7CE018F5A9F4F0E94D0638111EBCF11
:10E0C00041E050E05093E80B4093E70B0E94F22EA2
:10E0D0006C01892B19F086E0F601808720E030E0A2
:10E0E00043E050E060E2C1010E9437266596EEAD44
:10E0F000FFAD6597608171814FE150E0C1010E94E1
:10E10000FE866DEE73E0C1010E94D88626E040E8ED
:10E1100055E260E070E082ED97E00E94DE3860E05A
:10E1200070E0CE018F5A9F4F0E941A218093C90937
:10E1300082ED97E09093C8098093C7091092D40AA2
:10E140001092D60A1092D50A24E338E03093CB0916
:10E150002093CA094AE050E05093CD094093CC097E
:10E1600083E00E9443398111BEC066EB75E08FE603
:10E1700098E00E94CF5D0EEC19E0F8018191919139
:10E180008F01092E000CAA0BBB0B25968CAF9DAFFF
:10E19000AEAFBFAF259720E130E027963FAF2EAF5F
:10E1A0002797BE016F5B7F4F8FE698E00E94DC21CE
:10E1B00064EB75E00E94CF5D39E0023E1307E9F69B
:10E1C0008FE698E00E94F25E6091D2097091D309C7
:10E1D000072E000C880B990B0E94DB8320E030E0B7
:10E1E00048EC52E40E9431839B01AC0163EF73E081
:10E1F000C6010E942D650091D6091091D709A8018A
:10E2000065EF73E0C6010E94A4386091D80970914F
:10E21000D909072E000C880B990B0E94DB8320E0A4
:10E2200030E048EC52E40E9431839B01AC0169EF7D
:10E2300073E0C6010E942D656091DA097091DB09D7
:10E24000072E000C880B990B0E94DB8320E030E046
:10E2500040E251E40E9431839B01AC0167EF73E01F
:10E26000C6010E942D654091CE095091CF096BEFF8
:10E2700073E0C6010E94A438012B09F452C06796CE
:10E280008EAD9FAD6797FC012085253009F049C010
:10E2900061E00E945F38009709F443C024E630E053
:10E2A0006E963FAF2EAF6E97FC0161857285CE01F1
:10E2B0008F5B9F4F0E94AE61CE018F5B9F4F0E948C
:10E2C000B120882371F1E12CF12C01E09E01245A48
:10E2D0003F4F41E050E060E070E0CE018F5B9F4F28
:10E2E0000E94B9091EC090E0A0E0B0E025968CAF76
:10E2F0009DAFAEAFBFAF259720E130E027963FAF8F
:10E300002EAF27976EE975E08FE698E00E94CF5D0B
:10E31000BE016F5B7F4F8FE698E00E94DC210E9478
:10E32000F25E8091CE0983FF16C08EE398E0909351
:10E33000CB098093CA0941E050E05093CD09409346
:10E34000CC0983E00E94433981110CC04091CE0971
:10E350005091CF0902C040E050E06EEF73E0C6017B
:10E360000E94A43862E370E080E090E00E94F96AC5
:10E3700083E190E09093CB098093CA09E4E0F0E058
:10E38000F093CD09E093CC0983E00E9443398111D9
:10E39000AAC064E975E08FE698E00E94CF5D2EEC9C
:10E3A000E22E29E0F22E06ED19E0F701619171915C
:10E3B0007F014AE050E08FE698E00E94995E62E9B2
:10E3C00075E08FE698E00E94CF5D0E151F0569F796
:10E3D0008FE698E00E94F25E0091CE091091CF097D
:10E3E00001151105D1F0B801012E000C880B990B15
:10E3F0000E94DB832DEE3EE94CE35EE30E949084B5
:10E4000022E538EB42E152E40E94BF829B01AC015D
:10E4100062E074E0C6010E942D656091D0097091A0
:10E42000D109072E000C880B990B0E94DB832DEE7F
:10E430003EE94CE35EE30E94908422E538EB42E142
:10E4400052E40E94BF824B015C019B01AC0161EF71
:10E4500073E0C6010E942D656091D4097091D509C1
:10E4600016161706A4F4072E000C880B990B0E94B1
:10E47000DB8320E030E040E251E40E9431839B01E5
:10E48000AC0166E074E0C6010E942D6507C040E063
:10E4900050E066E074E0C6010E94A43820E030E05D
:10E4A00040E252E4C501B4010E948B841816BCF509
:10E4B000012BA9F16596EEADFFAD65976081718185
:10E4C0008AE094E00E946A65E12CF12C01E020E0F2
:10E4D00030E040E050E062E070E0CE018F5A9F4FA4
:10E4E0000E94B9091CC090E0A0E0B0E025968CAF76
:10E4F0009DAFAEAFBFAF259720E130E027963FAF8D
:10E500002EAF27976CE775E08FE698E00E94CF5D0D
:10E51000BE016F5B7F4F8FE698E00E94DC2180E0B8
:10E5200091E00E94A7778C01892B61F125961FAE9F
:10E530001EAE259727961FAE1EAE27974FEF5FEFB3
:10E5400029965FAF4EAF29978CE192E023969FAF5B
:10E550008EAF23972B961FAE1EAE2B972D961FAF17
:10E560000EAF2D9780E091E061969FAF8EAF6197DF
:10E570002F961FAE1EAE2F97B601CE018F5B9F4F19
:10E580000E94FB2CB801C1010E946A65C8010E946B
:10E590003F78C6010E9475651092E80B1092E70B58
:10E5A0007ACDCE018F5A9F4F0E94CE6484E690E0D0
:10E5B000092E000CAA0BBB0B480E591E6A1E7B1EAF
:10E5C0004092E4055092E5056092E6057092E705F9
:10E5D00021E0E0919A05F0919B05828193819093CF
:10E5E0009B0580939A05892B09F059CCE091E90BA2
:10E5F000F091EA0B8681978190939B0580939A0511
:10E600000E94336B0091E8051091E9052091EA051D
:10E610003091EB05601771078207930708F4ADC1CD
:10E62000E091E90BF091EA0B309709F4A6C1C6809E
:10E63000D78010E0C114D10409F4D8C065E070E0BF
:10E64000C6010E940427882309F4CCC064E0C601F7
:10E650000E945F387C01009709F4C4C00E94FA3B15
:10E66000823008F4BFC061E0C6010E945F38FC013F
:10E670001185028562E0C6010E945F38FC01418479
:10E6800052846384748463E0C6010E945F38FC0195
:10E690002185328543855485AD962CAF3DAF4EAF75
:10E6A0005FAFAD9760E0C7010E945F38FC018184D5
:10E6B0009284A384B48461E0C7010E945F38FC01A6
:10E6C0004185528563857485411551056105710544
:10E6D00009F084C2F601608171818FE698E00E94A2
:10E6E000F65E6EE576E08FE698E00E94CF5D20E072
:10E6F00030E048E152E4C501B4010E948B84181651
:10E700003CF4F601608171818AE094E00E946A65C0
:10E71000A1961FAFA197A2960FAFA297C301B20116
:10E720000E94DB832B013C01AB962EAD3FADAB9736
:10E73000A6963FAF2EAFA697F6010190F081E02D8F
:10E74000AF96FFAFEEAFAF978FE698E00E94F25E14
:10E75000AF966EAD7FADAF978FE698E00E94F65E04
:10E7600068E576E08FE698E00E94CF5D42E0C30165
:10E77000B2010E94835562E576E08FE698E00E9440
:10E78000CF5D42E0C501B4010E9483556CE476E0A0
:10E790008FE698E00E94CF5D4AE050E0AB966EAD08
:10E7A0007FADAB978FE698E00E94995EA2962EAD62
:10E7B0003FADA29761E0812F37FD26C20E94BD6A5E
:10E7C000A6968EAD9FADA697029709F029C260E08C
:10E7D000812F0E946E3667E476E08FE698E00E9413
:10E7E000CF5D11E0F601C280D38024CF0E94336B4D
:10E7F000DC01CB0188579C4EAF4FBF4F8093E8059B
:10E800009093E905A093EA05B093EB05E090F60B31
:10E81000F090F70BE114F10421F492E0E92E9CE072
:10E82000F92E0E94336B4B015C010E943C638823EC
:10E8300009F460C020E030E041E050E060E4C10154
:10E840000E94372640E450E06DE176E0C1010E946D
:10E85000A77A63E274E0C1010E94D88640E450E0E8
:10E8600064E176E0C1010E94A77AA0964EAD5FAD4B
:10E87000A0974E195F09052E000C660B770BCE0191
:10E880008F5B9F4F0E94DC25BE016F5B7F4FC101F4
:10E890000E94C56320E030E041E050E060E4C10147
:10E8A0000E94372640E450E06DE176E0C1010E940D
:10E8B000A77A63E274E0C1010E94D88640E450E088
:10E8C0006DE076E0C1010E94A77AC501B40128EE8F
:10E8D00033E040E050E00E941682BA01A901CE0167
:10E8E0008F5B9F4F0E94DC25BE016F5B7F4FC10194
:10E8F0000E94C5638091F60B9091F70B1123F9F0FC
:10E90000009711F08C0102C002E01CE068E276E0A2
:10E910008FE698E00E94CF5DA101401B510B052EB0
:10E92000000C660B770B2AE08FE698E00E94085EE9
:10E9300065E274E08FE698E00E94F65E1EC00097E4
:10E9400011F08C0102C002E01CE066E276E08FE686
:10E9500098E00E94CF5DA101401B510B052E000CD9
:10E96000660B770B2AE08FE698E00E94085E64E26F
:10E9700076E08FE698E00E94CF5D0E9429270E94F2
:10E98000535D30C8C0909405D0909505540183E044
:10E99000AA0CBB1C8A95E1F7AC0CBD1C67E0C50155
:10E9A0000E94213FF5019781891310C9E12CF12CB8
:10E9B000D4C88091980590919905892B09F406C9CE
:10E9C000E0919605F0919705EE0FFF1F80918E055F
:10E9D00090918F05E80FF91F21E030E0318320830B
:10E9E000E0909605F09097056FE575E08FE698E06A
:10E9F0000E94CF5D4AE050E0B7018FE698E00E94A8
:10EA0000995E68E575E08FE698E00E94CF5D8091A1
:10EA1000960590919705B3E0880F991FBA95E1F795
:10EA20002091940530919505820F931F0E940855FF
:10EA30008FE698E00E94F25E6091960570919705CE
:10EA400013E0660F771F1A95E1F780919405909176
:10EA50009505680F791FFB018081883261F48091F0
:10EA60009805909199050E94865480919005909107
:10EA700091050E949E24809196059091970501969C
:10EA80009093970580939605A1C8009196051091E3
:10EA9000970569E475E08FE698E00E94CF5D4AE053
:10EAA00050E0B8018FE698E00E94995E1092DF0571
:10EAB0001092DE0560E47FE1BBC96AEF75E08FE686
:10EAC00098E00E94CF5DE7CA012B29F5F092CB09AF
:10EAD000E092CA0941E050E05093CD094093CC093F
:10EAE00081E07DCA03301105B1F4F092CB09E092C8
:10EAF000CA0981E090E09093CD098093CC0984E02D
:10EB00006ECAF092CB09E092CA091093CD09009326
:10EB1000CC0982E064CA62EE75E08FE698E00E945C
:10EB2000CF5D62CAA7963FADA797832F90E0A0E084
:10EB3000B0E089839A83AB83BC8340E150E05E837D
:10EB40004D8360EC75E08FE698E00E94CF5DB101E7
:10EB50008FE698E00E94DC210E94F25E85CAC10126
:10EB60000E94B120882309F496CA8985843009F06F
:10EB700092CA60E070E0C1010E941A2188169906CD
:10EB800009F089CA61E070E0C1010E941A21E8160B
:10EB9000F90609F080CA03C002E010E0F4C9A996A2
:10EBA0006EAD7FADA997C1010E940A64E0919A05FC
:10EBB000F0919B058281938190939B0580939A05A8
:10EBC000892B09F068CAE091E90BF091EA0B868184
:10EBD000978190939B0580939A055DCA4150510996
:10EBE00061097109FC014187528763877487452B4E
:10EBF000462B472B09F07BCDF6016081718187E1BF
:10EC000094E00E946A6573CD81950E94BD6AA696C4
:10EC10004EAD5FADA6974230510509F061C01BC0F3
:10EC2000A6964EAD5FADA6974530510509F4CFCD00
:10EC300061E0C7010E945F38FC0181859285A38550
:10EC4000B485892B8A2B8B2B61F4A2962EAD3FAD18
:10EC5000A29737FFBCCD60E0812F81950E946E3670
:10EC6000B6CD20E030E040E85FE3C301B2010E948E
:10EC7000BF829B01AC01C501B4010E942C8387FFB8
:10EC800012C0A2962EAD3FADA29737FF05C060E03F
:10EC9000812F81950E946E3661E0812F0E946E3631
:10ECA00063E476E09ACDA5019401C301B2010E940C
:10ECB0002C83181694F0A2964EAD5FADA29757FF25
:10ECC00005C061E0812F81950E946E3660E0812F42
:10ECD0000E946E366EE376E080CD6FE276E07DCD09
:10ECE000A6968EAD9FADA697059709F0A1CFB3CF9D
:10ECF000E2EDF7E01382128248EE53E060E070E04C
:10ED0000448355836683778388E892E09183808388
:10ED100025ED30E03587248724ED30E037872687DE
:10ED200020ED30E0318B208B21ED30E0338B228BD6
:10ED300022ED30E0358B248B26ED30E0378B268BAF
:10ED4000118E128E138E148EEFE6F8E0138212826B
:10ED500044835583668377839183808385EC90E039
:10ED60009587848784EC90E09787868780EC90E095
:10ED7000918B808B81EC90E0938B828B82EC90E086
:10ED8000958B848B86EC90E0978B868B118E128E00
:10ED9000138E148EEEEEFAE08AE193E09183808385
:10EDA0001282138214821582E4EFFAE09183808349
:10EDB0001282138214821582EAEFFAE09183808333
:10EDC0001282138214821582ECE0F9E09183808331
:10EDD0001282138214821582E0E0FBE0918380832B
:10EDE0001282138214821582E6E0FBE09183808315
:10EDF0001282138214821582ECE0FBE091838083FF
:10EE00001282138214821582E2E1FBE091838083F7
:10EE10001282138214821582E2E1F9E091838083E9
:10EE20001282138214821582EAE1F9E013821282BF
:10EE300044835583668377832AE932E031832083D4
:10EE4000E8E1FBE0918380831282138214821582B1
:10EE5000EEE1FBE09183808312821382148215829B
:10EE6000E4E2FBE091838083128213821482158294
:10EE7000E1EEFAE01382128244835583668377833E
:10EE800024EF32E03183208324E024871092DC0ACF
:10EE90001092DB0A1092DE0A1092DD0A1092E00A4C
:10EEA0001092DF0AA6E2B9E013961C921E92129706
:10EEB0002CEA32E011963C932E939093BA098093FA
:10EEC000B9091092BB091092BC091092BD091092A9
:10EED000BE092FEF3FEF3093C6092093C509159661
:10EEE000FC93EE9314971092C4091092C309EAE2BE
:10EEF000FBE0918380831282138214821582E0E307
:10EF0000FBE0918380831282138214821582E6E3F0
:10EF1000FBE0918380831282138214821582ECE3DA
:10EF2000FBE0918380831282138214821582E2E4D3
:10EF3000FBE08FEF808312821182148613868FEF9D
:10EF40009FEFDC0187839087A187B28708950F9395
:10EF50001F93CF93DF938230910510F482E090E00D
:10EF6000E091F80BF091F90B20E030E0A0E0B0E088
:10EF7000309719F140815181028113814817590757
:10EF8000C8F08417950769F4109731F012960C9326
:10EF9000129713961C9327C00093F80B1093F90B4C
:10EFA00022C02115310519F04217530718F49A01B0
:10EFB000BD01EF01DF01F801DBCF21153105F9F0CB
:10EFC000281B390B2430310580F48A819B8161151F
:10EFD000710521F0FB019383828304C09093F90BA8
:10EFE0008093F80BFE01329644C0FE01E20FF31F3E
:10EFF0008193919322503109398328833AC020911B
:10F00000F60B3091F70B232B41F420910A0230913B
:10F010000B023093F70B2093F60B209108023091EE
:10F0200009022115310541F42DB73EB740910C027C
:10F0300050910D02241B350BE091F60BF091F70B6C
:10F04000E217F307A0F42E1B3F0B2817390778F0BF
:10F05000AC014E5F5F4F2417350748F04E0F5F1F1E
:10F060005093F70B4093F60B8193919302C0E0E02D
:10F07000F0E0CF01DF91CF911F910F910895CF93D1
:10F08000DF93009709F481C0FC013297138212824A
:10F09000A091F80BB091F90B109781F42081318188
:10F0A000820F931F2091F60B3091F70B2817390729
:10F0B00051F5F093F70BE093F60B67C0ED0120E0FC
:10F0C00030E0CE17DF0740F44A815B819E01411595
:10F0D0005105F1F0EA01F5CFD383C283408151811C
:10F0E000840F951FC817D90759F488819981840F17
:10F0F000951F0296918380838A819B81938382836B
:10F100002115310529F4F093F90BE093F80B3DC07C
:10F11000E901FB83EA8349915991C40FD51FEC178C
:10F12000FD0761F480819181840F951F0296E901AA
:10F1300099838883828193819B838A83E0E0F0E0D6
:10F1400012968D919C911397009719F0FD01DC01A7
:10F15000F7CF8D919C9111979D012E5F3F4F820FAC
:10F16000931F2091F60B3091F70B2817390769F49C
:10F17000309729F41092F90B1092F80B02C0138209
:10F180001282B093F70BA093F60BDF91CF91089505
:10F190008F929F92AF92BF92CF92DF92EF92FF92A7
:10F1A000CF93DF93EC01688179818A819B8161151E
:10F1B00071058105910521F464E279ED8BE597E015
:10F1C0002DE133EF41E050E00E94388249015A01BD
:10F1D0009B01AC01A7EAB1E40E9457826B017C015C
:10F1E000ACEEB4EFA50194010E946582DC01CB0175
:10F1F0008C0D9D1DAE1DBF1DB7FF03C00197A1095A
:10F20000B04888839983AA83BB83BC01CD019F77D3
:10F21000DF91CF91FF90EF90DF90CF90BF90AF90B4
:10F220009F908F9008958F929F92AF92BF92CF92AE
:10F23000DF92EF92FF9260910E0270910F02809127
:10F24000100290911102611571058105910521F45B
:10F2500064E279ED8BE597E02DE133EF41E050E09A
:10F260000E94388249015A019B01AC01A7EAB1E42E
:10F270000E9457826B017C01ACEEB4EFA5019401B2
:10F280000E946582DC01CB018C0D9D1DAE1DBF1D52
:10F29000B7FF03C00197A109B04880930E02909375
:10F2A0000F02A0931002B0931102BC01CD019F7711
:10F2B000FF90EF90DF90CF90BF90AF909F908F9096
:10F2C000089560930E0270930F0280931002909342
:10F2D000110208953F924F925F926F927F928F92A8
:10F2E0009F92AF92BF92CF92DF92EF92FF920F93D5
:10F2F0001F93CF93DF935C016B017A016115710558
:10F3000019F0FB0191838083E114F10429F0C70116
:10F310000297839708F0C9C0E5012196F501108195
:10F32000812F90E00E94957A892B11F05E01F4CF35
:10F330001D3229F42196F501118101E007C01B322D
:10F3400021F4E5012296F501118100E0E114F104B8
:10F35000B1F0F0E1EF16F10429F4B0C010E3E114CC
:10F36000F10401F12AE0E216F104B1F180E1E816BE
:10F37000F10471F0E8E0EE16F104F1F413C010337B
:10F3800041F588818F7D883549F719812296026081
:10F39000F0E1EF2EF12C88248A94982CA82CAFE071
:10F3A000BA2E20C078E0E72EF12C88248A94982C7D
:10F3B000A82CEFE1BE2E16C06FEF7FEFCB019701B7
:10F3C0000F2C000C440B550B0E94168249015A0168
:10F3D00009C08AE0E82EF12C69E9862E982CA82C29
:10F3E00069E1B62E40E060E070E0CB0127010F2C10
:10F3F000000C66087708FE0150ED352E310E29E02D
:10F40000231570F42FEB210F2A3118F439EC332E29
:10F4100006C02FE9210F2A3130F529EA322E310EAC
:10F42000232D30E02E153F05F4F44F3FC9F086162A
:10F430009706A806B90688F0A30192010E940682E9
:10F44000232D30E040E050E0620F731F841F951FB2
:10F45000621773078407950710F44FEF01C041E06E
:10F4600021961081C8CFC114D10451F0442311F06A
:10F47000219703C001FF04C02297F601D183C08306
:10F4800000FF07C090958095709561957F4F8F4FD5
:10F490009F4F4F3F79F482E290E09093010C80936C
:10F4A000000C3FEF2FEF9FEF0DC040E030E020E079
:10F4B00090E008C0462F372F282F04C0103309F0E2
:10F4C00067CF5FCF642F732F822FDF91CF911F9172
:10F4D0000F91FF90EF90DF90CF90BF90AF909F90F3
:10F4E0008F907F906F905F904F903F900895FC01B8
:10F4F00088279927E89421912032E9F3293010F0E8
:10F500002E30C8F32B3241F02D3239F4689404C008
:10F510000E94FC7A820F911D219120532A30C0F362
:10F520001EF4909581959F4F089591110C9402813E
:10F53000803219F089508550C8F70895FB01DC012D
:10F540008D91059080190110D9F3990B0895FB0155
:10F55000DC010D900020E9F711974150504028F050
:10F56000059000200D92C9F708951C920895FB01A3
:10F57000DC014150504048F005900D920020C9F741
:10F5800001C01D9241505040E0F7089544EF5BE008
:10F590000C94CA7AFA01A191B081009719F41097DE
:10F5A000E1F0CD01DC01CD010D90002011F4C0018E
:10F5B00013C0FB012191222319F02015D9F7F3CFB5
:10F5C000FB012191201519F41E92119606C02223E9
:10F5D000C1F70D900020A1F7D001FA01A193B083EB
:10F5E0000895BB274A3031F4992322F4BDE2909567
:10F5F00081959F4F0C94057B7AE0979F902D879F74
:10F60000802D910D11240895BB27FB015527AA27B2
:10F61000880F991FAA1FA41710F0A41B839550519F
:10F62000B9F7A05DAA3308F0A95DA193009779F717
:10F63000B111B1931192CB010C942D81FC01238166
:10F6400027FF10C0EAEFFBE020813181821793078A
:10F6500011F41182108232962CE0E030F207A1F70B
:10F660000E943F7880E090E008950F931F93CF931E
:10F67000DF93009731F46115710519F480E090E093
:10F680003AC08B01EC016EE070E081E090E00E94F6
:10F69000E680FC01892B91F380E883830115110535
:10F6A00071F01387028781E883838091FA0B909130
:10F6B000FB0B892B21F4F093FB0BE093FA0B2097C3
:10F6C000C9F0D187C0878381826083838091FC0BDE
:10F6D0009091FD0B892B71F4F093FD0BE093FC0BE3
:10F6E0008091FE0B9091FF0B892B21F4F093FF0B7F
:10F6F000E093FE0BCF01DF91CF911F910F91089501
:10F70000CF93DF93EC012B8120FF33C026FF0AC08B
:10F710002F7B2B838E819F8101969F838E838A818D
:10F7200090E029C022FF0FC0E881F9818081082E76
:10F73000000C990B009719F420622B831AC03196A4
:10F74000F983E8830EC0EA85FB85199597FF09C008
:10F750002B81019611F080E201C080E1822B8B8326
:10F7600008C02E813F812F5F3F4F3F832E83992713
:10F7700002C08FEF9FEFDF91CF9108950F931F93FA
:10F78000CF93DF93CDB7DEB708851985F801838164
:10F7900088608383AE01445F5F4F6A857B85C801C3
:10F7A0000E94F87BF8012381277F2383DF91CF918B
:10F7B0001F910F9108950F931F93CF93DF93CDB7B0
:10F7C000DEB708851985F801838188608383AE01DF
:10F7D000445F5F4F6A857B85C8010E94C17FF80145
:10F7E0002381277F2383DF91CF911F910F9108956C
:10F7F0002F923F924F925F926F927F928F929F9241
:10F80000AF92BF92CF92DF92EF92FF920F931F932E
:10F81000CF93DF93CDB7DEB72B970FB6F894DEBF4B
:10F820000FBECDBF6C017B018A01FC0117821682DD
:10F83000838181FFCCC1CE0101963C01F601938109
:10F84000F70193FD859193FF81917F01882309F44E
:10F85000BAC1853239F493FD859193FF81917F017F
:10F86000853229F4B60190E00E943D81E7CF912CCA
:10F87000212C312CFFE1F315D8F08B3279F038F4DC
:10F88000803279F08332A1F4232D20611DC08D32A6
:10F8900061F0803369F4232D216016C0832D8260CE
:10F8A000382EE32DE4603E2E2AC0F32DF8601DC0F3
:10F8B00037FC2DC020ED280F2A3040F08E32B9F4ED
:10F8C00036FC81C1232D2064322E19C036FE06C0BD
:10F8D0008AE0989E200D1124922E11C0EAE02E9EFF
:10F8E000200D1124222EF32DF0623F2E08C08C36FD
:10F8F00021F4832D8068382E02C0883641F4F70148
:10F9000093FD859193FF81917F018111B3CF982F52
:10F910009F7D9554933028F40C5F1F4F9FE399838C
:10F920000DC0833631F0833771F0833509F059C04B
:10F9300021C0F801808189830E5F1F4F8824839442
:10F94000912C530113C02801F2E04F0E511CF80115
:10F95000A080B18036FE03C0692D70E002C06FEF59
:10F960007FEFC5010E9422814C018201F32DFF77B8
:10F970003F2E16C0280122E0420E511CF801A08043
:10F98000B18036FE03C0692D70E002C06FEF7FEFDB
:10F99000C5010E9410814C01F32DF0683F2E8201B9
:10F9A00033FC1BC0822D90E088169906B0F4B60196
:10F9B00080E290E00E943D812A94F4CFF50137FC6B
:10F9C000859137FE81915F01B60190E00E943D81F3
:10F9D00021102A9421E0821A91088114910471F770
:10F9E000E8C0843611F0893641F5F80137FE07C0CA
:10F9F00060817181828193810C5F1F4F08C060819B
:10FA00007181072E000C880B990B0E5F1F4FF32D91
:10FA1000FF763F2E97FF09C0909580957095619570
:10FA20007F4F8F4F9F4FF0683F2E2AE030E0A301B9
:10FA30000E949281882E861845C0853731F4232D87
:10FA40002F7EB22E2AE030E025C0932D997FB92E6B
:10FA50008F36C1F018F4883579F0B5C0803719F0C9
:10FA6000883721F0B0C0E92FE061BE2EB4FE0DC092
:10FA7000FB2DF460BF2E09C034FE0AC0292F26607A
:10FA8000B22E06C028E030E005C020E130E002C020
:10FA900020E132E0F801B7FE07C060817181828108
:10FAA00093810C5F1F4F06C06081718180E090E000
:10FAB0000E5F1F4FA3010E949281882E8618FB2D96
:10FAC000FF773F2E36FE0DC0232D2E7FA22E8914E8
:10FAD00058F434FE0BC032FC09C0832D8E7EA82E54
:10FAE00005C0B82CA32C03C0B82C01C0B92CA4FEAF
:10FAF0000FC0FE01E80DF11D8081803321F49A2DA5
:10FB0000997EA92E09C0A2FE06C0B394B39404C086
:10FB10008A2D867809F0B394A3FC11C0A0FE06C01C
:10FB2000B21488F4280C922C9B180EC0B21460F406
:10FB3000B60180E290E00E943D81B394F7CFB21409
:10FB400018F42B1802C0982C212CA4FE10C0B6016A
:10FB500080E390E00E943D81A2FE17C0A1FC03C09B
:10FB600088E790E002C088E590E0B6010CC08A2DDD
:10FB7000867859F0A1FE02C08BE201C080E2A7FCAA
:10FB80008DE2B60190E00E943D81891438F4B601FF
:10FB900080E390E00E943D819A94F7CF8A94F3012C
:10FBA000E80DF11D8081B60190E00E943D81811039
:10FBB000F5CF222009F442CEB60180E290E00E9407
:10FBC0003D812A94F6CFF6018681978102C08FEF9E
:10FBD0009FEF2B960FB6F894DEBF0FBECDBFDF911F
:10FBE000CF911F910F91FF90EF90DF90CF90BF903A
:10FBF000AF909F908F907F906F905F904F903F90CD
:10FC00002F90089520FD09C0FC0123FD05C022FFAF
:10FC100002C07383628351834083089544FD17C0FB
:10FC200046FD17C0AB01BC01DA01FB01AA0FBB1FE7
:10FC3000EE1FFF1F1094D1F74A0F5B1F6E1F7F1F2F
:10FC4000CB01BA01660F771F881F991F09C033E0E7
:10FC500001C034E0660F771F881F991F3150D1F71C
:10FC6000620F711D811D911D08950F931F93CF93F6
:10FC7000DF938C01C8010E94807BEC0197FD08C0D6
:10FC80000E94957A892BB1F7B801CE010E94798143
:10FC9000CE01DF91CF911F910F9108958F929F9286
:10FCA000AF92BF92EF92FF920F931F93CF93DF9388
:10FCB0008C01D62F7A01B22E0E94807B9C013327C3
:10FCC0002B32310531F02D32310561F48B2D8068F6
:10FCD000B82ED15011F480E068C0C8010E94807B2A
:10FCE00097FDF9CFCB2DCD7F2B2D207309F58033D8
:10FCF000F9F4AA24AA94AD0E09F443C0C8010E94E5
:10FD0000807B97FD3EC09C012F7D33272835310530
:10FD100049F4C264D250A9F1C8010E94807B97FFC8
:10FD200007C02FC0B6FE02C0C26001C0C261DA2D9A
:10FD3000812C912C540120ED280F283080F0C4FF35
:10FD400004C0B8010E94798119C02A3040F0C6FF72
:10FD5000F8CF2F7D3FEE320F363098F727504C2FDB
:10FD6000C501B4010E940E7E4B015C01C260D150FE
:10FD700059F0C8010E94807B97FFDDCFC1FD04C010
:10FD8000AACF812C912C5401C7FF08C0B094A09435
:10FD900090948094811C911CA11CB11C2C2FB50146
:10FDA000A401C7010E94027E81E0DF91CF911F91E3
:10FDB0000F91FF90EF90BF90AF909F908F9008951C
:10FDC0005F926F927F928F929F92AF92BF92CF92EB
:10FDD000DF92EF92FF920F931F93CF93DF93CDB7F4
:10FDE000DEB7A0970FB6F894DEBF0FBECDBF5C01A3
:10FDF000962E7A01F9018E010F5F1F4F680180E294
:10FE0000D8011D928A95E9F7D50113968C9080E070
:10FE100090E0612C712C30E061E070E083FC259172
:10FE200083FE21918F01522E211103C080E090E0CA
:10FE300092C02E3511F4009751F1432F50E048172E
:10FE400059073CF42D3559F12D3219F4772009F179
:10FE500003C0772009F46AC0452D4695469546951E
:10FE6000D601A40FB11D452D47708B0102C0000FB4
:10FE7000111F4A95E2F7A8015C91452B4C9365143C
:10FE800059F0561410F45394E7CF5A94E5CF31E06B
:10FE900004C07724739401C0712C0196BFCF7720E2
:10FEA00019F08E8180628E83311103C0882483947F
:10FEB00017C0F6019E012F5D3F4F80818095819391
:10FEC0002E173F07D1F7F2CFE114F10429F0D70143
:10FED0008C93F70131967F019A94812C9920F9F047
:10FEE000C5010E94807B97FD18C0FC01FF2723E01D
:10FEF000F595E7952A95E1F7EC0DFD1D208130E0A1
:10FF0000AC014770552702C0359527954A95E2F711
:10FF100020FDDACFB5010E947981811087CFE114ED
:10FF2000F10411F0D7011C92C80115C0422F46956B
:10FF300046954695D601A40FB11D422F47708B01FF
:10FF400002C0000F111F4A95E2F7A8015C91452BF2
:10FF50004C93622EA2CFA0960FB6F894DEBF0FBED0
:10FF6000CDBFDF91CF911F910F91FF90EF90DF9068
:10FF7000CF90BF90AF909F908F907F906F905F9049
:10FF800008955F926F927F928F929F92AF92BF92ED
:10FF9000CF92DF92EF92FF920F931F93CF93DF9355
:10FFA0006C01EB015A01FC0117821682512CF601FB
:10FFB000E380FE01E3FC8591E3FE8191182FEF01C0
:10FFC000882309F4EEC090E00E94957A892B21F0F5
:10FFD000C6010E94357EEBCF153241F4FE01E3FCF1
:10FFE0001591E3FE1191EF01153281F4C6010E94D3
:10FFF000807B97FDD4C0412F50E09C01332724170C
:020000021000EC
:100000003507A9F2B6010E947981CBC01A3239F4C2
:10001000E3FC1591E3FE1191EF0101E001C000E066
:10002000F12C20ED210F2A3080F402606F2D70E05A
:1000300080E090E040E20E940E7EF62EFE01E3FC9E
:100040001591E3FE1191EF01ECCF01FF03C0F11018
:1000500003C0A7C0FF24FA94183619F01C3651F0DB
:1000600010C0FE01E3FC1591E3FE1191EF0118367B
:1000700041F408600460FE01E3FC1591E3FE119178
:10008000EF01112309F48DC0612F70E082E195E04A
:100090000E940581892B09F484C000FD07C0F50189
:1000A00080809180C50102965C0102C0812C912C58
:1000B0001E3651F4F6014681578160E070E0202F32
:1000C000C4010E94027E73CF1336A9F401FD02C061
:1000D000FF24F394C6010E94807B97FD60C08114C9
:1000E000910429F0F4018083C40101964C01FA9433
:1000F000F110F0CF50C01B3559F49E01A4016F2DB3
:10010000C6010E94E07EEC01892B09F044C03EC08C
:10011000C6010E94357E97FD42C01F3661F128F46A
:10012000143639F1193651F128C0133771F01537EB
:1001300001F123C08114910429F0F4016082C4010B
:1001400001964C01FA94FF2071F0C6010E94807B59
:100150003C0197FD08C00E94957A892B59F3B6019E
:10016000C3010E94798181149104A9F0F4011082E5
:1001700012C0006203C0006101C00064202FA4010E
:100180006F2DC6010E944E7E811105C0F60183814C
:10019000807329F406C000FD0ACF539408CF552080
:1001A00019F0852D90E002C08FEF9FEFDF91CF9186
:1001B0001F910F91FF90EF90DF90CF90BF90AF9085
:1001C0009F908F907F906F905F9008950F931F93F3
:1001D000CF93DF93869F8001879F100D969F100D10
:1001E0001124C8010E94A777EC01009729F0A8010B
:1001F00060E070E00E941B81CE01DF91CF911F91E2
:100200000F910895992788270895FC0105900616F7
:1002100021F00020D9F7C00108953197CF0108954A
:10022000FC010590615070400110D8F780959095C1
:100230008E0F9F1F0895DC0101C06D934150504007
:10024000E0F70895FC016150704001900110D8F76B
:10025000809590958E0F9F1F0895DC01FC01672FFC
:1002600071917723E1F7329704C07C916D9370838D
:100270006291AE17BF07C8F308950F931F93CF93F2
:10028000DF93FB01238121FD03C08FEF9FEF2CC083
:1002900022FF16C0468157812481358142175307BA
:1002A00044F4A081B1819D012F5F3F4F31832083B2
:1002B0008C93268137812F5F3F4F3783268314C06D
:1002C0008B01EC01FB010084F185E02D1995892B50
:1002D000E1F6D80116968D919C9117970196179685
:1002E0009C938E931697CE01DF91CF911F910F9122
:1002F0000895FB01238120FF12C026FD10C08F3F0F
:100300003FEF930761F082832F7D20642383268152
:1003100037812150310937832683992708958FEF3C
:100320009FEF0895FA01AA27283051F1203181F179
:10033000E8946F936E7F6E5F7F4F8F4F9F4FAF4FED
:10034000B1E03ED0B4E03CD0670F781F891F9A1F00
:10035000A11D680F791F8A1F911DA11D6A0F711DB4
:10036000811D911DA11D20D009F468943F912AE0C0
:10037000269F11243019305D3193DEF6CF010895A8
:10038000462F4770405D4193B3E00FD0C9F7F6CFD9
:10039000462F4F70405D4A3318F0495D31FD4052A1
:1003A000419302D0A9F7EACFB4E0A6959795879537
:1003B00077956795BA95C9F7009761057105089516
:1003C0009B01AC010A2E06945795479537952795C2
:1003D000BA95C9F7620F731F841F951FA01D08955A
:1003E000F999FECF92BD81BDF89A992780B50895FD
:1003F000262FF999FECF1FBA92BD81BD20BD0FB641
:10040000F894FA9AF99A0FBE01960895DB018F933A
:100410009F930E945782BF91AF91A29F800D911D23
:10042000A39F900DB29F900D11240895A1E21A2E62
:10043000AA1BBB1BFD010DC0AA1FBB1FEE1FFF1F88
:10044000A217B307E407F50720F0A21BB30BE40BD8
:10045000F50B661F771F881F991F1A9469F760951F
:100460007095809590959B01AC01BD01CF010895D9
:10047000052E97FB1EF400940E944F8257FD07D073
:100480000E94168207FC03D04EF40C944F825095C4
:100490004095309521953F4F4F4F5F4F0895909570
:1004A0008095709561957F4F8F4F9F4F08950E9463
:1004B0006A82A59F900DB49F900DA49F800D911D01
:1004C00011240895B7FF0C9457820E945782821B13
:1004D000930B0895A29FB001B39FC001A39F700D1D
:1004E000811D1124911DB29F700D811D1124911D3C
:1004F000089597FB072E16F4009407D077FD09D0D6
:100500000E94AB8207FC05D03EF4909581959F4FE9
:100510000895709561957F4F0895EE0FFF1F881F16
:100520008BBF0790F691E02D1994692796276927CC
:1005300078278727782708950E946A82332312F448
:100540008A1B9B0B0C94A6820E946A82B7FF0895B7
:10055000821B930B0895AA1BBB1B51E107C0AA1F66
:10056000BB1FA617B70710F0A61BB70B881F991F54
:100570005A95A9F780959095BC01CD0108955058E2
:10058000BB27AA270E94D7820C9451840E944384DF
:1005900038F00E944A8420F039F49F3F19F426F481
:1005A0000C9440840EF4E095E7FB0C943A84E92F18
:1005B0000E94628458F3BA1762077307840795078D
:1005C00020F079F4A6F50C9484840EF4E0950B2EBB
:1005D000BA2FA02D0B01B90190010C01CA01A00195
:1005E0001124FF27591B99F0593F50F4503E68F1F0
:1005F0001A16F040A22F232F342F4427585FF3CF31
:10060000469537952795A795F0405395C9F77EF401
:100610001F16BA0B620B730B840BBAF09150A1F04A
:10062000FF0FBB1F661F771F881FC2F70EC0BA0FD0
:10063000621F731F841F48F4879577956795B79558
:10064000F7959E3F08F0B0CF9395880F08F0992753
:10065000EE0F9795879508950E94168408F481E01F
:1006600008950E9445830C9451840E944A8458F056
:100670000E94438440F029F45F3F29F00C943A84AF
:1006800051110C9485840C9440840E94628468F318
:100690009923B1F3552391F3951B550BBB27AA273B
:1006A00062177307840738F09F5F5F4F220F331F75
:1006B000441FAA1FA9F335D00E2E3AF0E0E832D03D
:1006C00091505040E695001CCAF72BD0FE2F29D040
:1006D000660F771F881FBB1F261737074807AB0712
:1006E000B0E809F0BB0B802DBF01FF2793585F4F87
:1006F0003AF09E3F510578F00C943A840C9485842E
:100700005F3FE4F3983ED4F3869577956795B79568
:10071000F7959F5FC9F7880F911D9695879597F973
:100720000895E1E0660F771F881FBB1F62177307EC
:100730008407BA0720F0621B730B840BBA0BEE1F01
:1007400088F7E09508950E94AA836894B1110C94EB
:10075000858408950E946A8488F09F5798F0B92F85
:100760009927B751B0F0E1F0660F771F881F991FE6
:100770001AF0BA95C9F714C0B13091F00E94848480
:10078000B1E008950C948484672F782F8827B85F90
:1007900039F0B93FCCF3869577956795B395D9F73E
:1007A0003EF490958095709561957F4F8F4F9F4F48
:1007B0000895E89409C097FB3EF490958095709554
:1007C00061957F4F8F4F9F4F9923A9F0F92F96E99D
:1007D000BB279395F695879577956795B795F11112
:1007E000F8CFFAF4BB0F11F460FF1BC06F5F7F4FAF
:1007F0008F4F9F4F16C0882311F096E911C07723C1
:1008000021F09EE8872F762F05C0662371F096E8C9
:10081000862F70E060E02AF09A95660F771F881F98
:10082000DAF7880F9695879597F90895990F00083C
:10083000550FAA0BE0E8FEEF16161706E807F907B2
:10084000C0F012161306E407F50798F0621B730B4D
:10085000840B950B39F40A2661F0232B242B252BCE
:1008600021F408950A2609F4A140A6958FEF811D71
:10087000811D089597F99F6780E870E060E0089512
:100880009FEF80EC089500240A94161617061806A8
:100890000906089500240A94121613061406050684
:1008A0000895092E0394000C11F4882352F0BB0F15
:1008B00040F4BF2B11F460FF04C06F5F7F4F8F4F78
:1008C0009F4F089557FD9058440F551F59F05F3FB3
:1008D00071F04795880F97FB991F61F09F3F79F062
:1008E00087950895121613061406551FF2CF4695E4
:1008F000F1DF08C0161617061806991FF1CF869566
:100900007105610508940895E894BB276627772749
:10091000CB0197F908950E94168408F48FEF08958B
:100920000E94A3840C9451840E94438438F00E9456
:100930004A8420F0952311F00C943A840C9440845E
:1009400011240C9485840E94628470F3959FC1F3F6
:10095000950F50E0551F629FF001729FBB27F00D6D
:10096000B11D639FAA27F00DB11DAA1F649F6627C2
:10097000B00DA11D661F829F2227B00DA11D621F11
:10098000739FB00DA11D621F839FA00D611D221FCB
:10099000749F3327A00D611D231F849F600D211DAF
:1009A000822F762F6A2F11249F5750409AF0F1F032
:1009B00088234AF0EE0FFF1FBB1F661F771F881F9B
:1009C00091505040A9F79E3F510580F00C943A8415
:1009D0000C9485845F3FE4F3983ED4F38695779535
:1009E0006795B795F795E7959F5FC1F7FE2B880F41
:1009F000911D9695879597F90895FA01EE0FFF1FBF
:100A0000309621053105A1F16115710561F4803839
:100A1000BFE39B0749F168949038810561F0803805
:100A2000BFEF9B0741F099234AF5FF3FE1053105F0
:100A3000210519F1E8940894E795D901AA2329F42E
:100A4000AB2FBE2FF85FD0F310C0FF5F70F4A695F8
:100A5000E0F7F73950F019F0FF3A38F49F779F9399
:100A60000DD00F9007FC9058089546F00C944084E8
:100A700060E070E080E89FE308954FE79F775F9321
:100A80004F933F932F930E94FD852F913F914F915C
:100A90005F910E9490840C945A850E941684880B62
:100AA000990B089529F416F00C943A840C948484DC
:100AB0000C9440840E946A84A8F39638A0F707F843
:100AC0000F92E8942BE33AEA48EB5FE70E94A68492
:100AD0000F920F920F924DB75EB70F920E9445860C
:100AE000ECEFF1E00E948C854F915F91EF91FF91C7
:100AF000E595EE1FFF1F49F0FE57E0684427EE0F13
:100B0000441FFA95E1F74195550B0E94BF850F9060
:100B100007FE0C94B3850895DF93CF931F930F9333
:100B2000FF92EF92DF927B018C01689406C0DA2E6F
:100B3000EF010E94A384FE01E894A59125913591CF
:100B400045915591A6F3EF010E94D782FE019701CE
:100B5000A801DA9469F7DF90EF90FF900F911F9151
:100B6000CF91DF9108959B01AC0160E070E080E8D7
:100B70009FE30C9431830C943A840C9479860E9400
:100B80006A84D8F39923C9F3940F511DA3F39150AC
:100B9000504094F059F0882332F0660F771F881F79
:100BA00091505040C1F79E3F51052CF7880F911D81
:100BB0009695879597F908955F3FACF0983E9CF025
:100BC000BB27869577956795B79508F4B16093959F
:100BD000C1F7BB0F58F711F460FFE8CF6F5F7F4F8D
:100BE0008F4F9F4FE3CF0C94858416F00C94798639
:100BF0000C94408468940C943A840E946A84A8F30C
:100C00009923C1F3AEF3DF93CF931F930F93FF921A
:100C1000C92FDD2788232AF02197660F771F881FA9
:100C2000DAF720E030E040E85FEB9FE3883920F01E
:100C3000803E38F021968F770E94C082E4E2F2E095
:100C400004C00E94C082E1E5F2E00E948C858B0125
:100C5000BE01EC01FB2E6F5771097595771F880B4C
:100C6000990B0E94DB8328E132E741E35FE30E94B6
:100C7000A384AF2D9801AE01FF900F911F91CF91EA
:100C8000DF910E94D7820C945184FA01DC01AA0FF3
:100C9000BB1F9B01AC01BF5728F4222733274427F1
:100CA000507820C0B75190F4AB2F0024469537956B
:100CB0002795011CA395D2F3002071F0220F331F5A
:100CC000441FB395DAF30ED00C94BF8261307105E6
:100CD000A0E88A07B94630F49B01AC016627772764
:100CE00088279078309621F0208331834283538384
:100CF00008959F3F31F0915020F48795779567953F
:100D0000B795880F911D9695879597F9089581E07D
:100D100090E0F8940C94C2870F931F93CF93DF93C6
:100D20008C01FC0101900020E9F7CF01801B910BA1
:100D30000E94A777EC01009719F0B8010E94F7868E
:100D4000CE01DF91CF911F910F910895FB01DC013E
:100D500004C08D910190801921F441505040C8F792
:100D6000881B990B08956817790768F4FB01DC016B
:100D7000E40FF51FA40FB51F02C002900E92415060
:100D80005040D8F708950C94B987FB01DC018D9190
:100D900081341CF08B350CF4805E619161341CF061
:100DA0006B350CF4605E861B611189F3990B089515
:100DB000FB01DC010D900020E9F7119701900D92E5
:100DC0000020E1F70895FC018191861721F0882326
:100DD000D9F7992708953197CF010895FB01DC01D8
:100DE0008D91019080190110D9F3990B0895FB01A1
:100DF000DC0101900D920020E1F70895FB01DC0178
:100E00000D900020E9F711974150504028F00190D3
:100E100000200D92C9F708951C920895FB01DC0192
:100E20004150504030F08D910190801919F400200C
:100E3000B9F7881B990B0895FB01DC014150504024
:100E400048F001900D920020C9F701C01D92415059
:100E50005040E0F708950F931F93CF93DF93CDB7E2
:100E6000DEB72E970FB6F894DEBF0FBECDBF0E894A
:100E70001F89888D998D26E02C831A83098397FF1B
:100E800002C080E090E801979E838D83AE01445EAE
:100E90005F4F6A8D7B8DCE0101960E94F87B4D815C
:100EA0005E8157FD0AC02F813885421753070CF425
:100EB0009A01F801E20FF31F10822E960FB6F894F4
:100EC000DEBF0FBECDBFDF91CF911F910F9108956F
:100ED0000F931F93CF93DF93CDB7DEB72E970FB647
:100EE000F894DEBF0FBECDBF0E891F8986E08C83CC
:100EF0001A8309838FEF9FE79E838D83AE01465E41
:100F00005F4F688D798DCE0101960E94F87BEF814D
:100F1000F885E00FF11F10822E960FB6F894DEBF11
:100F20000FBECDBFDF91CF911F910F910895CF9349
:100F3000DF93CDB7DEB72E970FB6F894DEBF0FBEA6
:100F4000CDBF85E08C838C899D899A838983AE018E
:100F5000485E5F4F6E897F89CE0101960E94C17FF6
:100F60002E960FB6F894DEBF0FBECDBFDF91CF91A6
:100F70000895FB01DC0102C001900D9241505040E8
:080F8000D8F70895F894FFCFA3
:100F880003100000C00120000000020C80000100D6
:100F980000005E00BC00770100000000A52A475C45
:100FA800A565962AE42AC22AF22A572BA0650000D2
:100FB80000001D2B475CA565962A5E2B1A2CF22A89
:100FC800572BA06500044D51545404000000000044
:100FD8000000000000000000000000000000000009
:100FE80000000000000000000000000000000000F9
:100FF8000000003031323334353637383941424316
:101008004445460000000000E45C475C715C315DCB
:10101800A25C805C945C00000000E723BA23A5650D
:10102800D541B2239E238F2300000000AD5D8A5D69
:10103800A565A46500000000885D475CA565A465FA
:10104800885D885D885D00000000885D475CA56557
:10105800A46500000000885D885DA565885D885DE1
:10106800885D885D885D885D885D885D885D885D50
:1010780000000000083CB93CA5652042973C7D3C37
:10108800563C443D6A41793CCE43674218422A3C6B
:10109800283C0D421E3C00000000B05E000000002D
:1010A800885D01005E00000000000000D64121427A
:1010B800A565D541EC412A457344CC455D46C043FE
:1010C800CC46DC42F94553450B450442F441F04116
:1010D80000000000DC2B475CA565962A2F2BED2B22
:1010E800F22A572BA065000000001D2B475CA56560
:1010F800962A5E2B0A2CF22A572BA06500000000C6
:10110800B909CA1C4E494C0000000000000000004C
:1011180000000000000000000000000000000000C7
:101128000000000064653A61643A62653A65663AAF
:1011380066653A66650068656C700073617665007F
:101148006C6F616400676574006D6163006B696C46
:101158006C007265710069700070776400636C657B
:101168006172007265626F6F74000D0A005F7374BC
:10117800617400560052504D004900737700666C48
:10118800740073657400707772002F616C61726D02
:101198002F6F76726874002F616C61726D2F736E99
:1011A8007372002F0020004C6F61646564206672C2
:1011B8006F6D20666C6173682049503A0020444E78
:1011C800533A002047573A00204D41534B3A000A02
:1011D8004E6F204950206461746120666F756E649B
:1011E80020696E20666C6173680A002325325825D1
:1011F8003258253258006974656D0073636D640058
:1012080072636D6400656D6974004F4E004F464609
:10121800003B00726F6F7400626373740054005374
:10122800006D61700022006E756C6C0074727565DB
:101238000066616C7365002D002E00252525327827
:101248000057495A6E65740031772054696D656F8F
:101258007574005265736574206572726F72002030
:10126800636F6D705F69642100646D78696E0064F6
:101278006D78006D6F64627573006F7700697465CF
:101288006D7300746F70696373006D7174740025F9
:10129800783A25783A25783A25783A25783A25789B
:1012A80025D181002F726573702F23002F7265710D
:1012B8002F636F6E660031002F253032782D253070
:1012C80032782D253032782D253032782D25303260
:1012D800782D253032782E636F6E6669672E6A73B3
:1012E8006F6E006E616E00696E66006F7666002430
:1012F800636F6D6D616E64002564002C002F616C56
:0C13080061726D6F66662F736E73720069
:00000001FF
